:020000040800F2
:10C00000402E012001800208ED9F0208359E0208A3
:10C01000EB9F0208059202081DAC02080000000018
:10C020000000000000000000000000002FA1020836
:10C0300031930208000000002DA10208F5A30208B8
:10C040001B8002081B8002081B8002081B8002085C
:10C050001B8002081B8002081B8002081B8002084C
:10C060001B8002081B8002081B8002085D920208E8
:10C070001B800208BDC10008B19202081B800208A3
:10C080001B800208F19202081B8002081B80020834
:10C0900081AB02081B800208099202081B8002087B
:10C0A0001B8002081B8002081B8002081B800208FC
:10C0B0005DA402081B8002081B8002081B80020886
:10C0C0001B8002081B8002081B8002081B800208DC
:10C0D0001B80020899AA02080DAB02081B80020807
:10C0E0001B8002081B8002081B8002081B800208BC
:10C0F0001B8002081B8002081B8002081B800208AC
:10C100001B8002081B8002081B8002081B8002089B
:10C110001B8002081B8002081B8002081B8002088B
:10C120001B8002081B8002081B8002081B8002087B
:10C130001B8002081B8002081B8002081B8002086B
:10C1400000000000000000000000000000000000EF
:10C150001B8002081B8002081B8002081B8002084B
:10C160001B8002081B8002081B8002081B8002083B
:10C170001B8002081B8002081B8002081B8002082B
:10C180001B800208DFF80CD000F006F800480047DA
:10C190007F4E0308402E0120064C074D06E0E06864
:10C1A00040F0010394E8070098471034AC42F6D3FE
:10C1B000FFF7ECFF849E0108A49E010810B54FF420
:10C1C0000074204623F004F9002819D0204623F0FB
:10C1D0006FF80C4814F0A6FE0B4C802120682BF061
:10C1E000C4FF0028F9D1002108482BF0B9FF002135
:10C1F000074823F047F8BDE8104001201DF0CABEF3
:10C2000010BD00003C9600209C350020003001400D
:10C210003000024002E008C8121F08C1002AFAD10B
:10C2200070477047002001E001C1121F002AFBD1B6
:10C230007047000010B5442107480EF0CAFB0022E9
:10C24000062106480BF04AFF054CA06000F074FB85
:10C250000020207010BD000030980020EDC90008BB
:10C26000E8370020F8B5044618F0F0FF0026374DF7
:10C270000746009634B1E068686020460BF0FCFF8A
:10C28000686802E014F054FE686000690BF0D2FDAB
:10C290006868406908B10BF0CDFD6868C0690BF0B3
:10C2A000C9FD6868006A0BF0C5FD6868016991B155
:10C2B0000BF05CFE0CF06EFE0CF0BCFC6868B0F895
:10C2C0005011D9B30068017CC9071DD0C06840680F
:10C2D000D0B1002413E0A0F85061F8BD011991F825
:10C2E000301151B900F5AC700EF0CAFB696801EB72
:10C2F000C4010A6B0260496B4160641CA4B26868A7
:10C30000B0F85011A142E9D868684FF4807130301C
:10C310001BF0E7FE6868202100F598701BF0E1FE35
:10C320006868A0F85061384618F089FF0090686886
:10C330000068436A13B12A680099984717F050F9CA
:10C340000EF01AF8BDE8F84000F002B8603700209F
:10C3500070B5094E0024C4EBC40556F8250008B199
:10C3600017F0B2F906EB85001C2108F056FA641CA0
:10C37000E4B2042CEFD370BD4C9900207FB50D467C
:10C38000040003D114F0D4FD04002CD014F044FEBA
:10C39000002828D094F82800400724D4002605B3AC
:10C3A000ADF80060ADF80260204614F0D9FD401EE3
:10C3B000ADF80400204614F019FE401EADF806004A
:10C3C0006A46294602A80DF024FE00280BD02068FA
:10C3D000017C890708D5DDE90001C4E90C010120D1
:10C3E00029E0A4F850617FBD82690AB102A9904793
:10C3F00000250AE004EBC501002202A830310DF04F
:10C4000030FE0028EFD16D1CADB2B4F85001A84247
:10C41000F0D880B2202804D204EBC00002A930304A
:10C4200004E0A4F8506104F13000694605F08AF98F
:10C43000B4F85001401CA4F8500160680028D2D024
:10C440000BF02CFF7FBD10B50446006882680AB16E
:10C450002146904720680068002801D02060F5E759
:10C4600010BD8068002801D0B0F9160070478068C0
:10C47000002801D0807E8009704770B515460646B9
:10C480000C4651EA05001AD0304608F073FAB0683D
:10C4900001232A46018A21440182B068418A294445
:10C4A0004182214630460AF05BFB00220B213046D8
:10C4B00014F038FE012803D130460AF0ABFA01200F
:10C4C00070BD77B581B00E46050017D0622209F025
:10C4D000A4FE040012D0206880B1284631466322B1
:10C4E00009F09BFE10F0FF0208D023682046039954
:10C4F00098470090BDF80000ADF80C00039804B018
:10C5000070BD00002DE9F047054692B0408C1A9CA2
:10C5100040F00800688490462A8499468A46228919
:10C52000284609F07AFE0646A5F820902289514651
:10C53000284609F072FE0746688CBE4220F00800CB
:10C54000688403D13104B1EB074F68D0A5F820808F
:10C5500022895146284609F060FE06468046A5F825
:10C5600020905146284604F094FC21890068324608
:10C5700018F060FA20890B2823D147F6FF794E4541
:10C5800001D04F451DD1284609F093FF00EBD07034
:10C590004610284609F081F800EBD0704010C845DD
:10C5A00006D1711C431C994200DA00E01946884606
:10C5B0004F4506D1711C421C914201DA0F4600E042
:10C5C000174619480EF00DFA06002BD03560C6E963
:10C5D00003872089B0806846C6F808A004F0D8FF19
:10C5E0001248FF21CDE900601148029011480390E4
:10C5F00000200890CDE9090120880B9060889DF803
:10C60000421040420C90E0680790002060F3000167
:10C610008DF8421020690690684605F043F812B084
:10C62000BDE8F087FEE7000054980020A5980108B7
:10C63000A99A0108019A0108142101480EF0C9B90C
:10C64000549800202DE9F84F00249046894606466C
:10C6500025464FF0040AE3E0F1680AEBC5000858EC
:10C6600082017AD480B230EA090210D0002230EA86
:10C6700008000ED0002082426FD051F835706A4613
:10C680001021384617F0D2FF002871D103E00122B3
:10C69000EDE70120EFE76A461121384617F0C6FFA3
:10C6A000002865D16A461221384617F0BFFF0028DE
:10C6B0005ED16A461321384617F0B8FF002857D1DB
:10C6C0006A461521384617F0B1FF002850D16A4656
:10C6D0001421384617F0AAFFF0BB6A460A213846F3
:10C6E00017F0A4FFC0BB6A466B21384617F09EFFC7
:10C6F00090BB6A466C21384617F098FF60BB6A46CB
:10C700000121384617F092FF30BB6A4604213846B3
:10C7100017F08CFF00BB6A460221384617F086FFEF
:10C72000D0B96A460321384617F080FFA0B96A469F
:10C730000521384617F07AFF70B96A460621384657
:10C7400017F074FF40B96A463221384617F06EFF81
:10C7500010B96A466E2101E00AE060E0384617F041
:10C7600065FF28B96A466D21384617F05FFF10B1A2
:10C770000320BDE8F88F6A466921384617F056FF56
:10C78000F0BB6A466A21384617F050FFC0BB6A46C4
:10C790006E21384617F04AFF90BB6A466D21384635
:10C7A00017F044FF60BB6A463721384617F03EFF5A
:10C7B00030BB6A463821384617F038FF00BB6A465E
:10C7C0003521384617F032FFD0B96A464021384645
:10C7D00017F02CFFA0B96A464521384617F026FF0E
:10C7E00070B96A464121384617F020FF40B96A46C1
:10C7F0004221384617F01AFF10B96A46432100E07B
:10C8000009E0384617F012FF28B96A464921384630
:10C8100017F00CFF08B1022401E004B901246D1CDB
:10C82000708CC0F30510A8423FF616AF2046A0E773
:10C8300001484068704700006037002070470000E2
:10C8400010B5182103480EF0C4F803490120087000
:10C8500010BD000000980020303800202DE9F84F6E
:10C860008146407A0D4600F00700022819D0104694
:10C870008046954200DD2A46164603202A4F2B4B60
:10C8800000EB460020F00304B86819681034411A20
:10C890007A6804EB010C944505D2416821F000410F
:10C8A00024E00846E4E7944219D89A464FF0FF3B4B
:10C8B00008197968884210D9002269461C48CDF8C9
:10C8C00000B004F05BFB002269461A4804F056FBF6
:10C8D000B968DAF80000091AEAE7B868DDE7204627
:10C8E00016F066FEC0B1416841F0004188EA650279
:10C8F000416089EA02010160416801F04041491C40
:10C9000031F0804141608681A0F80E8005D500F1AC
:10C9100010018160BDE8F88FFEE7B96801F11002EF
:10C9200021448260B960F5E76837002010380020A4
:10C93000430A0108F90F010810B5084C01202070C6
:10C9400007480EF029F80028A06803D0BDE8104081
:10C950000BF0A4BCBDE810400BF08EBCE837002003
:10C960003098002010B5044690F84200A16B820771
:10C9700009D4B4F840204AB1A2F57F43FF3B1BD055
:10C98000521EA4F84020B4F84020AAB909B1820789
:10C9900012D5214614480EF09AF8FFF7CDFFE16852
:10C9A00009B120468847216909B1204688472046B9
:10C9B000BDE8104016F088BEE26B524222630029A7
:10C9C00011D0820702D4626B524222634210521C81
:10C9D00062F3410084F84200A26A206A2262A062E7
:10C9E000E06AE162A06310BD3098002070B5304E5F
:10C9F000706818F024FC0546707880F001007070B3
:10CA000047E00020307094F842007178C0F3800253
:10CA10008A4242D061F3820084F84200216B4A19B5
:10CA2000030719D4002917DC002A15DBC00709D138
:10CA3000616939B120468847216A01442162A16AAF
:10CA40000844A062A16809B12046884794F84200D2
:10CA500040F0080084F84200206B4019206316D48F
:10CA6000E16A884200DD2163E1692046884701468A
:10CA7000606A884204D0616262680AB120689047A7
:10CA8000D4E90B01814202DB2046FFF76BFF3078CF
:10CA900018B108480DF080FF03E0214605480DF06D
:10CAA0008DFF0400ADD118F0D1FB706070BD0000A7
:10CAB000E8370020309800202DE9FF4F8BB01E464C
:10CAC000DDE91801CDE90601002004901F981E9DA4
:10CAD000042809D0052809D006280CD014287CD1B8
:10CAE00001200290022004E00020FAE701200290D9
:10CAF0000320059008E00120029002200590FFF736
:10CB000097FE0068806B04900D98002416FB00F0DF
:10CB10000A900C98401E09900D98401E08902CE138
:10CB20001A980699604301EB20231B9807996043EC
:10CB300001EB202219124FEA222007D40C9FB942A0
:10CB400004DA002802DB0D9FB84201DB002011E16E
:10CB5000DBB2D2B2802B05DAC3F17F034FF0FF378F
:10CB60005B0003E001275B00A3F580739A46802AEF
:10CB700005DAC2F17F024FF0FF33520003E00123D8
:10CB80005200A2F58072914600FB0618DDF814C031
:10CB90000B9A08FB0C2201EB070C5FEA0C0E73D416
:10CBA000DDF82480C6456FDC10EB03086CD4DDF89B
:10CBB00020C0E04568DCDDF814C017FB0C2B13FB2C
:10CBC00006F707FB0C23029FF7B31F9F052F05D025
:10CBD000142F09D0062F47D053E0D2E092F802C0BC
:10CBE00099789BF8020010E0DDE90A7C0CEB47071E
:10CBF000394400FB06FC00FB067708FB06F81CF82E
:10CC000001C017F80E0018F80110614507D011FB9C
:10CC100009F7C9F580711CFB0171C1F3072160455B
:10CC200007D010FB0AF7CAF580701CFB0070C0F338
:10CC3000072008444008285556D01078517800EB5A
:10CC40000120ADF8000000E01FE01878597800EBF3
:10CC50000120ADF80C009BF800109BF8010001EBDF
:10CC60000020ADF804001CE00498118880B28142D5
:10CC70003FF46CAF19888142FAD0BBF800108142B2
:10CC8000F6D0FF210846D4E72FE01088ADF8000069
:10CC9000BBF80000ADF804001888ADF80C00FF20C8
:10CCA0002855BDF80000BDF80C10884203D1BDF82E
:10CCB0000410884212D009F0FF020099039804F092
:10CCC000A5FE0390DDE900100AF0FF0204F09EFECD
:10CCD0007F220190039904F099FE00901D98BDF801
:10CCE000001000EB4400018045E092F800C092F88B
:10CCF00001800CEB082C1FFA8CF8DDF874C02CF8BE
:10CD00001480DDF87CC0BCF1050F06D0BCF1060F25
:10CD100005D0BCF1140F08D109E092780FE0049A15
:10CD200092B2904501D1002209E0FF2207E00B9A60
:10CD300000FB062C0A9A01EB42021CF8022009B9FA
:10CD4000002F05DBDDF824C0614504D1002F02DD92
:10CD5000CAF1FF000BE008B9002B06DB08998842F6
:10CD60007FF4F4AE002B7FF7F1AEC9F1FF0010FBAA
:10CD700002F0000A2855641C24B21C988442FFF675
:10CD8000CFAE0FB0BDE8F08F2DE9F05F00228046F6
:10CD900011460AF081FD0021404609F0A6F904463B
:10CDA0000021404609F02DFA204407B200214046F8
:10CDB00009F003FA20440FFA80FB404609F03EF9DF
:10CDC000C11901EB0B000FFA80F9274C404608F01F
:10CDD000B1FB824600252BE0D8F808002349006803
:10CDE00050F82560304609F08AFB00BB304609F058
:10CDF00069FE60BB0021304609F044F938B30128D0
:10CE000025D0022823D0032821D00021304609F064
:10CE100097FA60B906F11400064604F0C0FC3844E5
:10CE2000A04203DB304604F0BAFCC41924B26D1CE6
:10CE30005545D1D341F6FF70C44212D004EB0B002C
:10CE400000B24946484500DC0846BDE8F09FB6F907
:10CE50001A10B8F91600081A411CA142E6DB0C466C
:10CE6000E4E74846F1E7000001E0FFFF01000400AD
:10CE70002DE9F05F0022054611460AF0F7FC00217B
:10CE8000284609F032F904460021284609F0ADF998
:10CE900020440FFA80F90021284609F09AF920442D
:10CEA0000FFA80F8284609F0D7F800EB080101EBEB
:10CEB00009000FFA80FB4B4C284608F03BFB8246EA
:10CEC0000021284609F0E4F801284FF000062CD094
:10CED0006AE0A8684449006850F82670384609F0AE
:10CEE0000EFB08BB384609F0EDFD38BB0021384683
:10CEF00009F0C8F810B3032820D006281ED008284F
:10CF00001CD00021384609F015FA68B907F1140061
:10CF1000074604F062FC4844A04204DB384604F0B3
:10CF20005CFC00EB090424B2761C5645D1D341F6D3
:10CF3000FF70C44241D004EB08003DE0B5F9180091
:10CF4000B7F91410401A411CA142ECDB0C46EAE789
:10CF5000A8682549006850F82670384609F0CFFACD
:10CF600008BB384609F0AEFD88BB0021384609F001
:10CF700089F860B301282BD0042829D0072827D0AE
:10CF80000021384609F0DCF968B907F114000746BA
:10CF900004F023FC4044A04204DB384604F01DFCAE
:10CFA00000EB080424B2761C5645D1D341F6FF703D
:10CFB000C44202D004EB090004B241F6FF70C4423F
:10CFC000584602D05C4500DD2046BDE8F09FFFE7F3
:10CFD000B7F91800B5F91410401A411CA142E1DB61
:10CFE0000C46DFE701E0FFFF010004001CB50B88E1
:10CFF00004892344ADF800304B8844892344ADF8BC
:10D0000002308B8804892344ADF80430C9884389F1
:10D010001944ADF806104369694698471CBD2DE9CF
:10D02000F04F8BB05FEA010A054643D0A5F818A07F
:10D03000286808B116F048FB0AEB4A00062101EB0C
:10D04000400016F0B5FA286058B3022202EB4A01FC
:10D0500001440422E96002EB8A010144C5E90101AF
:10D0600001210024BAF1010F1CD04FEACA00083098
:10D0700016F0CCFA064600EB8A074FEA8A0000B2A7
:10D08000ADF80000C0F101022146ADF80240801069
:10D09000A146A346ADF824204C463F1D01910590C2
:10D0A000B3E0FEE7B4220270E8680480E8684180DB
:10D0B000A86804800BB0BDE8F08F4FF00008BDF900
:10D0C0002400002808DCBDF80210032202EB410115
:10D0D0000844ADF824000DE0BDF80220BDF80010B2
:10D0E0000523521A03EB42021044491EADF82400F6
:10D0F000ADF80010BDF80200401CADF80200684613
:10D1000000F0F0F878B1BDF9000005AB821043F8EB
:10D11000282001AA00F0030142F8281008F10108B4
:10D12000B8F1040FCBDBB8F1040F74D1089905985E
:10D13000884212D126F8140027F81490DDE9010185
:10D140000844DDE903121144084469680855696818
:10D1500000010855641C24B255E00699884219D094
:10D1600026F8140027F814906A68019810556A6828
:10D1700000011055641C059A20B2521E26F810209A
:10D1800027F81090DDE902120A440499091D1144A0
:10D190006A6832E0079926F814008842494627F861
:10D1A000149015D0DDE9012010446A6810556A68B2
:10D1B00000011055641C059A20B2521E26F810205A
:10D1C00027F81010DDE90312114408316A6814E0F1
:10D1D000DDE901021044039A10446A6810556A6838
:10D1E00000011055641C059A20B2521E26F810202A
:10D1F00027F8101004996A680C3111546A68090103
:10D200001154401C04B209F10109684600F06AF8A3
:10D2100000287FF452AF40F2D3211AFB01F106EB54
:10D220004402881232F9022C824205D107EB4402F3
:10D2300032F9022C82421AD0A1EB8021B1F5007F95
:10D2400003DC494341F3CF3106E0C1F58061494336
:10D2500041F3CF31C1F10F0126F8140027F8140073
:10D2600068680155686809010155641C24B2A01E54
:10D270000DE037F8101026F8141036F8101027F8C3
:10D28000141069680A5C0A55641C24B2401E002808
:10D29000EFDAEB6800210846A3F800B01CE0EA686A
:10D2A00022F81100AB6836F8102023F811200BE0AB
:10D2B000D5F808C036F910303CF811209A4200DB4E
:10D2C0001A462CF81120401C37F910208A4201D14F
:10D2D000A042EDDB491C09B2A042E0DB304616F06B
:10D2E000E1F9E7E6B0F90210B0F90000814201DC93
:10D2F000012070470020704717B581B0022ABDF8A1
:10D30000080036D9BDF80410C0F3C403C1F3C40447
:10D3100023441F2B00D31F2363F3C70143079B0E36
:10D3200003EB503301F0070403EBC40303EB513369
:10D33000ADF804103F2B00D33F23DC0864F3020157
:10D3400063F34F31C0F30420C1F304231844ADF854
:10D3500004101F2800D31F2060F30C21ADF8041027
:10D36000FF2A08D0DDE9010104F02AFB0090BDF896
:10D37000000004B010BD88B2FBE717B581B0022AE7
:10D3800003D8BDF8080004B010BDBDF80410BDF806
:10D390000800C1F3C403C0F3C40413FB04F35B0926
:10D3A00063F3C701C1F30423C0F3042413FB04F3A4
:10D3B0005B0963F30C214B079B0E4407A40E03EBA0
:10D3C000513304EB503013FB00F35B0A63F30201AB
:10D3D0004B079B0E03EB513313FB00F0800960F306
:10D3E0004F31ADF80410FF2A07D0DDE9010104F048
:10D3F000E7FA0090BDF80000C5E788B2C3E717B5AB
:10D4000081B0022ABDF8080036D9BDF80410C0F377
:10D41000C403C1F3C4041B1B002B00DC002363F313
:10D42000C70143079B0E03EB503301F0070403EBE6
:10D43000C40303EB5133ADF80410002B00DC0023D0
:10D44000DC0864F3020163F34F31C0F30420C1F33D
:10D450000423C01AADF80410002800DC002060F39B
:10D460000C21ADF80410FF2A08D0DDE9010104F019
:10D47000A7FA0090BDF8000004B010BD88B2FBE729
:10D480002DE9FF4F83B00746DDF84080DDE91365E5
:10D490004FEA4800DDF848A000B2049C0190BAF1C0
:10D4A000040F1DD0BAF1060F1AD0BAF1050F5AD0E9
:10D4B000BAF1140F54D1B7F90010B7F9022008FBE4
:10D4C000021004EB4009384604F07BF983463846E5
:10D4D00004F09BF9044640004FF0000A009084E0FD
:10D4E000384612F078FD014600902846FF221AF0D7
:10D4F000F1FDB7F90010B7F9022008FB021004EBA8
:10D500004008384604F081F98346400002903446D2
:10D51000B7F902000BE020464146029A1AF0B9FD25
:10D52000019909F10100884404EB4B0400B2B7F9FA
:10D53000061081464945EEDABAF1060F10D14EF2D7
:10D5400007000021ADF804000246084605E036F861
:10D550001030934200D12954401C009B9842F6D3CE
:10D5600007B0BDE8F08FB7F90010B7F9022008FB4B
:10D57000021000EB40000444384604F046F9A8EBE2
:10D58000000000EB40000FFA80F8384604F019F96B
:10D590008146384604F039F90146002215E00020A2
:10D5A0000BE0A3782B5414F8013B14F8027B03EB37
:10D5B000072326F81030401C00B28842F1DB521CD1
:10D5C00006EB41060D44444412B24A45E7DBC7E787
:10D5D00030464946009A1AF05CFD01990AF10100B3
:10D5E00006EB440689440FFA80FADA45F0DBDDE900
:10D5F00004014A000699B7F9023002FB0100B7F9AD
:10D60000002008FB03210E18002708E028463146B9
:10D6100022461AF03EFD7F1C254446443FB25F453A
:10D62000F4DB9DE72DE9F04F0646C87A89B0154630
:10D630000F46022803D8012009B0BDE8F08F184634
:10D640003A69B9680CF05CFF041EF5D0207D00F04B
:10D650001F0007F06DF84FF4807808B1062010E045
:10D66000207D00F01F000E2806D0142809D007F0F6
:10D670004FF840B1052004E038884FF00E0938B962
:10D6800003E0814608E00420FBE77888404503D0AA
:10D6900000204FF00509A061226A22B129463046D8
:10D6A0000CF0D9F8B7E0A069F0B3294602A804F05D
:10D6B00052F8B7F9003013B97888404529D0A888C6
:10D6C00029886A88401A401C01B2E88807F1040CD6
:10D6D000801A401C02B27888CDE9000C02A80CF038
:10D6E00059FEBDF8080029880844ADF80800BDF8C7
:10D6F0000A0069880844ADF80A00BDF80C002988C2
:10D700000844ADF80C00BDF80E0069880844ADF877
:10D710000E0002AA04A8B1680CF07BFC00287AD0A5
:10D7200004A8D6F8088000E00BE0B060CDF80090C7
:10D730002A4639463046A36904F0F4FBC6F808804F
:10D7400069E02A4603A8B1680CF063FCF0B3BDF8A9
:10D750001000BDF80C10401A401C0FFA80FA0AEBBA
:10D760004A0015F053FF059003A901A8D6F808B0A8
:10D7700003F0F1FF012101A812F07AFCBDF90C00C1
:10D78000B5F90010401A0890BDF90E80B5F90200F5
:10D79000A8EB000536E001AA594606A80CF039FCB2
:10D7A00070B3059800900898534601B22AB22046FB
:10D7B00014F066FE01280ED0204614F0B6FD059840
:10D7C00015F070FF204614F0B0FD00E023E00020CB
:10D7D000C6F808B030E706A8B060CDF8009001AAFE
:10D7E00039463046059B04F09DFBBDF80600401C01
:10D7F000ADF80600BDF80A00401CADF80A006D1C2B
:10D8000008F10108BDF912004045C4DAC6F808B0B5
:10D81000059815F047FF204614F087FD0BE7000040
:10D820001CB50C4814460078002812D088880A8855
:10D830004B88801A401C82B2C888C01A401C83B230
:10D8400050005843CDE900404C88088821461BF021
:10D85000A0FD1CBD243700202DE9F74FC87898B0F3
:10D860000C4602287ED911460AA803F08FFFB4F9AE
:10D870002000012829DD94F82200FD2825D32088E6
:10D8800018B394F82300BDF828104008C0F38002B4
:10D890001144ADF82810BDF82A10C0F34000084428
:10D8A000ADF82A0094F82310BDF82C004908C1F304
:10D8B000C001401AADF82C0094F82310BDF82E00DA
:10D8C000C1F34001401AADF82E0018980AA98268E9
:10D8D0000CA80CF09EFB00287ED0E07B10F0070522
:10D8E00019D0E088ADF80000BDF8000061898842D9
:10D8F00000D100250AA805F06FF807461C2103A8EF
:10D900001AF0EFFBA0788DF82500BDF80000ADF807
:10D9100014001FB105E060680090E5E7208800B9B9
:10D92000F5B3E078FD2800D3FF2083460AA803F072
:10D9300078FF81460AA803F04AFF06464846B145EB
:10D9400000DB3046B4F90010B1EB600F00DB411092
:10D9500088460CA803F065FF82464FF0FF30169012
:10D96000002000E038E00090B8F1000F00DC77B153
:10D97000504615F04BFE0090002342460AA90EA81F
:10D9800005F094FA00210EA804F036FE1690BDF8BA
:10D990003000ADF80400BDF83400ADF8080000E038
:10D9A00011E00098069001A803900890FF208DF8E0
:10D9B000240032464946A01D06F028FE060018D075
:10D9C000022D0CD015E00AA80390E0788DF8240011
:10D9D00003A9189805F029FD1BB0BDE8F08FBDF92B
:10D9E0003010B06800EB4100BDF92810A0EB4100F9
:10D9F00004907FB3BDF9324027E027B2ADF806703E
:10DA0000ADF80A7052465946009806F001FFBDF97C
:10DA1000301053463A46009804F0A0FF8DF81C00E1
:10DA2000012802D102208DF81C00012D08D1BDF97A
:10DA30002A10B068611A00EB41000088ADF81400AC
:10DA400003A9189805F0F1FC641CBDF93600A0424A
:10DA5000D3DABCE0FFE7002054E0BDF82A1001EB68
:10DA60000900BDF82E1004B2A1EB090007B2BDF900
:10DA70003200A04203DDBDF93600B84240DB524619
:10DA80005946009806F0C4FEBDF9041053462246DC
:10DA9000009804F063FF8DF81C00012802D10220D9
:10DAA0008DF81C00BDF93200A04212DCADF8064032
:10DAB000ADF80A40012D08D1BDF92A10B068611AED
:10DAC00000EB41000088ADF8140003A9189805F098
:10DAD000ACFCBDF93600B84212DBADF80670ADF80B
:10DAE0000A70012D08D1BDF92A10B068791A00EB2F
:10DAF00041000088ADF8140003A9189805F095FCC2
:10DB000009F1010081464045A7DBBDF82800ADF8CA
:10DB10005000BDF82C00BDF82A10ADF8540001EB00
:10DB20000800BDF82E10ADF85200A1EB0800ADF8CA
:10DB3000560014A804F050FF074628430DD0BDF945
:10DB40002E100120A1EB0809BDF92A108DF824B090
:10DB50008DF81C0001EB080437E0BDF82A108DF8A1
:10DB600024B001EB0800ADF80600BDF82E10A1EBC3
:10DB70000800ADF80A000020069003A9189805F0E7
:10DB800054FC24E06FB152465946009806F040FE1E
:10DB9000BDF93010534622B2009804F0DFFE8DF834
:10DBA0001C00ADF80640ADF80A40012D08D1BDF9C2
:10DBB0002A10B068611A00EB41000088ADF814002B
:10DBC00003A9189805F031FC641C4C45DADD009877
:10DBD00008B115F067FD1698401C05D0169805F0A1
:10DBE0000FFA0EA804F0DCFE002E3FF4F5AE30462E
:10DBF00006F005FDF0E62DE9F0410646086990B013
:10DC000015460C4600287DD0A07E02287AD92946E8
:10DC10000DA8B2680CF0FDF9002873D00DA8D6F855
:10DC20000880B060206906F08BFD022806D001A9AB
:10DC3000206914F09BFB012849D0C9E0002741F678
:10DC4000FF70CDE900700297D4E904123B460FA89B
:10DC500017F0E6FC284603F0E4FD01462A88BDF9EA
:10DC60003C0001EBD17102EB610100EBD072A1EB42
:10DC700062010844401EADF83000ADF82C10284673
:10DC800003F0A5FD01466A88BDF93E0001EBD171A4
:10DC900002EB610100EBD072A1EB62010844401E6F
:10DCA000ADF83200ADF82E1003A804F0F1FB606966
:10DCB0000390208BADF81800A07E8DF82600009709
:10DCC0000BAA03A93046236904F04EF980E004A8AA
:10DCD00004F030F9A0788DF81C00208BADF8180006
:10DCE000E07E8DF81A00A07E8DF81B00207F4FF09B
:10DCF000FF3740B101996888ADF80A0007EB515130
:10DD000008445DE066E0284603F08BFD298800EBBF
:10DD1000D07001EB60000199C1F38A21A0EB5100A2
:10DD2000ADF80800284603F052FD698800EBD0707A
:10DD300001EB60010198A1EB9051C0F38A22ADF88C
:10DD40000A10BDF80830521E1A4407EB5050ADF8C7
:10DD50000C200844ADF80E0002AA04A9304623693D
:10DD600004F0B4F834E001992888C1F38A21ADF8B1
:10DD70000800491E084410E002AA04A9304623699D
:10DD800004F0A4F80198BDF80810C0F38A200144FB
:10DD9000ADF80810BDF80C100844ADF80C00BDF942
:10DDA0000800B5F904108842E6DDBDF80A100198B4
:10DDB00001EB5051ADF80A10BDF80E1001EB5050B8
:10DDC000ADF80E00BDF90A00B5F906108842CADDAB
:10DDD000C6F8088010B0BDE8F0812DE9F04180461A
:10DDE00091F8220086B00C461646022868D9208C8D
:10DDF000002865D094F8230010F03E0F60D0C007D3
:10DE00005ED1104603F00DFD0746304603F0DFFCFF
:10DE1000B4F90050874200DA3846B5EB600F00DDF8
:10DE20004510314604A803F0B1FC94F82300BDF975
:10DE30001020C0F344014807B4F9200001D428445D
:10DE400040421044ADF810000807BDF91420B4F9A1
:10DE5000200001D428444042101AADF8140094F870
:10DE60002300BDF9121040088007B4F9200001D446
:10DE7000284440420844ADF8120094F82300BDF94C
:10DE800016104008C007B4F9200001D128444042D0
:10DE9000081AADF81600208C281A01B2002900DA01
:10DEA0000021A27894F82200CDE90202E08BADF8BF
:10DEB000040000912B4604AA3146404600F003F8C6
:10DEC00006B0BDE8F0812DE9FF4FA3B01F46DDE9A4
:10DED000326ADDF8C08015460C46FF2E00D3FF26BF
:10DEE000084604F079FD8146384350EA08006DD0B9
:10DEF00023982146826803A80CF08BF800286CD088
:10DF000003A803F08EFC02901C2108A806F089FCEF
:10DF1000029815F07BFB0B904FF0FF300090002F24
:10DF20000ADD00233A46214616A804F0BFFF00216F
:10DF300016A804F061FB00900123424629461CA864
:10DF400004F0B4FF00211CA804F056FB01900FA8B8
:10DF500008900D90BDF8C4008DF83860ADF8280029
:10DF60008DF839A0B4F90000B5F9001038448842A2
:10DF700000DC0846ADF85000B4F90400B5F904100F
:10DF8000C01B884200DB0846ADF85400B4F902001B
:10DF9000B5F902103844884200DC0846ADF852005A
:10DFA000B4F90600B5F90610C01B884200DB08462C
:10DFB000ADF8560014A803F034FC0146B4F9020091
:10DFC000B5F9022090420BDC01200AE000962A46B7
:10DFD0002146319B239800F0D0F927B0BDE8F08F9F
:10DFE00000208046B4F90600B5F90620904201DB16
:10DFF000012600E00026B9F1000F44D0BDF80C0066
:10E00000ADF83C00BDF81000ADF84000BDF90E4081
:10E0100022E0B8F1000F03D1BDF95200A0421ADC92
:10E020001EB9BDF95600A0421ADB25B2ADF8425028
:10E03000ADF83E5002990B9806F0F8FBBDF90C10B4
:10E040002A46029B0B9804F089FC8DF8300008A941
:10E05000239805F0EAF9641CBDF91200A042D8DA51
:10E060001CA804F09DFC019804F0CAFF0098401C15
:10E0700005D016A804F094FC009804F0C1FF0B989A
:10E0800015F010FBA9E7B4F90000B5F900209042A3
:10E0900001DC012000E000208146B4F90400B5F95C
:10E0A0000420904201DB012000E00020824609EAC2
:10E0B0000A0202EA08024FF0010B324203D0322971
:10E0C00001DA4FF0000B01208DF8300018EA0B0F39
:10E0D00012D0BDF85000ADF83C00BDF85400ADF8CA
:10E0E00040006088ADF83E00688808A9401EADF881
:10E0F0004200239805F099F916EA0B0F12D0BDF8EB
:10E100005000ADF83C00BDF85400ADF84000E88880
:10E1100008A9401CADF83E00E088ADF84200239805
:10E1200005F083F9B9F1000F12D02088ADF83C005A
:10E13000288808A9401EADF84000BDF85200ADF88F
:10E140003E00BDF85600ADF84200239805F06DF989
:10E15000BAF1000F12D0A88808A9401CADF83C0005
:10E16000A088ADF84000BDF85200ADF83E00BDF803
:10E170005600ADF84200239805F057F9BDF80C00A1
:10E18000BBF1000FADF83C0008D0BDF95000BDF95F
:10E190001010421E914248DA084647E0BDF81000D0
:10E1A000ADF84000B5F90200B4F90210401AB842C7
:10E1B00000DB07460FFA87F8002533E06088284423
:10E1C00006B2E088401B07B2BDF90E00B04203DD85
:10E1D000BDF91200B84224DB02990B9806F026FB29
:10E1E000BDF93C103246029B0B9804F0B7FB8DF84A
:10E1F0003000BDF90E00B04207DCADF83E60ADF86E
:10E20000426008A9239805F010F9BDF91200B84240
:10E2100007DBADF83E70ADF8427008A9239805F011
:10E2200004F96D1C4545C9DBA0E0401EADF8400077
:10E230000FA803F0F6FA051E41DD59EA08001DD0CB
:10E24000BDF90E4016E027B2ADF84270ADF83E7051
:10E2500029460B9806F0EAFABDF93C102B463A46DF
:10E260000B9804F07BFB8DF8300008A9239805F08B
:10E27000DCF8641CBDF95200A042E4DC59EA060057
:10E280001DD0BDF9564015E027B2ADF84270ADF88B
:10E290003E7029460B9806F0C9FABDF93C102B4692
:10E2A0003A460B9804F05AFB8DF8300008A92398E1
:10E2B00005F0BBF8BDF91200641CA042E4DABDF918
:10E2C0005400BDF90C10421C914201DD084600E0EB
:10E2D000401CADF83C00BDF81000ADF840000FA8A0
:10E2E00003F09FFA051E41DD5AEA08001DD0BDF972
:10E2F0000E4016E027B2ADF84270ADF83E702946E8
:10E300000B9806F093FABDF93C102B463A460B9851
:10E3100004F024FB8DF8300008A9239805F085F857
:10E32000641CBDF95200A042E4DC5AEA06001DD08C
:10E33000BDF9564015E026B2ADF84260ADF83E603A
:10E3400029460B9806F072FABDF93C102B4632466E
:10E350000B9804F003FB8DF8300008A9239805F012
:10E3600064F8BDF91200641CA042E4DA1CA804F0B1
:10E3700017FB019804F044FE7BE62DE9FF478AB0C5
:10E380000C46824615461C216846169E06F049FA40
:10E3900007A80090BDF83400ADF808008DF81860AB
:10E3A000B4F90200B5F90210884201DC012700E04F
:10E3B0000027B4F90600B5F90610884201DB0126F2
:10E3C00000E00026B4F90000B5F90010884201DC35
:10E3D000012100E000218846B4F90410B5F90420B9
:10E3E000914201DB012100E00021ADF81C00A08872
:10E3F000ADF820006088ADF81E0068888946401E90
:10E40000ADF822001FB16946504605F00EF8E888C5
:10E41000401CADF81E00E088ADF822001EB1694630
:10E42000504605F002F82088ADF81C002888401EF0
:10E43000ADF8200017B1B5F9020001E0B4F902000F
:10E44000ADF81E0016B1B5F9060001E0B4F90600FA
:10E45000ADF82200B8F1000F03D06946504604F031
:10E46000E4FFA888401CADF81C00A088ADF820008F
:10E47000B9F1000F03D06946504604F0D6FF0EB044
:10E48000BDE8F0872DE9F0412F4F0646786812F07D
:10E4900063FD04463068C56B696B09B1284688473F
:10E4A000786800680188408811FB00F0E1688842C4
:10E4B00001D1012000E00020216859B1616849B113
:10E4C00028B107E078680068816A01B1884720694F
:10E4D0000028F7D10121216178680068C06882694D
:10E4E000D20704D08069800701D5616101E0002076
:10E4F0006061606908B1012700E000273068416968
:10E5000071B1016911F0300F06D0490704D5D5E982
:10E51000001000F01BF803E0D5E90021FEF766FDCE
:10E52000206800280BD06168002908D03268127C6E
:10E53000BA43D20703D1A268824202D1A160BDE8EA
:10E54000F081A060FBE70000603700202DE9F34F69
:10E550000446854887B041680D682869820701D55F
:10E5600042076FD4C0F30110022829D0012801D03E
:10E57000032867D100200090084612F0EDFC834686
:10E58000204603F030F90646204603F00EF94FF41A
:10E59000A051B1FBF6F20190824201DAB1FBF6F034
:10E5A0000390B4F902000290287CC0F30110012806
:10E5B00013D020886080711E0844E0800027C4E0EA
:10E5C00021462846089A00F0DBF8089A09B021464F
:10E5D0002846BDE8F04FFEF709BD68882188401A3B
:10E5E000401EE080801B401C6080E7E70399C01B51
:10E5F000884200DD08460FFA80F90120CBF81000B0
:10E600000FBB0198B0421EDB287CB146C0F301105D
:10E61000032810D000204946089A00F0E5F8287C2D
:10E62000C0F30110012808D029880298081A401E5A
:10E63000A080801B54E00120EDE702982080029822
:10E64000304463E08DE0009820B94FF4205014F07E
:10E65000DDFF0090287CC0F3011003281AD00020B1
:10E660008646DDF820C000984946069016FB01F06A
:10E67000401E0590701E4843049000208246884248
:10E6800021DA0498BEF1000F504401D0059A101A07
:10E69000002212E00120E3E7069BBEF1000F03EB2E
:10E6A000400863460CF1020C1B88A8F8003001D02A
:10E6B000084400E0401A521C12B2B242ECDB0AF1EC
:10E6C000010000B2DAE7287CC0F30110012819D05C
:10E6D00029880298081AC01B401EA080A0EB0900E0
:10E6E000401C208001984F44874212DBDBF8180061
:10E6F000C0070ED0DBF8180080070AD50120CBF840
:10E70000140009E00298384420804844401EA0804C
:10E71000E8E70021CBF81410009828B10246214602
:10E720002846FEF763FC05E0089AF8E7A96A09B1F4
:10E7300028468847DBF810000028F7D1089906FB27
:10E7400009F001EB40003FB2089001988742FFF6C4
:10E750004DAF0098002804D009B0BDE8F04F14F088
:10E76000A1BF09B0BDE8F08F6037002030B5048844
:10E770000D88058010880880188810801C8030BDA6
:10E78000F8B5054616460C46084603F02CF8074631
:10E79000204603F00AF817FB00F300200CE006EB1C
:10E7A000430706EB40013A88ADF80020B1F800C0FD
:10E7B000A7F800C00A80401C5B1E8342EFD869881E
:10E7C0006288E088891A491EE1806988081A401E1B
:10E7D000608029882288A088891A491EA1802988FA
:10E7E000081A401E2080F8BD2DE9F0470C46164659
:10E7F0008246002701EBD47931E00025601C00EB54
:10E80000D07827E0E01B401E01B2601B401E00B222
:10E81000BAF1000F0AD015FB041206EB420311FBFC
:10E82000040106EB410210FB047009E010FB0472C6
:10E8300006EB420311FB040006EB400215FB04103B
:10E8400006EB400117FB045006EB4000FFF78EFF7C
:10E850006D1C2DB2B5EB680FD4DB7F1C3FB2B7EB5C
:10E86000690FCADBBDE8F0872DE9FF4F95B0987BB3
:10E870008A7E00F00F04DDF888800D46032C00D15D
:10E880000424012C19D0022C1FD0042C25D0082CD4
:10E890007DD1DFF890924FF0FF0A6101FD2A35D259
:10E8A000DFF884C29CF80000904203D1DCF8040039
:10E8B000A04225D000209D4F20E0DFF868924FF065
:10E8C000800AA9F116090221E8E7DFF858924FF013
:10E8D000C00AA9F114090421E0E7DFF848924FF0DB
:10E8E000F00AA9F110091021D8E719F80060FF2EED
:10E8F0001CD016FB02F6360A3E54401C8842F4D364
:10E90000DFF828928CF80020CCF804401798DE88B5
:10E910000996B0F900101598B3F808B066438068FE
:10E92000B0F90020914203DB002202E01646E3E743
:10E93000521A0A92099A8B18B0F90420934201DC0A
:10E94000099901E0511A491C0B911799B0F902205D
:10E95000B1F90210914201DB002200E0521A0E923E
:10E96000B0F9060001EB0B02824201DC584601E0DF
:10E97000401A401C0F900E980A99704301FB040046
:10E9800008EBD00700F0070668461C2100E0C5E050
:10E9900019F0A7FBA889ADF80800A87E8DF818002B
:10E9A000A87FC0F3C2008DF81900FDF741FF12F0F7
:10E9B000D7FA099901FB0BF1814200DC084610905F
:10E9C00014F024FE834603901798002501880A98C6
:10E9D0000A181798ADF81C2001880B98401E0144B6
:10E9E000ADF82010179843880E9818448B1A5B1CBA
:10E9F000ADF81E00ADF822001BB21193ADF8341033
:10EA0000ADF830200F99ADF832000844ADF836006B
:10EA10000CA803F0E1FF139007A800900590C4F143
:10EA200008001290DDE9090101440B98081A6043BF
:10EA300014900E985BE02B462AFA06F04FF0000C7B
:10EA40000A991AE03A78DDF848800240A8EB0608F7
:10EA500032FA08F204D019F802800BF8058001E0C0
:10EA60000BF805C0129A964202D22644E04002E01A
:10EA7000002650467F1C491C6D1C0B9A9142E1DB1D
:10EA8000139880B10BEB0300BDF92220BDF91C10D7
:10EA90008046119B03F062FF8DF8100018B94046C4
:10EAA000119919F01EFBDDE90A10401A411910985E
:10EAB000814205D2BDF82200401CADF822000EE0D4
:10EAC00002208DF810006946159804F0AEFCBDF8E0
:10EAD0002200401CADF81E00ADF82200002514985D
:10EAE000304407EBD00700F007060998401C0F9947
:10EAF000099088429FDBBDF91E10BDF922008142BA
:10EB000009D0401EADF8220002208DF810006946A1
:10EB1000159804F08AFC584614F0C4FD19B0BDE8FD
:10EB2000F08F00005A9D010874370020AC96002039
:10EB30002DE9F04F8346B1F902000C46401E41100A
:10EB400000F001004618B2F90000B3F9005089B096
:10EB5000A84200DB2846ADF80000B2F90000B3F986
:10EB60000030984200DC1846401EADF80400508882
:10EB7000801BADF8020050880844ADF806006946D5
:10EB80000846DBF808200BF044FA002822D0E08881
:10EB900018B1A08808B1012000E0002080460126BD
:10EBA000684603F019FF10B9B8F1000F00D0002635
:10EBB0001C2102A805F033FECDF808D02088ADF85E
:10EBC0001000207A6D468DF8200036B102A9584613
:10EBD00004F02BFC09B0BDE8F08FBDF80410BDF9BE
:10EBE0000000BDF906A0091A491C0EB2BDF80210BA
:10EBF000ADF806104FF00009B8F1000F08D0B4F9D5
:10EC00000610B4F90420114490FBF1F201FB120943
:10EC1000304614F0FBFC079505900746BDF90250FD
:10EC20003EE03146384605F0FEFDBDF900103346A2
:10EC30002AB2384603F092FE8DF81800B8F1000FA2
:10EC40001FD0F0B1002148460B4615E0B4F904206E
:10EC5000824205DB121A1144104409B200B207E0E7
:10EC6000B4F906C06244824201DC002000E07B541B
:10EC7000491C401C09B200B2B142E7DB02208DF80A
:10EC8000180002A9584604F0D0FBBDF80200401C51
:10EC9000ADF80200BDF80600401CADF806006D1C82
:10ECA0005545BEDD384614F0FDFC93E72DE9FF4FD6
:10ECB000B2F90250B3F90240BBB0A54208DA12889B
:10ECC00065F31F4062F30F0064F31F411A8807E0E9
:10ECD0001B8864F31F40128865F31F4163F30F0024
:10ECE00062F30F010FFA81F906B20714A9EB0604CB
:10ECF0004FEA214AAAEB07053791002C01DD204697
:10ED000000E06042002D01DD294600E069428842B2
:10ED100001DD012000E0002000903C98B0F90210D5
:10ED2000009858B1002D01DD284600E068424201FC
:10ED3000002C01DD20460CE060420AE0002C01DDE1
:10ED4000204600E060424201002D01DD284600E03F
:10ED5000684292FBF0F0AB4A105C10FB01F03F30D0
:10ED6000C0114FEA600800F0010202EB080B4946AF
:10ED70004E4500DA3146A1EB0001ADF8601001DD2F
:10ED8000314600E049460144ADF86410514657450C
:10ED900000DA3946A1EB0001ADF8621001DD394619
:10EDA00000E051460844ADF866003B9818A9826817
:10EDB00008460BF02EF900287ED00098002100288C
:10EDC0007BD0002C16DDAAEB080000B2CDE90001D3
:10EDD000A7EB080002B24B46314602A803F09AFEA8
:10EDE0000AEB0B00012100B2CDE900014B4607EB15
:10EDF0000B0015E00AEB0B0000B2CDE9000107EBB8
:10EE00000B0002B24B46314602A803F083FEAAEB88
:10EE10000800012100B2CDE900014B46A7EB080034
:10EE200002B231460DA803F075FE002102A803F0DE
:10EE3000E3FB399000210DA803F0DEFB38904FF082
:10EE4000FF30804600903C98407AC00623D43819A1
:10EE5000032100B2CDE90001701B03B23A463146EE
:10EE600021A803F057FE379902200A14111909B29C
:10EE7000CDE90010379801B2481B03B22CA803F06B
:10EE800049FE002121A803F0B7FB009000212CA827
:10EE900003F0B2FB8046BDF86400BDF86010401A74
:10EEA000401C06B2FDF7C4FC12F05AF8044618A83C
:10EEB00011F091F8A04201E0A1E028E003D218A8E7
:10EEC00011F089F80446A146204614F09FFB8246C3
:10EED000BDF966B0BDF86200ADF866000024494691
:10EEE000504605F0A0FC1C211AA805F098FC3C989F
:10EEF00018A91A910088ADF870003C98007ACDF8F6
:10EF000074A08DF880001F91BDF9625044E009EBB8
:10EF10000B00CDE900A103B206EB0B0001B23A46AB
:10EF200002A803F0F7FD0121A9EB0800CDE900A13B
:10EF300003B2A6EB080001B23A4673E70AEB0407F6
:10EF4000BDF9601033462AB2384603F007FD8DF84C
:10EF5000780018B93846314605F061FC3444A119EF
:10EF6000494505D2BDF86600401CADF8660012E0C8
:10EF700002208DF878001AA93B9804F056FABDF8E3
:10EF800066000024401CADF86200ADF866004946FA
:10EF9000504605F048FC6D1C5D45CFDDBDF96210A3
:10EFA000BDF96600814209D0401EADF8660002201E
:10EFB0008DF878001AA93B9804F037FA504614F0FF
:10EFC00071FB02A803F0ECFC0DA803F0E9FC00982B
:10EFD000401C02D021A803F0E3FCB8F1FF3F02D0AF
:10EFE0002CA803F0DDFC399804F00AF8389804F0F6
:10EFF00007F8009804F004F8404604F001F83FB028
:10F00000BDE8F08F5A9E01082DE9F04F8346B1F913
:10F0100002000C46401E411000F00100158889B026
:10F020000844281AADF8000010880844ADF8040020
:10F03000B2F90200B3F90210884200DB0846ADF8CD
:10F040000200B2F90200B3F90210884200DC08465F
:10F05000401EADF8060069460846DBF808200AF0B5
:10F06000D8FF00281FD0E08818B1A08808B1012778
:10F0700000E000270125684603F0AEFC00B907B1A7
:10F0800000251C2102A805F0CAFBCDF808D0208875
:10F09000ADF81000207A6E468DF8200035B102A937
:10F0A000584604F0C2F909B0BDE8F08FBDF804007D
:10F0B000BDF80010BDF90690401A401C0FFA80F808
:10F0C000BDF80200ADF80600404614F09FFA8246F3
:10F0D00000250796059057B1B4F90600B4F904105D
:10F0E0000844BDF9021091FBF0F200FB1215BDF9C6
:10F0F00002602EE04146504605F095FBBDF9001038
:10F10000434632B2504603F029FC8DF818008FB107
:10F1100070B1B4F90400A84202DA00208DF818009A
:10F12000B4F90600B4F904100844A84200DC002534
:10F130006D1C2DB202A9584604F077F9BDF8020003
:10F14000401CADF80200BDF80600401CADF80600FA
:10F15000761C4E45CEDD504614F0A4FAA3E770B5F8
:10F16000054691F82A0088B00C46022858D9E18C4F
:10F17000002955D0114604A802F008FB218DBDF8E6
:10F180001000491E401AADF81000BDF81200401AD8
:10F19000ADF81200BDF814000844ADF81400BDF835
:10F1A00016000844ADF8160004A906A802F0EEFA0D
:10F1B000BDF81810E08C091AADF81810BDF81C1035
:10F1C0000844ADF81C00BDF81A00E18C401AADF8F7
:10F1D0001A00BDF81E00E18C0844ADF81E0004A81A
:10F1E00002F01FFB064604A802F0F1FAB4F9001081
:10F1F000864200DA3046B1EB600F00DD4110E08C52
:10F20000A278084403B294F82A00CDE90202A08C47
:10F21000ADF80400009104AA06A92846FEF753FEA3
:10F2200008B070BD7CB50446806961896D4686680A
:10F23000A08961B1002865D0814203D12289E38889
:10F240009A427CD302297BD003297AD0AFE010BB4D
:10F25000E088218988421ED2B4F9060016F014F91C
:10F26000B4F90410B4F90E20891A4843216849887A
:10F2700001EBE030ADF80200E0885A3000B216F041
:10F2800003F9A18810FB01F02168098801EBE03047
:10F29000ADF8040040E020680088ADF80000206868
:10F2A000A18840880844ADF80600B4F9060016F0BD
:10F2B000EBF8B4F90410B4F90E20891A4843216818
:10F2C000498801EBE030ADF80200E0885A3000B226
:10F2D00016F0DAF8A18810FB01F02168324609889F
:10F2E00001EBE030ADF80400694608460AF091FEF3
:10F2F00030B1A0698560D4E90520216903F090FE52
:10F30000A08970BB2068A18800880844ADF804007B
:10F3100020684088ADF80200B4F9080016F0B4F88F
:10F32000A18810FB01F02168498801EBE030ADF8BD
:10F33000060020895A3000B216F0A6F802E015E067
:10F3400012E00FE0B4F90410B4F90E20891A484312
:10F3500021683246098801EBE030ADF800006946CB
:10F360001AE024E0022801D0012820D1206832468A
:10F370000088ADF8000020684088ADF802002068E1
:10F38000A18800880844ADF804002068A18840885E
:10F390000844ADF80600294608460AF03AFE30B1A6
:10F3A000A0698560D4E90520216903F039FEA069D0
:10F3B00086607CBD7CB50446806961896D4686683F
:10F3C000A08901290CD0012867D0814203D122896C
:10F3D000E3889A427ED300297DD003297CD0B5E012
:10F3E000012822D1E088218988421ED2B4F9060082
:10F3F00016F04AF8A18810FB01F02168498801EB5A
:10F40000E030ADF80600E0885A3000B216F03CF863
:10F41000B4F90410B4F90E20891A48432168098808
:10F4200001EBE030ADF8040042E02068A1880088DC
:10F43000401AADF8000020684088ADF80200B4F929
:10F44000060016F021F8A18810FB01F02168498818
:10F4500001EBE030ADF80600E0885A3000B216F05B
:10F4600013F8B4F90410B4F90E20891A484321683E
:10F470003246098801EBE030ADF8040069460846E1
:10F480000AF0C7FD30B1A0698560D4E90520216983
:10F4900003F0C6FDA089012858D120680088401ECD
:10F4A000ADF804002068A18840880844ADF8060043
:10F4B000B4F9080015F0E8FFB4F90410B4F90E200F
:10F4C000891A48432168498801EBE030ADF8020011
:10F4D000208902E018E010E014E05A3000B215F084
:10F4E000D3FFA18810FB01F021683246098801EBA7
:10F4F000E030ADF8000069461DE0022804D0032882
:10F5000002D023E0022821D12068A1883246008859
:10F51000401AADF8000020684088ADF8020020686D
:10F520000088401EADF804002068A1884088084487
:10F53000ADF80600294608460AF06BFD30B1A06917
:10F540008560D4E90520216903F06AFDA069866021
:10F550007CBD7CB50446806961896D468668A0895A
:10F5600002290CD002287ED0814203D12289E3886F
:10F570009A4279D3002978D0012977D0D4E00228A3
:10F580003FD1E088218988423BD25A3000B215F041
:10F590007BFFA18810FB01F02168098801EBE030B6
:10F5A000ADF80000B4F9060015F06EFFB4F90410D0
:10F5B000B4F90E20891A48432168498801EBE030EC
:10F5C000ADF80600B4F9080015F05EFFA18810FB45
:10F5D00001F02168498801EBE030ADF80200208994
:10F5E0005A3000B215F050FFB4F90410B4F90E20EF
:10F5F000891A48432168098801EBE030ADF804001E
:10F6000066E020680088401EADF804002068A188EC
:10F610004088401AADF80200E0885A3000B215F078
:10F6200033FFA18810FB01F02168098801EBE0306D
:10F63000ADF80000B4F9060015F026FFB4F9041087
:10F64000B4F90E20891A484321683246498801EBF3
:10F65000E030ADF80600694608460AF0DAFC58B119
:10F66000A069856003E00AE03BE034E036E0D4E9DD
:10F670000520216903F0D4FCA089022854D1206818
:10F68000A1880088401AADF8000020684088401E1C
:10F69000ADF8060020895A3000B215F0F5FEB4F935
:10F6A0000410B4F90E20891A48432168098801EB37
:10F6B000E030ADF80400B4F9080015F0E5FEA188CB
:10F6C00010FB01F02168498801EBE030ADF8020041
:10F6D000324669461DE0032803D025E0032800D008
:10F6E00010BB2068A18832460088401AADF800009F
:10F6F0002068A1884088401AADF802002068294699
:10F700000088401EADF8040020684088401EADF817
:10F71000060008460AF07DFC30B1A0698560D4E996
:10F720000520216903F07CFCA06986607CBD7CB566
:10F730000446806961896D468668A08903290ED0D8
:10F74000032867D0814203D12289E3889A427ED37D
:10F7500002297DD001297CD002297BD0B1E0032889
:10F760001FD1E088218988421BD25A3000B215F09F
:10F770008BFEB4F90410B4F90E20891A48432168AD
:10F78000098801EBE030ADF80000B4F9060015F08F
:10F790007BFEA18810FB01F02168498801EBE03075
:10F7A00040E02068A18800880844ADF80400206883
:10F7B0004088401EADF80600E0885A3000B215F0CF
:10F7C00063FEB4F90410B4F90E20891A4843216885
:10F7D000098801EBE030ADF80000B4F9060015F03F
:10F7E00053FEA18810FB01F021683246498801EBE5
:10F7F000E030ADF80200694608460AF00AFC30B174
:10F80000A0698560D4E90520216903F009FCA0897D
:10F81000032856D120680088ADF800002068A18830
:10F820004088401AADF8020020895A3000B215F025
:10F830002BFEA18810FB01F02168098801EBE03064
:10F84000ADF80400B4F9080015F01EFE03E016E060
:10F8500010E013E00FE0B4F90410B4F90E20891A97
:10F86000484321683246498801EBE030ADF8060094
:10F8700069461BE018B1012801D022E008BB2068CE
:10F8800032460088ADF800002068A1884088401A00
:10F89000ADF802002068A18800880844ADF8040093
:10F8A000206829464088401EADF8060008460AF048
:10F8B000B0FB30B1A0698560D4E90520216903F06F
:10F8C000AFFBA06986607CBD70B5A4B00C46054650
:10F8D00022AA20A906F083F820A810F07CFB20B90A
:10F8E00022A810F078FB00283ED012A9284609F083
:10F8F000D9FD012838D12146684605F05DFC1B483A
:10F9000001900220029012A804904FF480300D90D4
:10F9100020A810F060FB80B120A803906A461A214D
:10F92000284611F0FFFB20AA12A9204603F078FB1D
:10F930006A461B21284611F0F5FB22A810F04BFB6C
:10F94000002811D022AE6A461A212846039611F0EB
:10F95000E9FB22AA12A92046039603F061FB6A463E
:10F960001B21284611F0DEFB24B070BD209D01084C
:10F970002DE9F74FB1F92E00A2B014460D4600282C
:10F9800072D095F8361002296ED9012808D1B5F940
:10F990003400002804DC288E10B9688E0028EFD0CF
:10F9A0002088298EAA8E0844801AADF82000A388EA
:10F9B00019441144ADF8241062886B8E1A44AB8E42
:10F9C000D21AADF82220E3886E8E3344AE8E3344D3
:10F9D000ADF82630B5F92E6006EBD676A0EB6600C2
:10F9E000401EADF82800012000EB66063144ADF85A
:10F9F0002C10B5F92E1001EBD171A2EB6101491E5B
:10FA0000ADF82A10B5F92E1001EBD17100EB6100B1
:10FA10001844ADF82E0095F836000D90FD2801D958
:10FA2000FF200D9022980AA9826820A80AF0F1FA16
:10FA30000028A5D0214603A801F0A8FE4FF0FF370B
:10FA400039463A4603A810F0F2FAB5F9009003A837
:10FA500001F0E7FE044603A801F0B9FE844203A8C2
:10FA600003DA01F0DEFE02E0FEE301F0B0FEB9EBE6
:10FA7000600F01DD4FEA6009B5F9006008A801F0E8
:10FA8000D0FE044608A801F0A2FE844208A802DACB
:10FA900001F0C7FE01E001F09AFEB6EB600F00DD59
:10FAA0004610B5F92E00841904FB04F0400013F051
:10FAB000ADFD00900146B5F92E20334608A809F0A7
:10FAC00009FE0AA802F088FF012620B9E878FF287D
:10FAD00001D3A87800B100261F9756B901234A46E2
:10FAE00003A912A803F0E2F9002112A802F084FD94
:10FAF0001F900AA801F095FE13F088FD83461C2193
:10FB000018A804F08EFE01A81890CDF86CB01D90D6
:10FB1000A88DADF8680095F836008DF87800A878C3
:10FB20008DF879000AA801F07CFEBDF8281000EBE2
:10FB3000D07001EB60000FFA80FA0AA801F047FECE
:10FB4000BDF82A1000EBD07001EB600007B2BDF8E1
:10FB50002C00ADF80800001B401C00B2621EADF87E
:10FB60000400ADF8061011440C9209B2ADF80A1069
:10FB70005246504500DC1046ADF80400B94200DBA7
:10FB800039462298ADF80A1001A9826805A80AF042
:10FB900040FAC0B34A4603A905A80AF062FA90BB2E
:10FBA00005A801F03EFEBDF91610BDF92A200E9001
:10FBB000891A0098BDF92C2001FB0400BDF914102E
:10FBC000121B891A0844401E119046B14A4603A9E7
:10FBD00005A80AF0B6FA10B10120079000E00796D8
:10FBE0000E98002827DDBDF81400ADF80400CDF80C
:10FBF0006CB0BDF81800ADF8080002208DF8700058
:10FC0000BDF9168013E016E0ADF80A800798ADF84C
:10FC10000680E8B311981B9018A9229803F005FC00
:10FC200011982044119008F101000FFA80F8BDF9F5
:10FC30001A104145E8DABDF82C00ADF80800001BA9
:10FC4000401C00B2ADF80400BDF82E20ADF80A202B
:10FC5000111B491C09B2ADF806105246504500DC94
:10FC60001046ADF80400781C0F90814200DC791C2E
:10FC70002298ADF8061001A9826805A80AF0C9F912
:10FC8000D0B34A4603A905A80AF0EBF9A8B15FE092
:10FC9000FFE722465846119904F0B8FDBDF914104B
:10FCA000424658460E9B02F059FE8DF8700001281E
:10FCB000B2D102208DF87000AEE705A801F0B1FDC9
:10FCC000BDF90A10BDF91A200E90891A0098BDF9E5
:10FCD0002C2001FB0400BDF91410121B891A0844E2
:10FCE000401E11904EB14A4603A905A80AF029FA10
:10FCF00018B10120079001E02AE007960E9800282D
:10FD000026DDBDF81400ADF80400CDF86CB0BDF8E8
:10FD10001800ADF8080002208DF87000BDF91A80B7
:10FD200012E0ADF80A800798ADF80680B0B31198DC
:10FD30001B9018A9229803F078FB11982044119089
:10FD4000A8F101000FFA80F8BDF916104145E8DD71
:10FD5000BDF828002044ADF80400BDF82C00001BBD
:10FD6000ADF80800BDF82A000C99ADF8060008446B
:10FD700000B2ADF80A00B84200DB3846ADF80A0020
:10FD8000229801A9826805A80AF043F990B34A466F
:10FD900003A905A80AF065F9A8B178E0FFE72246B3
:10FDA0005846119904F032FDBDF9141042465846E8
:10FDB0000E9B02F0D3FD8DF870000128B9D102200E
:10FDC0008DF87000B5E705A801F02BFD0E90BDF988
:10FDD0001610BDF906200098891A01FB0400119045
:10FDE0004EB14A4603A905A80AF0ABF918B10120A3
:10FDF000079001E04BE007960E98002847DD079832
:10FE000060B100201B90BDF81400ADF80400BDF8EF
:10FE10001800ADF80800BDF9160033E0CDF86CB05D
:10FE2000F1E7ADF80A800798ADF8068060B10D984B
:10FE3000FF281198007804D095F8361010FB01F0D7
:10FE4000000A8DF8780013E011980E9A0178584650
:10FE500004F0DEFCBDF91410424658460E9B02F039
:10FE60007DFD8DF87000012802D102208DF8700010
:10FE700018A9229803F0D9FA11982044119008F19A
:10FE8000010000B2BDF91A1080464145C9DA95F863
:10FE900036008DF87800BDF828002044ADF8040045
:10FEA000BDF82C00BDF82E10001BADF80800081B93
:10FEB000401CADF80A1000B20F99ADF80600884258
:10FEC00000DC781CADF80600229801A9826805A81C
:10FED0000AF09FF8F0B34A4603A905A80AF0C1F852
:10FEE000C0BB05A801F09DFC0790BDF90A10BDF943
:10FEF0001A200098891A01FB040011900798002825
:10FF000055DD2EB14A4603A905A80AF01AF900B931
:10FF100066B100201B90BDF81400ADF80400BDF8D8
:10FF20001800ADF80800BDF91A003BE0CDF86CB040
:10FF3000F1E7ADF80680ADF80A802EB14A4603A974
:10FF400005A80AF0FEF800B976B10D98FF281198BF
:10FF5000007800E02BE004D095F8361010FB01F09B
:10FF6000000A8DF8780013E01198079A0178584636
:10FF700004F04EFCBDF9141042465846079B02F0AF
:10FF8000EDFC8DF87000012802D102208DF8700080
:10FF900018A9229803F049FA119820441190A8F169
:10FFA000010000B2BDF9161080464145C1DD95F84B
:10FFB00036008DF87800BDF82C00ADF80800011B64
:10FFC000BDF82A00491C09B22044ADF8041000B263
:10FFD000ADF80600BDF82E200F9B121B12B2ADF833
:10FFE0000A20984200DB781CADF80600BA4200DC1B
:10FFF0003A46ADF80A205046514500DC01462298A9
:020000040801F1
:10000000ADF8041001A9826805A80AF002F8C8B387
:100010004A464D4603A905A80AF023F890BB05A857
:1000200001F0FFFB10900C990098BDF92C2001FB0A
:100030000400BDF91410121B891A0844401E1190C7
:1000400046B12A4603A905A80AF07BF810B14FF083
:10005000010802E0B6F1000801D0119800E058460E
:100060001B901098002832DDBDF81400ADF8040094
:10007000BDF81800ADF8080002208DF87000BDF939
:10008000165020E023E0ADF80650ADF80A50B8F164
:10009000000F12D1DDE91021584604F0B7FBBDF97D
:1000A00014102A465846109B02F058FC8DF8700038
:1000B000012802D102208DF8700018A9229803F0BF
:1000C000B4F96D1C2DB2BDF91A00A842DBDA002389
:1000D000009815E000EB040EAEF10101002204EBE4
:1000E000D47C07E0057891F8008000F8018B01F8D6
:1000F0000159521CB2EB6C0FF4DB5B1C70461BB257
:10010000A342E7DBBDF828000C99ADF804000844D1
:1001100001B2BDF82A000F9B204400B2ADF80600E2
:10012000BDF82E20ADF80810121B12B2ADF80A204F
:10013000984200DB781CADF80600BA4200DC3A4673
:10014000AAF10100ADF80A201090814200DB0146BF
:100150002298ADF8081001A9826805A809F059FF96
:10016000B8B34A464D4603A905A809F07AFF80BBFB
:1001700005A801F056FB0E900C990098BDF90420DB
:1001800001FB0400BDF91410891A0844119046B10E
:100190002A4603A905A809F0D4FF10B14FF00108C1
:1001A00002E0B6F1000801D0119800E058461B901B
:1001B0000E98002832DDBDF81400ADF80400BDF83B
:1001C0001800ADF8080002208DF87000BDF9165037
:1001D00020E023E0ADF80650ADF80A50B8F1000F6A
:1001E00012D158460E9A119904F010FBBDF9141063
:1001F0002A4658460E9B02F0B1FB8DF8700001288C
:1002000002D102208DF8700018A9229803F00DF990
:100210006D1C2DB2BDF91A00A842DBDABDF828002A
:100220000C99ADF80400084400B2ADF80800BDF820
:100230002A100C9AADF806101144109A09B2ADF8C4
:100240000A10904201DBAAF10100ADF80800B942A2
:1002500000DB39462298ADF80A1001A9826805A88A
:1002600009F0D7FEC8B300E044E14A464D4603A971
:1002700005A809F0F6FE80BB05A801F0D2FABDF989
:100280001620BDF906100D90511A0098BDF90420F2
:1002900001FB0400BDF91410891A01EB000846B1F6
:1002A0002A4603A905A809F04CFF10B101200790C8
:1002B00000E007960D98CDF86CB0002821DDBDF860
:1002C0001400ADF80400BDF81800ADF808000220D5
:1002D0008DF87000BDF916500FE012E0ADF80A502D
:1002E0000798ADF80650D0B3CDF86C8018A92298C5
:1002F00003F09BF86D1CA0442DB2BDF91A00A84272
:10030000ECDABDF82800ADF804000C99BDF82E20F9
:10031000084401B2101BADF80810401CADF80A20CB
:1003200000B20F9AADF80600904200DC781CADF8E0
:1003300006001098814201DBAAF101012298ADF874
:10034000081001A9826805A809F063FEC0B34A46F7
:100350004D4603A905A809F084FEA8B158E0FFE7BF
:1003600022464146584604F051FABDF914102A4677
:1003700058460D9B02F0F2FA8DF870000128B5D1B5
:1003800002208DF87000B1E705A801F04AFABDF926
:100390000A10BDF91A208246891A0098BDF9042076
:1003A00001FB0400BDF91410891A0F184EB12A463A
:1003B00003A905A809F0C5FE18B14FF0010801E036
:1003C00026E0B046CDF86CB0BAF1000F20DDBDF8E4
:1003D0001400ADF80400BDF81800ADF808000220C4
:1003E0008DF87000BDF91A500EE0ADF80650ADF86A
:1003F0000A50B8F1000F2FD01B9718A9229803F0CC
:1004000014F86D1E27442DB2BDF91600A842ECDD8C
:10041000BDF8280001A92044ADF80400BDF82C0067
:10042000001BADF80800BDF82A002044ADF8060016
:10043000BDF82E00001BADF80A002298CDF86CB074
:10044000826805A809F0E5FDF0B34A4603A905A8AE
:1004500009F007FEA0B140E022463946584604F0B4
:10046000D5F9BDF9141053462A46584602F076FADB
:100470008DF870000128C0D102208DF87000BCE713
:1004800005A801F0CEF9051E27DDBDF81400ADF872
:100490000400BDF81800ADF80800BDF9164018E0DA
:1004A000ADF80640ADF80A402946584604F0BEF9BA
:1004B000BDF914102B462246584602F04FFA8DF82B
:1004C000700018A9229800E007E002F0AEFF641C5B
:1004D00024B2BDF91A00A042E2DA2EB912A802F045
:1004E0005FFA1F9802F08CFD009813F0DBF8584675
:1004F00013F0D8F825B0BDE8F08F00002DE9FF4FCC
:1005000083B00446DDE910870E460846139D01F0CE
:1005100076F98346304601F04EF90190012D0FD057
:10052000022D0FD0032D3ED1404E6FB12088ADF883
:10053000000038784FF0000AFD2837D3424638E0F3
:100540003B4EF2E73B4EF0E72088ADF80800ADF8EF
:100550000000424602990698B047002702901FE02B
:10056000002517E0BDF8000034F8151088420BD0C4
:1005700004EB450042460088ADF80800ADF80000E5
:1005800002990698B047029004EB4500BDF80810A8
:1005900001806D1C5D45E5DB05987F1C04EB400484
:1005A00001988742DCDB07B0BDE8F08F00FB08F064
:1005B000020A00990698B0470290002030E000251A
:1005C00025E0785D10B3504505D1BDF8001034F832
:1005D0001520914215D0FD2801D3424602E000FBD0
:1005E00008F0020A04EB45000088ADF80800029903
:1005F0000698B047029017F805A034F81500ADF83A
:10060000000004EB4500BDF8081001806D1C5D453D
:10061000D7DB059804EB40041298074409F1010068
:10062000019981468842CADBBDE700007BD3000800
:10063000F9D20008FFD300082DE9FF4F85B004462A
:10064000DDE9127593460E46084601F0D8F880465B
:10065000304601F0B0F882466DB1BDF82000FD2FA4
:1006600000EB00497DD3A8F1040001900020009028
:10067000BDF820703AE1FD2F0ED3002507E0424679
:100680002046089910F05EFA04EB4B046D1C5545AA
:10069000F5DB09B0BDE8F08FBDF80010002060F375
:1006A000020189B260F3C70189B260F30C2189B2FB
:1006B00060F34F31ADF8001088B20090BDF8000033
:1006C000009001463A46089801F07AF93F1D0190E2
:1006D0000899F808C00689B2000EC1F3C40212FBE3
:1006E00000F2ADF808204A07920E02EB513212FBDD
:1006F00000F2ADF80A20C1F3042111FB00F1ADF8BE
:100700000C10C0F1FF02002556E000204FE0BDF8BC
:10071000001034F81030994243D004EB40010988AE
:10072000ADF80410ADF80010BDF80430BDF80810A5
:10073000C3F3C40616FB021101EBC11606EBC1316F
:10074000BDF81060C1F3C45161F3C7065907890EA3
:10075000BDF80A7001EB533111FB027101EBC117B7
:1007600000E0C9E007EBC137BF0E67F3020601EBFB
:10077000C11707EBC131C1F3C25161F34F36BDF868
:100780000C10C3F3042313FB021101EBC11303EBA1
:10079000C131C1F3C45161F30C26B1B2ADF81060A0
:1007A000019104EB4001BDF804300B80401C404532
:1007B000ADDB04EB4B046D1C5545A6DB69E7002659
:1007C00010E02A78FF2A12D02088ADF8080002999C
:1007D000089801F0F5F80290BDF808002080A41CEC
:1007E0006D1C761C464557DAA807EAD154E02780ED
:1007F000F5E72868411C43D0F0B32A78FF2A4FD090
:100800002088ADF808000299089801F0D9F8029004
:10081000BDF80800208015F8012FA41CFF2A41D044
:100820002088ADF808000299089801F0C9F80290F4
:10083000BDF80800208015F8012FA41CFF2A33D032
:100840002088ADF808000299089801F0B9F80290E4
:10085000BDF80800208015F8012FA41CFF2A25D020
:100860002088ADF808000299089801F0A9F80290D4
:10087000BDF80800208000E00BE0A41C6D1C0AE01D
:10088000A00704D02780C4F80290E78001E0C4E903
:10089000009908342D1D361D01988642A9DD18E007
:1008A0002780B8E72780C6E72780D4E72780E2E7DC
:1008B0002A78FF2A1ED02088ADF8080002990898EF
:1008C00001F07EF80290BDF808002080A41C6D1C89
:1008D000761C4645ECDBABEB080004EB40041498B7
:1008E000A0EB080005440098401C00905045FFF61E
:1008F00066AFCEE62780E9E700212388ADF8043013
:100900008946084633E0002627E0287818B3884255
:1009100005D0FF282FD000FB07F2120A914688422B
:1009200003D134F81600834210D0B9F1FF0F24D060
:1009300004EB46004A460088ADF804000199089887
:1009400001F03EF80190297834F8163004EB4600A7
:10095000BDF8042002806D1C761C4645D5DB14983A
:1009600004EB4B04A0EB080005440098401C0090E9
:100970005045C8DB8DE63A46D0E70898E2E72DE916
:10098000FF4F85B00D46DDE912A7FBF751FFBDF81B
:10099000209080464FB1284600F031FF0390284652
:1009A00000F009FF8346002640E0B5F9026017E039
:1009B000B5F900400FFA86FB0DE0CDF808A0ADF8C0
:1009C0000490CDF800B0D8F8000023B2079AC769A8
:1009D0000599B847641CB5F90400A042EDDA761C0D
:1009E000B5F90600B042E3DA09B0BDE8F08F0024A3
:1009F00016E0385D98B100FB0AF0000A0290ADF8ED
:100A000004906888079A304400B2009028880599BD
:100A1000204403B2D8F80000D0F81CC0E047641CA2
:100A200003988442E5DB1498761C07445E45DEDBC0
:100A3000DAE700680968884201D101207047002088
:100A4000704740680A6820F04040904200D2086039
:100A50000020704770B50D46C06A22F052F9044676
:100A6000284612F031FE0CB10C2070BD002070BD84
:100A700070B50D46C06A20F08EFA0446284612F082
:100A800023FE0CB10C2070BD002070BD70B5C56A8E
:100A90000E46342012F08CFD040009D00146324687
:100AA000284621F047FA0028204602D012F00CFE1A
:100AB000002070BD2DE9F043C3B00025D0F82C8094
:100AC000144689468DF808502F2602AF6A464946DB
:100AD000404621F07BFC00280CDD9DF80000022838
:100AE00004D03946204617F05DFB05E026703946F4
:100AF000601CF8E710D1257008A1204617F037FBDD
:100B00000028E3D006A1204617F031FB0028DDD0F5
:100B1000002043B0BDE8F0830C20FAE72F2E000040
:100B20002F2E2E002DE9F041C56A0E46022A17D05D
:100B3000012A17D0032A17D00024542012F038FDC0
:100B4000071E0BD0014623463246284622F098FA6B
:100B50000028384602D012F0B7FD0020BDE8F08131
:100B60000124EAE70224E8E70324E6E710B5C06AB7
:100B7000029C22F0C8FB002801DA0C2010BD206086
:100B8000002010BD10B5C06A23B1012B02D0022B8A
:100B900000D0002322F06EFC002801DA0C2010BDEA
:100BA000002010BD10B51446C06A22F035FD0028A3
:100BB00001DA0C2010BD2060002010BD2DE9F041AD
:100BC000C56A0F46069E284622F030FD040005D473
:100BD0003946284622F0B1FC002802DA0C20BDE894
:100BE000F08100203460FAE7B0F90C00032101EB3A
:100BF000400020F00300103070472DE9F041054619
:100C000000206B8C0E460427C3F30514EA680EE03F
:100C100007EBC00151585FEAC11C07D521F07F41A5
:100C2000B14203D152F83000BDE8F081401C84424B
:100C3000EED84FF0806000EBB3204FEAB0506884EC
:100C4000C0F30510C100104612F062FDE860C0B3A9
:100C5000688CC0F30514641E16D06FF003025300B5
:100C6000E86802EBC40141585FEAC11C0CD4890159
:100C70000AD400EBC40103EBC40C6044641ED0E949
:100C800000C0C1E900C0EBD1E868082100EBC40056
:100C900017F027FA082012F08BFCE96841F83400BD
:100CA00013F016FDEA6807EBC400115841F080719B
:100CB0001150EA6866F317011150E86850F83400E3
:100CC000B2E7FFE7FEE700002DE9FC410068C068DD
:100CD000C068B0FBF1F5954200DD1546134F78680A
:100CE0000068806900B30020ADF80000ADF8040092
:100CF000ADF802002CB2601E06B2ADF8066078684E
:100D00006946006882699047684600F04EFDA84237
:100D100002DD341EEFDC01E0002C02DC0020BDE827
:100D2000FC81BDF906506D1C2846F8E760370020AD
:100D30002DE9FF4F83B0064698468B46059809F08B
:100D4000FAFE01218140B6F820A001F0FF096FEA08
:100D50000A0080B2019096F822004FF0FF37C0F3EE
:100D6000C00500241CE0F16801EBC4004268920158
:100D70003BD5A5B9042202EBC402895801F47F01D6
:100D800059450CD10068817911EA090F07D06A46EC
:100D9000059913F04BFC01282ED0022830D0641C9A
:100DA000708CC0F30510A042DDD81EE0F06850F84A
:100DB0003430997911EA090F16D0042101EBC401EE
:100DC000405800F47F0185B259450DD10198054284
:100DD0000AD1BD4208DD18466A46059913F026FC83
:100DE000012810D002280BD0641C708CC0F30510B1
:100DF000A042DBD8002F0FDB00990120C8F80010BB
:100E000007B0BDE8F08F5545F6D0AF42ECDA009957
:100E10002F46C8F80010E7E70020F1E72DE9F0477A
:100E2000814642F30006C0F15A001D460F465408A1
:100E300000B2761C14F028FBA7EB040800FB08F0B6
:100E4000C711484614F020FB00FB08F0C011002F2A
:100E500006DD7F3F39120A1B32442A80214405E017
:100E60007F3739120A1B21442A80891BA980002858
:100E700006DD7F380012011B31446980204405E003
:100E80007F300012011B20446980801BE880BDE890
:100E9000F0872DE9F04104460020678C0D460426BA
:100EA000C7F30513E2680AE006EBC00151585FEA98
:100EB000811C03D521F07F41A94202D0401C83420E
:100EC000F2D8834203D002EBC000BDE8F0814FF0BE
:100ED000806000EBB7204FEAB0506084C0F305108B
:100EE000C100104612F014FCE060608CC0F30510E5
:100EF000401E0DD06FF00703E16803EBC00601EB65
:100F0000C0023144401ED1E90061C2E90061F3D161
:100F10000821E06817F0E5F8082012F049FBE168C5
:100F2000086013F0D5FBE168486840F00070486045
:100F3000E16865F317004860E068C6E701460020F5
:100F4000A1F13002092A01D8D0B27047612901D33A
:100F50002039C9B241390629F7D2DFE801F003058B
:100F600007090B0D0A2070470B2070470C207047B3
:100F70000D2070470E2070470F2070472DE9F0417B
:100F8000064615460F46002005E039462046B04784
:100F900001280AD0204607F033FC040002D0606824
:100FA0008000F2D10020BDE8F08105B12C60012065
:100FB000F9E7000010B50C461EF0B2FF0D4998B1DC
:100FC0000122A27306280DD2DFE800F00C0305070A
:100FD000090B0B2006E0092004E00A2002E01120A2
:100FE00000E01220086002E00020A0730868606042
:100FF00010BD0000283700202DE9F041044640686C
:10100000096820F04040884227D12046FFF7ECFDD8
:10101000DFF84C800546D8F80800021BA0EB05005D
:10102000561BC8F8080015D02746384661193246C5
:1010300017F02FF806E0A068401BA0602046FFF7DD
:10104000D3FD0444D8F808008442F4D1B8192946E5
:1010500017F047F80120BDE8F0810020FBE7000011
:10106000683700202DE9FC41064614468846D8071B
:1010700029D004F108000125002206F114010746D9
:1010800008F0EFFF58B100208DF800006A461221E9
:101090003046019710F046F89DF8000098B160893D
:1010A000218A0844401EE081B4F90E10B4F906000C
:1010B000814200DDE08102B02A4621464046BDE87B
:1010C000F04101F00BBA0025EEE72DE9F0410746AB
:1010D00088B01C46164688460846FBF7C2F9054606
:1010E00002A9404604F0B0FA2A46114602A80EF0C2
:1010F0009EFF022E05D0012E22D0002008B0BDE8B0
:10110000F081DDE90201CDE9040100231A4604A9BA
:10111000404605F01BF904AA06A8B96808F079FF53
:101120000028EBD0DDE90601CDE900010123002212
:101130006946404605F00AF9694602AA084602E0F7
:1011400002AA6846B96808F064FF0028D6D0009863
:101150002060019860600120D0E7000070B505466E
:1011600004F0E8F90646002406E0A868006850F894
:101170002400FFF7F3FF641CB442F6D3688CC10768
:101180001AD020F001006884284605F041FF284667
:1011900005F05AFE86B10021284604F0C6FF58B17A
:1011A0000C494968884207D80B49096801EBC0001F
:1011B00050E9022128469047688C810708D520F025
:1011C000020068842846BDE87040002105F082BD19
:1011D00070BD000054370020003800202DE9F04792
:1011E0008046089D1F46E86900FB01F39B1200281A
:1011F00006DD934206DD95F8280080070DD489E0CE
:101200009342F8DBCB1943439B12002808DD93423D
:1012100037DA95F8280080077CD40120BDE8F087F4
:101220009342F6DCA869521C504340F39500021229
:10123000C0B2FF23002826D06E6AC0F1FF0404FB71
:1012400006F4A3EB2426A2EB0104A14636D0002C21
:1012500015DBBC4213DAC0F1FF00C6F1FF014843C1
:10126000A3EB6020C1B295F82800800701D5C1F139
:10127000FF0118F8040007F0B4FA08F80400641C31
:101280001CE0A869D0E74FF0FF06DCE7002C10DB7C
:10129000BC420EDAA6EB6000C1B295F828008007C8
:1012A00001D5C1F1FF0118F8040007F09AFA08F817
:1012B0000400686A641C361ABC4202DA686AB042EA
:1012C000E4DBBC4218DA002C16DBA86970438012FC
:1012D0007043C0F34721E869002801DAC1F1FF013A
:1012E00095F82800800701D5C1F1FF0118F8040026
:1012F00007F077FA08F8040095F82800800707D56A
:101300004946B94506DC00290DDB404609E001E00D
:10131000641C01D5002081E7BC4204DC391B08EBCA
:10132000040003F07AFA022078E72DE9F05F8A469C
:101330000A9F06461D46B96901FB02F4A012002966
:1013400000DD401C97F82830504502DA980707D492
:10135000D2E0A0120AEB050C844502DA98077ED48D
:1013600080E044F39500521C4A4342F395044FEA4F
:101370002029221204F0FF08C0B2A9EB0A0491450B
:1013800005D0002903DA10B9FF209146641E91456B
:1013900026D1002C0BDBAC4209DA40444108980707
:1013A00001D5C1F1FF01305D07F01BFA305597F808
:1013B0002800641C800706D5A9EB0A01A9424EDA71
:1013C0008CE0304609E0AC4200DD2C46002C46D0D3
:1013D00005DDA5EB040106EB040003F01EFA88E02E
:1013E0004FF0FF0B002943DAF969494241434FEAC4
:1013F000A128002C0DDBAC420BDA08FB00F1C1F395
:101400004721980701D5C1F1FF01305D07F0E9F9E7
:101410003055B969A8F1FF0041438812641E11D408
:10142000AC420FDAC8F1FF014143ABEB6120C1B21E
:1014300097F82800800701D5C1F1FF01305D07F062
:10144000D0F9305597F82800A41C800708D5A9EBDF
:101450000A01491EA9424CDC0029B2DC49E04BE0FC
:10146000AC4202DD0120BDE8F09F002CB1DA40E083
:10147000F969C0F1FF0041434FEAA128002C0EDBBF
:10148000AC420CDA00FB08F0ABEB6020C1B298076D
:1014900001D5C1F1FF01305D07F0A3F93055B969FD
:1014A000C8F1FF0041438912641C0ED4AC420CDA2F
:1014B0004843C0F3472197F82800800701D5C1F1C0
:1014C000FF01305D07F08DF9305597F82800641C56
:1014D000800707D5A9EB0A01A9420DDC0029BFF658
:1014E00070AF06E0AC4200DD2C46002C04D03FF784
:1014F00070AF4FF00200B6E74FF00000B3E7000016
:101500002DE9F04107460E464FF00008134809F058
:1015100043FA04461CE02146104809F04FFA0546FC
:101520002068B84200D097B96068B04200D076B960
:1015300021460A4809F0CBFA216909B120468847BB
:10154000204612F0C1F8FBF7F7F94FF001082C46DE
:10155000002CE0D14046BDE8F0810000309800202A
:1015600070B505460C46094809F016FA0BE001680B
:10157000A94204D14168A14207D0002C05D0014600
:10158000024809F01BFA0028F1D170BD3098002004
:1015900010B50446442116F0A4FD4FF4FA70E06241
:1015A000002020626420A0620120A4F840000448CA
:1015B000E06194F8420040F0010084F8420010BD60
:1015C0002F16010838B504464FF480650095D4E91C
:1015D0000B200023194611F0CCFF4FF46E7332221A
:1015E000002100950EF097FD0146A26A206A121AAA
:1015F0004A4300EBA22038BD38B504464FF480655D
:101600000095D4E90B200023194611F0B2FF40F2F7
:10161000B6334FF46172002100950EF07CFD014657
:10162000A26A206A121A4A4300EBA22038BD38B5DC
:1016300004464FF480600090D4E90B200023194643
:1016400011F097FF0146A26A206A121A4A4300EB82
:10165000A22038BD38B504464FF480650095D4E922
:101660000B200023194611F084FF40F214534FF46D
:101670007A72002100950EF04EFD0146A26A206AA2
:10168000121A4A4300EBA22038BD8B1A002B00DC53
:10169000531A4FF47A714B43B3FBF0F0002800D19A
:1016A0000120704770B54168054611B12868FFF701
:1016B00027FF194809F002FA184E10B113F0C6FDC1
:1016C0007060154809F08DF9040024D029464422A1
:1016D00016F0DFFC2868A84200D12460717894F8E5
:1016E000420061F3820084F84200C0070FD06169B4
:1016F00039B120468847216A01442162A16A084421
:10170000A06262681AB1206808B1216A9047FBF7AD
:1017100013F9204670BDFEE730980020E83700201E
:101720000A8802804A8842808A888280C988C1806B
:1017300070470A8802804A8842808A888280C988E5
:10174000C18070470A8802804A8842808A888280E5
:10175000C988C18070470A8802804A8842808A8886
:101760008280C988C18070470A8802804A88428086
:101770008A888280C988C18070470A8802804A8826
:1017800042808A888280C988C18070470A88028026
:101790004A8842808A888280C988C1807047C1880F
:1017A0004088081A401C00B27047C1884088081A57
:1017B000401C00B27047C1884088081A401C00B223
:1017C0007047C1884088081A401C00B27047C18821
:1017D0004088081A401C00B2704781880088081AA7
:1017E000401C00B2704781880088081A401C00B273
:1017F000704781880088081A401C00B270478188B1
:101800000088081A401C00B2704781880088081AB6
:10181000401C00B2704781880088081A401C00B242
:10182000704781880088081A401C00B27047F0B5E4
:1018300004464FF4FA66C1F341307710642501285D
:101840000BD121F4C040B04207DCB84201DDC0F545
:101850007A70584390FBF5F001B2C2F34130012891
:101860000BD122F4C040B04207DCB84201DDC0F524
:101870007A70584390FBF5F002B2944201DA2046A8
:1018800000E01046884201DA0846F0BD944201DAD1
:101890002046F0BD1046F0BDF0B504464FF4FA66A0
:1018A000C1F341307710642501280BD121F4C040E9
:1018B000B04207DCB84201DDC0F57A70584390FBB6
:1018C000F5F001B2C2F3413001280BD122F4C0403F
:1018D000B04207DCB84201DDC0F57A70584390FB96
:1018E000F5F002B2944201DA204600E01046884248
:1018F00001DA0846F0BD944201DA2046F0BD1046F8
:10190000F0BD002208B51146104600F027F80090FF
:10191000BDF8000008BD002208B51146104600F0D1
:1019200036F80090BDF8000008BD18B54C09BDF8A8
:101930000030D20864F30203ADF80030C308BDF8EC
:101940000000890863F3C70080B262F30C2080B204
:1019500061F34F30ADF8000080B218BD18B54C09E6
:10196000BDF80030D20864F30203ADF80030C308BC
:10197000BDF80000890863F3C70080B262F30C2051
:1019800080B261F34F30ADF8000080B218BD18B5D9
:101990004C09BDF80030D20864F30203ADF8003002
:1019A000C308BDF80000890863F3C70080B262F382
:1019B0000C2080B261F34F30ADF8000080B218BD4A
:1019C00018B580B2030243EA102083B288B2010244
:1019D00041EA1020121D0C4980B2D40840EA0040B0
:1019E00043EA034208400A40121A624300EB5210D5
:1019F000084040EA104080B2010241EA1020ADF8F0
:101A0000000080B218BD00001FF8E00718B580B2D2
:101A1000030243EA102083B288B2010241EA102097
:101A2000121D0C4980B2D40840EA004043EA034248
:101A300008400A40121A624300EB5210084040EA84
:101A4000104080B2010241EA1020ADF8000080B2DF
:101A500018BD00001FF8E00781B2C1F3C402C2EB59
:101A6000C20000EB0220C01D4209184662F3174075
:101A70004A07920E02EB513202EB420303EB0222C1
:101A8000D21C920962F30F20C1F30421C1EBC10201
:101A900002EB0121C91D490961F30700FF2161F330
:101AA0001F607047FF2208B511461046FFF76FFF11
:101AB0000090BDF8000008BD7CB50E7BDDE9065442
:101AC000022E08D94E88002E05D0A54203D0CDE9BC
:101AD00000544469A0477CBD38B50446102116F077
:101AE00000FB01206080FF202073BDF80010002063
:101AF00060F3020189B260F3C70189B260F30C217F
:101B000089B260F34F31ADF8001088B20090BDF893
:101B100000000090BDF80000208038BD2DE9F04F96
:101B200085B0824610B294468B460FFA82F9AAEB32
:101B3000000EDDF838800FFA8EF2049203F5B471CE
:101B4000ABEB00021E4613B203920AEB0002119C9B
:101B50005844029212B207B2019088457DD04FF4EA
:101B6000B4718E4202D9A6F5B476B6B2884503D9CF
:101B7000A8F5B4701FFA80F80F99ACEB010000B221
:101B80000090109818B101EBD1704010401C05B2C4
:101B90005A21B6FBF1F0B8FBF1F1C0B2C9B204288A
:101BA00000D10320042900D1032188427ED146457B
:101BB0007CD868B3012854D0022878D003287ED17D
:101BC00006F15A0000B213F05FFC009910FB01F11E
:101BD0000AEBE130401B208030B213F055FC10FBC3
:101BE00009F10BEBE130401B608008F15A0000B2B4
:101BF00013F04AFC10FB09F10AEBE1302844A08005
:101C00000FFA88F013F040FC009910FB01F15AE143
:101C100030B213F039FC009910FB01F10BEBE1300D
:101C2000401B60805A3630B213F02EFC10FB09F1D5
:101C30000AEBE1302844A0800FFA88F013F024FC6E
:101C400010FB09F10BEBE1302844E08008F15A0069
:101C500000B213F019FC009900E0E6E010FB01F17E
:101C600029E030B213F010FC10FB09F10BEBE1306E
:101C70002844E0805A3630B213F006FC009910FB7D
:101C800001F10AEBE1302844A0800FFA88F013F04C
:101C9000FBFB009910FB01F10BEBE130401B608076
:101CA00008F15A0000B213F0EFFB02E036E009E061
:101CB00005E010FB09F10AEBE130401B208005B084
:101CC000BDE8F08F06F15A0000B213F0DDFB10FB07
:101CD00009F10AEBE130401B208030B213F0D4FB55
:101CE000009910FB01F10BEBE1302844E0800FFA82
:101CF00088F013F0C9FB10FB09F10BEBE130401B3E
:101D0000608008F15A0000B213F0BEFB009910FB8E
:101D100001F10AEBE1302844A080D0E730B101287E
:101D200037D0022861D003287ED099E001297CD1E8
:101D300008F15A0000B213F0A7FB10FB09F10AEBFF
:101D4000E130401B20800FFA88F0029013F09CFBDA
:101D5000074630B2804613F097FB874201DA0298BB
:101D600000E0404613F090FB009910FB01F10BEBF3
:101D7000E130401B60805A3630B213F085FB10FB17
:101D800009F10AEBE1302844A08001982844E08062
:101D900095E7022964D1AEEB050020800FFA88F0A8
:101DA00013F072FB10FB09F10BEBE130401B60807C
:101DB00006F15A0000B2019013F066FB074608F1E5
:101DC0005A0000B2804613F05FFB874201DD0198A4
:101DD00000E0404613F058FB009910FB01F10AEBBC
:101DE000E1302844A08030B269E0032938D106F1FF
:101DF0005A0000B213F048FB10FB09F10AEBE13086
:101E0000401B20800398401B608008F15A0000B2FC
:101E100013F03AFB10FB09F10AEBE1302844A080F3
:101E20000FFA88F0804601E019E019E013F02CFB6E
:101E3000009910FB01F730B2064613F025FB00991C
:101E400010FB01F0874201DD404600E0304613F010
:101E50001BFB009910FB01F00BEBE03096E729B17A
:101E6000049820806380A280E78028E708F15A0068
:101E700000B2039013F008FB074606F15A0000B2C7
:101E8000019013F001FB874201DA039800E001980A
:101E900013F0FAFA009910FB01F10AEBE130401B54
:101EA000208030B213F0F0FA10FB09F10BEBE130B7
:101EB000401B608002982844A0800FFA88F013F03D
:101EC000E3FA10FB09F10BEBE1305FE72DE9F0419C
:101ED0001D0017460E4604461AD0F07A02281AD979
:101EE000D4F81CC0BCF1000F03D02046E047012805
:101EF00011D02B463A4631462046FBF793FB01288A
:101F000009D006A239462046BDE8F04107F0A3BC3F
:101F100002A23946F8E7BDE8F08100004E6F0A647E
:101F20006174610038B58469049D002C01D000956E
:101F3000A04738BD38B50446182116F0D2F8002263
:101F400011461046FFF7F1FC0090BDF8000000902C
:101F5000BDF800002081FF20E072401C608001205D
:101F6000207538BD704700002DE9FF4FADB0887E69
:101F70003A9E98460C4602287ED9206800287BD0DD
:101F80002D98006A002877D0202216A816F081F834
:101F900020681590B8F1000F6ED098F80000002866
:101FA0006AD02D982F9982682AA808F032F8002864
:101FB00062D0207FB0F1000A01D14FF0010A607FAA
:101FC000810703D42F98FFF714FC0FE0B4F9121027
:101FD000009141F6FF72CDE90120B4F91430414679
:101FE0001FA8226813F01CFBBDF97C001599B4F9F9
:101FF00012200025B1F908906F1E02EB09011F9114
:102000002F990988ADF80C102F994A88ADF80E2049
:10201000B4F916102791B4F918100A44ADF80E203F
:10202000EEB1E1B92F99B1F90210002917DAB368BE
:102030005A1A002A00DCCA1A1F994FF480634942D9
:1020400003EB41018A4200DD37603168002906DB7D
:102050000D46BDF80E10B2881144ADF80E10627F27
:102060000021CDE90012B4F91420249008EB0507F3
:1020700003463846159900E09FE008F09BFD47199C
:102080002BE0617F0020CDE90001B4F9142008EBBA
:102090000700249B159908F08DFD3D464719BDF8B2
:1020A0000E101F98084400B2ADF80E008EB110F566
:1020B000806F0EDB306800280BDA35602F98BDF991
:1020C0000E10B0F90200081A70602F98B0F90200E3
:1020D000B06018F8050000286FD02D98BDF90E10DB
:1020E00080684944B0F902008142CADB5046CDF80D
:1020F00088A0BAF1020F02D0032816D029E0607F31
:102100000090B4F91430791B08EB0500159A13F010
:10211000E8FA06462F98FFF76CFB801BBDF80C1001
:1021200000EBD07001EB600011E0607F0090B4F92B
:102130001430791B08EB0500159A13F0D2FA064605
:102140002F98FFF756FBBDF80C10801B0844ADF824
:102150000C00D4E9019AD14502D94846D1468246BD
:10216000A07F800717D012A800F023FAA089ADF84D
:102170004800159890F90E0000B90120ADF84A000A
:10218000A07E8DF85000A07FC1089DF8510061F33A
:1021900001008DF8510000202090FFF7B2FB239042
:1021A000FFF7AFFB029004A800F04EFF208AADF8C5
:1021B0001400BDF90C0026905FE163E1BDF80C103E
:1021C000279800260844ADF80C0008EB0500259080
:1021D0001E96781B2890B3E00021A9F57F4200915C
:1021E000FF3A09D0AAF57F42FF3A05D0A74A29183D
:1021F00040461268904700901EAB29AA21A9259855
:1022000008F0C0FC607FC00710D02198232802D0BE
:10221000012E12D00AE026B1012E06D0022E0AD0DD
:1022200004E01E98012620908AE00026E0680290D3
:10223000022E41D042E0002682E0202807D11E99DC
:102240002098081A072803D0A0890226239077E057
:10225000209A259968461144062215F01AFF00209D
:102260008DF806009DF80100FEF768FE06469DF811
:102270000000FEF763FE06EB001023909DF80300BC
:10228000FEF75CFE06469DF80200FEF757FE06EBE1
:10229000001B9DF80500FEF751FE06469DF8040060
:1022A000FEF74CFE06EB0010C2B223980BF0FF01C4
:1022B000C0B2FFF753FBC8E723980290299A2199EF
:1022C00015980FF044F883464FF6FF70814522D0F1
:1022D000824520D0009848451DD350451BD2BDF8FB
:1022E0000C00ADF80000BDF80E10ADF80210A28A87
:1022F0000244ABF101001044ADF804001F986A4697
:10230000401E0844ADF8060004A92D9800F088FE90
:10231000E089ADF80800BDF80800ADF8640003AA34
:1023200016A9219B2D9800F032F9BBF1000F07DDB3
:10233000BDF80C00A18A014401EB0B00ADF80C00C4
:1023400028991E9881423FF647AFA07F800723D58A
:102350002698ADF800002068BDF94A1001ABB0F92D
:10236000080001EBD17100EBD070401000EB610070
:10237000BDF80E106A460844BDF80C10ADF8041004
:10238000ADF80200ADF80600BDF80800ADF8480051
:1023900012A92D9800F000F9A07FC0071FD0269841
:1023A000ADF800002068BDF80E1001AB028940892D
:1023B0001144091A15986A4690F90D00081ABDF8DB
:1023C0000C10ADF80410ADF80200ADF80600BDF831
:1023D0000800ADF8480012A92D9800F0DDF8617FE3
:1023E0000020CDE9000108EB0706B4F914203046BF
:1023F000249B159908F0DEFB3D4647192F9800886D
:10240000ADF80C002298022802D0032815D027E04E
:10241000607F0090B4F91430791B3046159A13F0A0
:1024200060F906462F98FFF7E4F9801BBDF80C1001
:1024300000EBD07001EB600010E0607F0090B4F919
:102440001430791B3046159A13F04BF906462F9835
:10245000FFF7CFF9BDF80C10801B0844ADF80C0055
:10246000BDF80E101F9808442D9900B2ADF80E006B
:102470008968B1F90610884204DC18F805000028C4
:102480007FF49CAE31B0BDE8F08F000054380020DE
:1024900038B50446202115F024FEFF20A076FFF772
:1024A00030FA0090BDF80000A0810B4820604FF684
:1024B000FF706060A060FFF724FA0090BDF8000094
:1024C000E081052011F046FB0090BDF8000020825D
:1024D0000020E07638BD000010DA0408036C002B01
:1024E00000D018477047436C002B00D01847704746
:1024F0002DE9F0410546C06B17460E46002826D050
:10250000E86C11F055F804001CD0E96C15F0E9FDF9
:10251000FAF78EF9296821626968E161A968A16109
:1025200000683A462146007CC0F3801084F82400FD
:102530003068206070686060EB6B28469847050043
:1025400001D003E0FEE7204611F0BEF82846BDE8C2
:10255000F08170B50C46054601F07DFF206A2860C9
:10256000E0696860A069A860FAF762F9006894F809
:102570002420016962F386110161AA6C12B121461F
:10258000284690472046BDE8704011F09DB830B411
:10259000046AA44630BC604730B44C88002C06D096
:1025A0000C7A022C03D9446AA44630BC604730BC84
:1025B000704738B504460A2115F093FD012060806C
:1025C000FF202072BDF80010002060F3020189B2E4
:1025D00060F3C70189B260F30C2189B260F34F3117
:1025E000ADF8001088B20090BDF800000090BDF872
:1025F0000000208038BD000010B504460A4A0020C3
:1026000052F8303023B1401CC0B21028F8D301E09A
:10261000102802D34FF0FF3010BD42F8304002EBDB
:10262000C002516010BD0000BC9900202DE9FF4F91
:1026300081B08B460E9C15461E46B4F90A10B4F9BB
:102640000C00571AB4F9082004F1100AABEB02028F
:1026500004F13C09B4286DDAB4F90E30B42B7DDAFC
:1026600000287BD0002BFCD0984277DDA94276DC95
:10267000616D79434FEAA12CA16A7F1C79438912CD
:10268000A0F20F14582C01D8002909DB441E592C44
:1026900001D8002904DB5B38B32802D2002900DD11
:1026A0000021A3F20F10582801D8002909DB581E79
:1026B000592801D8002904DB5B3BB32B02D2002947
:1026C00000DD0021ACEB010001EB60000124871A62
:1026D000B74200DD3746002F0DDD3BB22A46594692
:1026E000CDF800A0019800F09FF9040003D139460D
:1026F000019802F092F8B74200DD3746002F00DA69
:1027000000270BEB070001B2F61B019833B2074418
:10271000CDF800902A46384600F086F9050003D12E
:102720003146384602F079F8AC4277D1204605B000
:10273000BDE8F08F68DDB4F90E30B42B64DD98424B
:1027400062DDA9420BDB616DA46A79437F1C7C4387
:102750008912A412A0F20F17582F01E054E0A5E04F
:1027600001D8002C09DB471E592F01D8002C04DBAF
:102770005B38B32802D2002C00DD0024A3F20F1036
:10278000582801D8002C09DB581E592801D8002CE4
:1027900004DB5B3BB32B02D2002C00DD0024081BC2
:1027A00004EB60000127841AB44200DD3446002C9B
:1027B0000DDD23B22A465946CDF80090019800F06D
:1027C00033F9070003D12146019802F026F8B442FC
:1027D00000DD3446002C00DA00240BEB040001B2CB
:1027E000361B019833B20444CDF800A02A46204697
:1027F00000F01AF9050003D13146204602F00DF829
:10280000AF4251D1384692E74FF001084746B4280D
:1028100005D040B10ADAA94203DC09E044E0A9424C
:102820000FDC03200CE0A942FBDC0AE0A942F8DD42
:1028300033462A465946CDF800A0019800F0F4F836
:102840008046B4F90E00B42806D050B1B4F90A009D
:102850000CDAA8420CDC0DE0B4F90A00A84207DC4F
:1028600011E0B4F90A00A8420DDC01E0A84201DC45
:10287000032708E033462A465946CDF800900198D0
:1028800000F0D2F80746B8F1000F09D047B1B8F10F
:10289000030F03D0B8F1010F04D005E0032F03D1DB
:1028A000002044E7012F01D0022040E701203EE74D
:1028B0002DE9F8430546884640F26710411C089C04
:1028C0001746002B01DA002302E08B4200DB0346AF
:1028D000002C01DA002402E08C4200DB04469C421A
:1028E00003DAC3F5B470204403E0E01A002800DCEA
:1028F000181BA5F86800AB81EC81A5F808806F81F2
:1029000015482860012028718B4200D9FEE7B42BBE
:1029100001D2002000E00120002C01DB8B4200DD11
:10292000FEE7B42C05D3A4F1B401B42901D20026EA
:1029300000E0012600903A46414605F1100000F003
:10294000C6F823463A46414605F13C00009600F0A1
:10295000BEF8BDE8F88300002D2601082DE9F843F4
:102960001E4617468846814600250C4C0DE0009017
:10297000D0F800C033463A4641464846E047002872
:1029800008D0022800D10125083420680028EED1A3
:1029900015B10220BDE8F8830120FBE7BC990020B7
:1029A00010B50179022906D0052913D18068BDE848
:1029B000104010F089BE0446406900280AD0016921
:1029C000002904DA406810F07FFE6069EFE7416992
:1029D000491E416110BD000070B5124D060007D0C0
:1029E000002455F83410B9B10879022805D002E066
:1029F0002868002800D0012070BD887CB1F9102023
:102A0000C007304601F1080102D007F09AFB01E04F
:102A100007F027FB0028EED0641CE4B2102CE0D3B2
:102A2000002070BDBC990020F8B5069CA58A266AD6
:102A3000521B658A12B2491B94F8285009B24FEA1A
:102A4000C57526B100948DB3FEF7C8FBF8BD85B1FE
:102A5000207C810728D000F00301012924D002291D
:102A600001D1511C20D4C043800719D1002A1BDC9E
:102A700016E0227C02F00304022C15D0D543AD07EA
:102A800012D0012C01D100290EDC920701EB0302C8
:102A900008D0002A04DB494200D5002199420DDB11
:102AA0000020F8BD002A02DA0120F8BD0CE04A42FD
:102AB000F6D49A4206DA991A104401E0002901DBA3
:102AC00001F0ABFE0220F0E7FEF72FFCEDE72DE969
:102AD000FC471C46DDF8288016460F468146B42B7D
:102AE00001DDB43C24B204F15A0000B212F0CCFC77
:102AF00007EB6015204612F0C7FC06EB601000B231
:102B0000CDE900082BB232463946484600F002F8BB
:102B1000BDE8FC872DE9F0470F46DDE908699846D6
:102B2000154604462C2101F078FEB54206D1B9F1D4
:102B3000030F03D16D1E761E2DB236B2B54205DDF0
:102B40004046B846074630462E46054627816581F1
:102B5000A4F80C80E68184F810906782A8EB070047
:102B60004B46A582002801DD024601E0A7EB0802E2
:102B7000711B002901DD0D4600E0AD1BAA4294F84F
:102B8000282002DD42F0010201E022F0010284F877
:102B900028200025E561244E2660A5612571D60711
:102BA0004FF480150DD020B195FBF0F64E43B612D0
:102BB000E66121B195FBF1F141438812A061E06922
:102BC0000CE021B195FBF1F64643B612A66120B1A7
:102BD00095FBF0F048438012E061A06920629807FD
:102BE00009D003F00300012808D0022813D0D843ED
:102BF000800714D006E022F0020001E042F002005B
:102C000084F82800206A81106162002801DA4842B5
:102C10006062BDE8F087206A0028EFDCEBE7206AFD
:102C20000028EBDDE7E70000292A01082DE9FE4F27
:102C30000546DDF830900F461C4699F81200904684
:102C4000C0F3000BB9F91060684609F10801FEF7FE
:102C50008BFDBDF90210BBF1000F2FD041454FDCB9
:102C6000BDF9061041454BDBBDF900008119B942A1
:102C700005DCBDF904203919921B914209DDBDF92B
:102C800002108B1943453FDCBDF90620931B4345D9
:102C90003ADBBBF1000F18D0C01B00D50020A042CA
:102CA00030DCBDF90410C91B091A491C4218A242A4
:102CB00000DD211A002925DB2844F4E0414513DC1E
:102CC000BDF9061041450FDBCEE7C61BA6420BDC63
:102CD000002E03DB3146284601F09FFDBDF90400BC
:102CE000C71B7F1C002F02DC0020BDE8FE8FA7421F
:102CF00003DAE11BE81901F090FD1EB9A74201D1EA
:102D00000120F2E70220F0E7BDF80430C21B181AD8
:102D1000401C0FFA80FCBDF80600401A401C03B2AC
:102D2000A8EB010000B2B04202DA301A401E01E006
:102D3000991B401AD9F8141000B20223CF6803EB94
:102D40004003FB5A37F81080A3EB0803ADF80830B6
:102D50008B68496833F8103037F8100000EB010A2F
:102D600002EB0C00801B18440FFA80F99019C01A6E
:102D7000401E07B2BBF1000F4FF0000621D06DE0FE
:102D8000811B01EB0A0010F801BC09EB06005FEAA9
:102D9000000808D4A04506DA15F80810584605F0D2
:102DA00020FD05F80800B7EB060808D4A04506DAB0
:102DB00015F80810584605F014FD05F80800761CB3
:102DC00036B2BDF908008642DADB09EB0600A04204
:102DD00001DA014600E02146002901DA002002E084
:102DE000A04200DB204600B2211A284401F015FD64
:102DF000BDF90800381A411CA14201DA0A4600E078
:102E00002246002A01DA002402E0A14200DA0C4640
:102E100021B2284647E0811B01EB0A0010F8010CA3
:102E2000C0F1FF0B09EB06005FEA000808D4A045DB
:102E300006DA15F80810584605F0D3FC05F8080026
:102E4000B7EB060808D4A04506DA15F8081058466E
:102E500005F0C7FC05F80800761C36B2BDF908007D
:102E60008642D8DB791CA14201DA781C00E02046BA
:102E7000002801DA002704E0A14201DA7F1C00E00B
:102E800027463AB2A9EB0200A11A884201DA0346AA
:102E900000E00B46002B01DA002002E0884200DB54
:102EA000084601B2A81801F0B8FC2BE72DE9F04163
:102EB0001546064688880A881C46801A401C02B2BD
:102EC000C8884B88C01A401C00B2824200DA104603
:102ED000B5EB600F00DD4510002D00DA002506F18E
:102EE0000800FEF741FC3582B47437483060022098
:102EF00030710023BDB1354A00204FF47A77C0EB22
:102F0000C00102EB8101B1F91810A9421BD1C0EB3D
:102F1000C00002EB80004169491C41610269102D2B
:102F200004DA012103E07361BDE8F0812911114445
:102F3000B94205DA102D01DA012100E029115718F4
:102F400007617061F0E7401C0428D8D300242046B4
:102F5000C0EBC00102EB8101D1F814C0BCF1000F3D
:102F600007D12CB1D1F810C0D4F810E0F44500DA44
:102F70000C46401C0428EBD33CB16069401CC4E9FA
:102F80000430102D0EDA01200DE01C2010F010FB93
:102F9000040006D01C2101F040FC4FF0FF302061FE
:102FA0000BE0FEE728111844B84205DA102D01DACB
:102FB000012000E028111F1827612046294674616E
:102FC000BDE8F041FAF72BB82D2C01084C990020F0
:102FD000F0B50026094D0746344605EBC4004068AD
:102FE000B84204D155F83460204600F009F8641C5A
:102FF000E4B2102CF1D33046F0BD0000BC990020A3
:103000000021421C08D0054A002352F8301042F833
:10301000303002EBC000436008467047BC99002086
:1030200030B4D38854881B1B5B1C1BB2012B09DBFB
:10303000938814881B1B5B1C1BB2012B02DB0369EA
:1030400030BC184730BC704738B50446382115F0FD
:1030500048F8FEF727FD0090BDF8000024F8040FA3
:10306000FEF720FD0090BDF800006080FEF753FCE5
:103070000090BDF80000E080FF2525720220A072BC
:10308000FEF749FC0090BDF800006083FEF743FCAA
:103090000090BDF8000020850748206104F8015C1D
:1030A000A57584F82650A57784F83250E07F20F08B
:1030B0003E001E30E07738BD10DA04082DE9F04FED
:1030C000C7B08346DDE95065087B984614460F4635
:1030D00002287DD9B7F90200002879D0AE4277D016
:1030E0001AB281469246404500DD914601A8FFF79D
:1030F000ABFF787B00F003008DF80600B86840B1A4
:1031000000208DF80700B8680590387B8DF81E0008
:1031100005E0387B8DF807003888ADF80800218875
:10312000A8F10102A1EB0803ADF8F8306188A1EB2A
:103130000800ADF8FA0021881144ADF8FC10B4F88D
:1031400002C0ADF800316244ADF80411ADF8FE20C4
:10315000ADF80201ADF80621B7F802C06344ADF83E
:103160000031B7F802C060440FFA80FCADF802C12C
:103170007888081AADF804017988C01A511A4FF0FE
:10318000FF3231920022401C09B200B2ADF80611A4
:103190004292002813DDA1EB0C00401C00B2002875
:1031A0000DDD012347F6FF7240A932A8FFF77EFE2E
:1031B00001204290002132A8FFF71EFA319000232F
:1031C00047F6FF723EA938A8FFF770FE002100E025
:1031D00028E038A8FFF710FA439006F5B470A8422B
:1031E00005D005F5B4714FF4B4708E4220D147F686
:1031F000FF70ADF804003EAA01A95846FFF710FF82
:103200004398FFF7FDFE3198401C02D03198FFF73C
:10321000F7FE38A8FFF7C4FB4298002802D032A876
:10322000FFF7BEFB47B0BDE8F08FA6F5B476B6B2A7
:103230008642FAD202E0A5F5B475ADB28542FAD263
:1032400028B245900090B4F90220B4F9001033B2CE
:103250000FA84493FFF72CFB00210FA8FFF7CCF930
:103260004690B54203D9A81BC0F5B47000E0701BAE
:10327000DBF8081000913C282ADDB8F10A0F27D9A5
:103280005A20B6FBF0F1B5FBF0F000F00300ADF80A
:10329000B40001A8ADF8ACA0ADF8B05001F0030146
:1032A0002E902A94ADF8AE60ADF8B210ADF8B6909D
:1032B0003EA8CDE92F0B2AA8FBF7B4FF2AA8FCF7FC
:1032C00079F82AA8FCF745F92AA8FCF730FA04E0B7
:1032D0003EAA01A95846FFF7A3FE0FA8FFF760FB1F
:1032E00038A8FFF75DFB429810B132A8FFF758FBF2
:1032F0004698FFF785FE4398FFF782FE3198401C01
:1033000002D03198FFF77CFE787B40078AD509F020
:10331000FF022AAB51464498FDF780FDBDF8A80096
:1033200021882AAA0844ADF8A800BDF8AC0021887D
:103330000844ADF8AC00BDF8AA0061880844ADF8B7
:10334000AA00BDF8AE0061880844ADF8AE0042A8FE
:10335000009906F05EFE42ADC0B1002347F6FF7251
:103360002AA92CA8FFF7A2FD00212CA8FFF744F9F9
:10337000064658463EAA01A9CBF80850FFF750FE72
:103380003046FFF73DFE2CA8FFF70AFB09F0FF02CD
:103390002AAB51464598FDF741FDBDF8A8002188AC
:1033A0002AAA0844ADF8A800BDF8AC00218808445A
:1033B000ADF8AC00BDF8AA0061880844ADF8AA00D9
:1033C000BDF8AE0061880844ADF8AE0042A800998F
:1033D00006F01FFEC0B1002347F6FF722AA92CA8F1
:1033E000FFF764FD00212CA8FFF706F904463EAA6A
:1033F00001A95846CBF80850FFF712FE2046FFF708
:10340000FFFD2CA8FFF7CCFA0098CBF8080009E7DD
:1034100070B514460D460646FAF71EFA22462946AE
:103420003046BDE87040FAF7E6BB7CB50446087E3E
:103430000D4602280ED9A2686846296806F0E9FD03
:10344000002807D0626B0AB120469047626D29467A
:10345000204690477CBD2DE9F04FCD6889B00C46E1
:10346000804615B1207C00286ED0207C012800D138
:103470000025D8F80400FEF7C2F90790D8F8082014
:1034800005A8216806F0C5FD00285DD0F9F7D0F940
:1034900083460068D8F80090C16951BB007C4006A3
:1034A00011D4D8F80400BDF91410B0F90020B0F917
:1034B0000200891ABDF91620121A079800FB0211A2
:1034C00009EB410014E0D8F80410BDF91630B1F949
:1034D0000200B1F90010181A079B584300EB400096
:1034E00000EB0902BDF91400401A00EB4000104443
:1034F0008146D4F804A05FEA0A0013D02068FEF7E2
:103500007EF906462068BDF91410B0F90020B0F924
:103510000200891ABDF91620121A06FB02110AEBE5
:10352000410A00E0002645B3DBF80000007C0007FC
:1035300010D460690CF04FFD0246002108E0685C81
:10354000802802D9FF2001E035E000206854491CA2
:103550009142F4DB6069FEF752F907466069BDF9F4
:103560001410B0F90020B0F90200891ABDF9162034
:103570002944121A07FB021500E00027D8F80400BE
:103580004188008849420AB2404201B205A80CF0C5
:103590005BFDDBF80000C069C8B160680028207ED0
:1035A0000CD001A9009681E8A100534605A9484620
:1035B000079A05F0B1F809B0BDE8F08F8DE8A100D9
:1035C000A36805A94846079AFDF7D9F9F3E7607E95
:1035D00078B161680029217E23D00096CDE903707F
:1035E000CDE90115534605A94846079A04F066FE41
:1035F000E1E760680028207E0AD001A9009681E8F2
:10360000A100534605A94846079A04F011FFD2E7E6
:103610008DE8A100A36805A94846079AFDF70CF8B4
:10362000C9E7CDE90270CDE90015A36805A94846B0
:10363000079AFCF763FFBEE72DE9F0471F46914666
:10364000DDE9082AB7F9024014FB09F001EB40015B
:10365000B7F900000A9B01EB4005B3F9021001FB2A
:103660000AF102EB4101B3F9002001EB4206B988EF
:10367000081A401C00B24FEA40080AE028463146CA
:10368000424614F006FD641C05EB490506EB4A06AC
:1036900024B2B7F90600A042F0DABDE8F0872DE9C0
:1036A000FF4F9BB00C461B981546DDF8A0B0816813
:1036B00017A8FEF762F817A8FFF78EF91390208875
:1036C00018B96088B0F5807F01D0012000E00020AB
:1036D000149006A81C2114F004FDE07A8DF8300047
:1036E000207B0EAF00F00F008DF831000697DDE96A
:1036F000131001434FF000062CD1BBF1040F06D08C
:10370000BBF10E0F0AD0BBF1140F21D022E0A07A3A
:1037100000BB1E9806A9CDE9065013E01B98294668
:103720008268684606F075FC00280ED01E98079641
:103730000B9509902089ADF8200002208DF8280013
:1037400006954BE01B98FFF770FE1FB0BDE8F08FA9
:10375000A07A78B31B9880680188ADF8381080880B
:10376000ADF83C001B9880684088ADF83A001B9883
:103770008068C088ADF83E002846FEF746F81590F0
:103780002846FEF71EF812900EA8FEF71AF881469A
:103790000EA8FEF73AF88046F9F74AF80DF0E0FB7C
:1037A00006460EA80CF017FC01464046B14217D859
:1037B0004E4617E0FFE72846FEF727F8044628465E
:1037C000FDF7FFFF1E9907910A46610001FB0020EB
:1037D0000990069502200B958DF8280006A9B1E7FF
:1037E000B6FBF8F67043169040000FF00FFF8246CC
:1037F00016980FF00BFF8146099002208DF82800E3
:10380000BDF93E000D90761EBDF83A001996304481
:103810000B97CDF81CA0ADF83E00BBF1040F05D10D
:10382000208818B96088B0F5807F01D0022000E0C0
:1038300001208DF82800C0E00EA910A8FDF79DFF1B
:103840006888404202B22888404201B210A80CF0B9
:10385000FBFB149870B1CDE9024BCDE904A9159991
:103860001298CDE9000110A9159B1E9A1B9800F033
:10387000D7FD0BE0CDE9014BCDE903A915980090E8
:10388000024610A8129B1E99F9F7FAFDA07A0228A9
:1038900061D9218989B2C1F3C40212FB00F2ADF8EB
:1038A00008204A07920E02EB513212FB00F2ADF8EB
:1038B0000A20C1F3042111FB00F1ADF80C10C0F196
:1038C000FF00002344E00AEB43073988ADF80410F9
:1038D000BDF80420BDF80810C2F3C40616FB0011A1
:1038E00001EBC11606EBC131BDF80060C1F3C45154
:1038F00061F3C7065107890EBDF80AC001EB5231CA
:1039000011FB00C101EBC11C0CEBC13C4FEA9C6CEC
:103910006CF3020601EBC11C0CEBC131C1F3C251C7
:1039200061F34F36BDF80C10C2F3042212FB0011F4
:1039300001EBC11202EBC131C1F3C45161F30C269A
:10394000ADF80060B1B20091BDF8001039805B1C89
:1039500016998B42B7D31398E0B14E46BDF93A7031
:1039600014E0BDF9381043463A463046FEF7F6FFFC
:1039700010B1022804D006E03046414614F0B1FBF5
:1039800002208DF828007F1C46443FB2BDF93E005E
:10399000B842E6DA06A91B98FFF747FDBDF83E00DE
:1039A0001999401CADF83A00084400B20D99ADF8E1
:1039B0003E00884201DDADF83E10BDF93A100D9889
:1039C00081427FF739AF48460FF06CFE50460FF04A
:1039D00069FEBAE610B50C460846582114F081FB82
:1039E0001048606110482061104820631048206230
:1039F0001048A061104860621048A0621048E06260
:103A0000104860631048A0631048E06310482064C9
:103A1000104860641048A064104860652C20E06481
:103A200010BD0000BD3001086541010811340108D6
:103A30002F3C01089F360108453D0108E93E010879
:103A40009D4101081F44010839360108333B010834
:103A5000613A0108B33A0108293C010857340108CA
:103A60002DE9F04117460C460646F8F7E1FE0546FB
:103A7000F8070ED0A16A606921F0004114F031FB13
:103A8000A06A40F00041A1622868016941F040014C
:103A900007E0A06A20F00041A1622868016921F0D6
:103AA0004001016160690834C6E90004B460BDE802
:103AB000F081FEB50546006802900098164620F099
:103AC000E00000900C466868FDF7A5FE009960F3E1
:103AD000942100916868C1884088081A0099401CA8
:103AE00060F35F510091A06A002801DA052000E030
:103AF000042060F304010091206A2860E069686096
:103B0000A069A860F8F794FE006894F824206B463A
:103B1000016962F38611016104F108023146284609
:103B2000FEF7D4F9284600F096FC68460EF0AEF891
:103B3000FEBD70B5064615460C46D00701D00020E4
:103B400070BDA80743D5A06A00F0004000F5C04052
:103B5000A06220460CF03FFAA16A400021F000422A
:103B6000824202D960F31E01A162A06A20F00040E7
:103B70000FF01EFD2146606168B9A06A00F00040A8
:103B800000F54060A06220F000400FF011FD2146DA
:103B900060610028D4D00846D0E900128160E2605C
:103BA0006188E181A1892089081A401CA16A00B2BC
:103BB00021F0004100EB400291FBF2F12182A16A69
:103BC00021F0004191FBF0F0411061822AE00846AB
:103BD000D0E900128160E2600CF0FDF94100A06ABA
:103BE00061F31E00A06220F000400FF0E1FC606174
:103BF000A16A21F0004114F074FAA06A05F00105F1
:103C000065F3DF70A0626069002899D0306004F12C
:103C100008007060B060F8F70BFE0068016965F39A
:103C200086110161204670BD48690FF04DBDF0B5A9
:103C30001D46074697B014460E46086800232A46DC
:103C40000FA90DF0DEFAF0B3BDF84420002A3FD0F2
:103C5000BDF842C0BCF1000F3AD02088BDF8461034
:103C6000084401B2ADF84C10306803894089181A35
:103C7000638801EB0C041844BDF84830801AC01A60
:103C800003B2ADF84E30B868B0F900C064451FDB30
:103C9000B0F90440A1421BDC9918B0F9022091420E
:103CA00016DBB0F90600834212DC29460F980DF0AE
:103CB000A4FA00280CD00F99097B890708D10FAB13
:103CC00013AA314600E005E000903846FAF7CCFD33
:103CD00017B0F0BD202DFBD3A5F57840FF38F7D005
:103CE000A5F500500C38F3D02088BDF84610BDF87B
:103CF0004820084401B26088104402B2BDF8440074
:103D0000104400B20090BDF84200084403B214A869
:103D10000CF0A7F901A8FFF797F902208DF807002A
:103D20008DF82E008DF83A008DF81E00B089ADF8A0
:103D300022000120ADF824003B6914AA01A93846ED
:103D40009847C5E72DE9F0471546B1F9022092B032
:103D50001C460E468146002A7ED0307A02287BD946
:103D6000B5F90010B4F90000814205D1B5F902306F
:103D7000B4F90270BB426FD0814200DA084602EB10
:103D8000D271A0EB6100ADF84000B5F90000B4F9C4
:103D90000010B6F90220884200DC084602EBD2711E
:103DA00000EB6100ADF84400B5F90200B4F902106F
:103DB000B6F90220884200DB084602EBD271A0EB84
:103DC0006100ADF84200B5F90210B4F90200B6F98D
:103DD0000220814200DD084602EBD27100EB610057
:103DE000ADF8460010A90846D9F8082006F011F9E8
:103DF000002875D010A9D9F808A0C9F80810B5F99D
:103E00000200B4F90210884206D123462A46314600
:103E10004846FAF78DFE0EE0B5F90000B4F900103F
:103E2000234688422A463146484602D1FBF7ECF841
:103E300001E0FAF73BFF707A010701D440074DD546
:103E40006846FFF701F93088ADF8040047F6FF70C7
:103E5000ADF80000307A00E042E08DF80300B6F9DA
:103E60000200471040F3000000F10108707A40079B
:103E700018D528880EAAC01BADF838006888C01B6A
:103E8000ADF83A002888C119A1EB0800ADF83C0054
:103E90006888C119A1EB0800ADF83E0069464846A4
:103EA000FFF7BEF8707A000718D520880EAAC01B4D
:103EB000ADF838006088C01BADF83A002088C11901
:103EC000A1EB0800ADF83C006088C119A1EB080027
:103ED000ADF83E0069464846FFF7A2F8C9F808A0C9
:103EE00012B0BDE8F08700002DE9FF4F8BB01F46F0
:103EF0001646032B7ED3002E7CD0B8000FF086FB35
:103F000004007BD000253068206028467A1E15E02A
:103F100006EB800136F92030B1F904C0634505D1C4
:103F2000B1F90230B1F906C0634505D004EB850351
:103F300009686D1C1960ADB2401C80B29042E7DB8D
:103F400006EB8700B6F9001030F9042C914205D138
:103F5000B6F9021030F9022C914206D004EB85012B
:103F600050F8040C6D1C0860ADB2032D43D37C489F
:103F7000D0E90010CDE90210002027E0BDF90810BB
:103F800034F92020914200DB1146ADF8081004EB13
:103F90008003BDF90A10B3F90220914200DB1146FB
:103FA000ADF80A10BDF90C1034F92020914200DC64
:103FB0001146ADF80C10BDF90E10B3F90220914274
:103FC00000DC1146401CADF80E1080B2A842D5D3DB
:103FD0000B9802A9826805A806F01BF858B10B9847
:103FE00005A90026806809900B988160B4F9022029
:103FF000012010E002E020460FF054FB0FB0BDE8B6
:10400000F08F04EB8001B1F90210914201DA0A4607
:1040100006B2401C80B2A842F3D32C2105FB01F06C
:104020000FF0F4FA8346B2460490D1464FF00008F0
:10403000701E00D528446A1E09F1010107929142C1
:1040400000DD002134F8203034F8262034F82170C7
:104050009B1A04EB8000BA1A478804EB860004EB35
:104060008101408849883E1A081A0021089116FBF0
:1040700002F110FB03F0814267DA0120089001E0B1
:104080000898E8B307980AF10106864200DD002689
:10409000B9F1010700D52F4404EB860004EB8A0137
:1040A000B0F90200B1F90220904216DB12D034F9C7
:1040B000263034F92A108B420CD04FF0010CCDE998
:1040C000000C5846FEF726FD58460499FEF794FA70
:1040D0000BF12C0B08F10108B246A84523D004EBE4
:1040E000870004EB8901B0F90200B1F90220904287
:1040F00017DB13D034F9273034F929108B4200E054
:1041000023E00BD00026CDE900065846FEF702FD5D
:1041100058460499FEF770FA0BF12C0B08F10108D0
:10412000B946A845ACD3DDE90B0102AAFEF778FF3A
:104130000498FEF74DFF04980FF0B4FA20460FF0F4
:10414000B1FA0B990998886058E7BAF1010600D5D1
:104150002E44079809F1010787429DDD00279BE760
:104160007C9E010870B514460D460646FBF700FC20
:10417000224629463046F9F76FFB2246294630464B
:10418000F9F739FD224629463046F9F726FE224640
:1041900029463046BDE87040FAF7E1BF2DE9FF4FF0
:1041A00099B00F4628984FF480314FF00A0BB0F9C0
:1041B0000000DDE92A6540420F9028984088B1FB55
:1041C000F0F00F990E9091FBFBF4289804F1010A8E
:1041D00040681290604200EB800001EB400920B281
:1041E00011F052F901900FFA8AF011F04DF95A349A
:1041F000009020B211F048F980460AF15A0000B24E
:1042000011F042F9019AC9F10A0101FB02F4009B85
:1042100001FB08F100FB091103FB094391FBFBF0D3
:1042200093FBFBF20D9050110C900D9840110D90E6
:10423000BDF9480000021090BDF94A00000211903B
:10424000B8883988401A401C04B2F8887988401A26
:10425000401C00B21790002049E014A80090B7F964
:10426000021013AB01EB0A02B7F9001008A805F021
:104270000EFD16A80090B7F9021015AB01EB0A026B
:10428000B7F9041008A805F002FDDDF84CC0159838
:10429000149AA0EB0C0816980021831A0846012CEA
:1042A00007DD601E4FEA082191FBF0F11B0293FB32
:1042B000F0F0289B80320CF1800C1B7DDB07299BE2
:1042C0001CD00DF10C08CDF800C088E85100CDE9F4
:1042D0000121CDE90653DDE91B01DDE92623F8F7CD
:1042E000EBFB0AF1010006EB4406254400B21799E6
:1042F00082468842B1DB1DB0BDE8F08F042B4BD065
:10430000052B10D0062B47D0142BEAD1DDE91B3842
:10431000CDF81080DDE926EBCDE90010CDE902C231
:10432000B146002078E0DDE91BE3CDE900100393FE
:10433000269B0293B146E346DDF89C80002028E0EE
:10434000009941430BEB21230199414302EB2121C9
:104350001B124FEA212C08D403998B4205DABCF1D9
:10436000000F02DB02998C4502DB002129540EE08C
:104370000CFB083303EB430303EB0E010B7891F8BE
:1043800001C003EB0C2329F810308B782B54401C10
:1043900000B2A042D4DBA4E70DF10C08CDF800C0B8
:1043A00088E85100CDE90121CDE90653DDE91B0183
:1043B000DDE9262304F0CBFE93E70099029A4143FE
:1043C00002EB21220199DDF80CC041430CEB2121C5
:1043D00012124FEA212107D4DDF810C0624503DA3A
:1043E000002901DB714502DB0021295412E001FBA9
:1043F0000B2C03EB4C0C09EB4008BCF800C0A8F8F0
:1044000000C00BFB0EFC03EB4C0C624401FB0B21C8
:104410000A782A54401C00B2A042CEDB61E7704704
:104420002DE9F04387B08946DDE91251DDE91076C8
:10443000DDE90E8C70B1C46A002C08D0CDF8008084
:10444000CDE904510396CDE901C74946A04707B01D
:10445000BDE8F083FEE7416B002900D008477047B4
:1044600010B5174917481FF022FF38B114491548F5
:104470001FF037F9124913481FF019FF12480CF0CA
:1044800091FF1148432101704FF4007141800F49A1
:1044900081600F49C1600F4901610F4941610F49B6
:1044A00081610F49C1610F4901620F4981620F4962
:1044B00041620449C162BDE810400CF077BF0000C2
:1044C000583F040870420020AC970020250B0108DB
:1044D000550A01086D0B0108BD0B0108850B010889
:1044E000A50B01088D0A0108710A0108B50A010827
:1044F0002DE9FC418646807815460C4610FB04F0F9
:104500000012824203DCBEF80000BDE8FC819EF888
:1045100008C00EEB8C0212F8023C13FB04F31B12D2
:104520009D4202DB32F8040CEFE70022012324E075
:104530000EEB8307BF7817FB04F73F12BD421ADC6E
:104540000EEB830737F8040DADF804000198FDF772
:1045500083FA0646B888ADF804000198FDF77CFAA6
:104560000146B87810FB04F0BA79001212FB04F28D
:10457000C0EB222203E05B1CDBB29C45D8D8E2B33F
:10458000281A00B2C0EB002090FBF2F0C0B2C0F1DC
:10459000FF02C1F3072313FB00F3C6F3072414FB48
:1045A000023303EBC31404EBC334BDF80050230FF4
:1045B00063F30205C1F3074313FB00F3C6F3074798
:1045C00017FB023303EBC31707EBC3339B0E63F3F5
:1045D000C705C9B211FB00F0F1B211FB020000EBFC
:1045E000C01101EBC030800E60F30C25600E60F34B
:1045F0004F35ADF80050A8B287E7FFE7FEE7416806
:10460000002901DA0FF060B870470000FEB50546DA
:10461000407A16460C4640072ED0224F387820B9F3
:10462000002000F043F801203870687A00F007009D
:10463000022817D0304680EA6400684001900020CC
:1046400000906A4601A91848FCF798FC01280BD095
:10465000324621462846F8F701F9009000280BD091
:10466000002418E02046E6E700980422416802EBA7
:10467000B1714FEAB1014160FEBD22462846FFF705
:1046800037FF02900098BDF80810806800EB4400E6
:10469000641C018024B20098B0F90E10A142ECDC39
:1046A000FEBD000068370020330A010870B5094DCF
:1046B000044628680FF008F820460EF079FF2860BD
:1046C000054DA86020B1214613F00BFD6C6070BD54
:1046D000FEE7000010380020683700200146002067
:1046E0000F290AD2DFE801F009090909080A080CB4
:1046F0000E10120C0E101200102070471820704778
:10470000012070470220704704207047082070473E
:1047100001460020891E0D2909D2DFE801F00708B3
:104720000807080707070707070707000120704762
:1047300001460020032901D0062900D1012070473D
:10474000032130B10078A0F120015F2903D80120B6
:10475000704708467047802801D302207047002028
:104760007047000038B5174C2078002829D10EF08A
:10477000C1FFF8F765F805F001FEF7F75BFD05F0FE
:1047800003FEFDF7EFFBF7F757FF4FF4B4710E4848
:1047900006F01FF95C210D4806F01BF9F8F74EF8FA
:1047A00005F0D8FE0A4800909DF80000112802D0BC
:1047B000002010B1FEE70120FBE70CF0DEFC012039
:1047C000207038BD4C3700200C980020189800202D
:1047D000443322112DE9F0410A4C07460A4D606826
:1047E0000E46401CC100606028680EF091FF2860F2
:1047F00038B1616800EBC10040E902760846BDE8C7
:10480000F081FEE7543700200038002013F041BC4F
:1048100013460A46194613F05DBC13F062BC13F050
:1048200060BC13F05EBCFF2213F054BCFF2213F0F7
:1048300051BC2DE9FF410C46074602F043F90646FC
:10484000E00702D0384602F0E5F8F8692043F86145
:10485000E00711D00221384601F056FE60B138461B
:1048600000F016FF050007D00CF0B2FF28460DF04F
:104870002FF808B102F0CEF8384602F023F9B04222
:1048800002D114F0C07F07D0384600F041FF02F09B
:1048900052F9384602F04FF9E0060CD502AA6946F3
:1048A000384601F09CF86946384602F0D6F802A96D
:1048B000384602F0D2F8BDE8FF81028C11438A42EB
:1048C00001D003F0A2B870472DE9F047174688469B
:1048D0004FF6FF79054600234A46394605F004F9AC
:1048E000698C00240426C1F30513EA6808E006EB8E
:1048F000C40010585FEA801C01D4C00102D5641CBA
:10490000A342F4D84FF0806000EBB1204FEAB050E2
:104910006884C0F30510C10010460EF0F9FEE8608F
:10492000688C6FF00703C0F3051009E0E96803EB3A
:10493000C00C01EBC0026144D1E900C1C2E900C171
:10494000401EA042F2D8E868082100EBC40013F032
:10495000C8FBE96841F83480E86806EBC4014258B6
:1049600067F3170242504A4639462846BDE8F047E9
:1049700002F0E4BC10B504468068002813D10B484F
:104980004168491C41601C200EF012FEA06058B125
:104990001C2113F0A6FBA1680F204876A068017EB9
:1049A00041F00301017610BDFEE700004C37002006
:1049B0002DE9FC410D460746012101F099FD002833
:1049C00050D1384600F0A8FE044600F043FE0646EB
:1049D0000CF0F6FAA0420ED030460CF0F9FAA042E4
:1049E00009D030460CF0DAFAA04204D030460CF080
:1049F000CDFAA04236D14FF400263146384601F0B8
:104A00007EFD18BB3846F7F72CFD044607F114016C
:104A10006846FCF78EFEBDF800002946001BADF885
:104A20000000BDF802006A46001BADF80200BDF8A8
:104A300004002044ADF80400BDF806002044ADF8A1
:104A40000600084605F0E5FA00280CD000230122F4
:104A50002946384601F07AFC38461DE0012101F074
:104A600047FD10B10020BDE8FC813146204601F031
:104A700046FD80B9D4E90501CDE9000100230122FA
:104A80006946204601F062FC29466A46084605F060
:104A9000C0FA0028E7D0204600F03AFE0400DDD13D
:104AA0000120E0E72DE9F0410E460746002401F021
:104AB00019FC050035D03146384601F007FC0228C4
:104AC0002FD905EBD570012101EB60053146384641
:104AD00001F002FC28440FFA80F83146384601F014
:104AE000E9FB05463146384601F0EAFB002D01DDC1
:104AF000294600E06942002801DD024600E042420A
:104B0000914205DD002D01DD284604E0684202E007
:104B1000002800DC4042404400B2002800DA204671
:104B200004463146384601F042FB05000ED03146BE
:104B3000384601F030FB022808D93146384601F0EA
:104B400030FB2844A04200DB044624B238463146FC
:104B5000692201F062FB05B2384631466A2201F053
:104B60005CFB00B2854200DD2846002801DD2044C0
:104B700004B22046BDE8F08170B50D4606465B22C2
:104B800001F04BFBC4B230462946162201F045FB2A
:104B900004B90124204670BD002803D00068884273
:104BA00001D1012070470020704700002DE9F0413D
:104BB000074605460E464FF00008354800E02D68D0
:104BC000ADB1A9690142FAD0A869C0F30F15284612
:104BD0000EF0EEFC041E31D0294613F082FAC4E92F
:104BE000007601256F1F26B1B06880B333E04546DB
:104BF000EDE70CF09DF906001CD0F26802B3706A74
:104C0000401C8100706210460EF082FDF060716AF7
:104C100007EB81014450A4F81480A4F8168000200A
:104C20000CF09EF9401E208300200CF0DFF9401E9E
:104C3000608322E020460EF047FD0020BDE8F081B1
:104C400004200EF0B5FCF06004607562E3E7FFE756
:104C50003046FFF78FFEB068016881B14168491C9A
:104C60004160B068890000680EF052FDB1680860CC
:104C7000B168496807EB810144502046DEE7042013
:104C80000EF096FCB16808600460B0684560F4E717
:104C9000F0FF0F0070B5054601F04DFF002000F059
:104CA00093FA284610F04AFA284600F06FF80120DF
:104CB00000F08AFA4FF6FF724FF47021284602F096
:104CC0003DFB284602F022FB0CF0F6FD030007D066
:104CD000284601F0E9FE18B1294618460CF024FDDB
:104CE000284600F015FD04000DD02A4622210CF0C4
:104CF00019FA2A46232120460CF014FA2846BDE86A
:104D0000704001F087BE70BD7FB50C46064601F0CD
:104D1000D9FE0546E0060CD502AA6946304600F0E9
:104D20005EFE6946304601F098FE02A9304601F069
:104D300094FEF069A043F061E0070ED0304601F028
:104D400069FE304601F0BEFE38B1304600F0E0FCAE
:104D500001F0F1FE304601F0EEFE304601F0B2FE09
:104D6000A84202D114F0C07F07D0304600F0D0FC3A
:104D700004B0BDE8704001F0DEBE7FBD028C22EAC7
:104D800001018A4201D002F040BE704770B505684B
:104D90000446286818B120602046FFF7F7FF256019
:104DA0006A682846002A03D02146BDE870401047B3
:104DB00070BD2DE9F0414D680C46EDB1284600F07C
:104DC0002DFD0646284600F0F5FD07462846002141
:104DD000102201F022FAE98A12220844C01BE08264
:104DE000401E60832846002101F017FAA98A084472
:104DF000801BA082401E208341F20200E061002D52
:104E000005D043F20200E06143F20230E06140F07D
:104E1000740040F40060E06102D040F40040E061C2
:104E2000BDE8F08110B501460348FFF7BFFE044618
:104E3000FFF730FF204610BD209D01082DE9F0410D
:104E4000074601F0E7FD384600F062FC4FF0000431
:104E50000500264608D1384600F0FCFB040018D0B7
:104E60002069B84200D10126384603F0E1FC65B163
:104E7000284602F027FD0022222128460CF052F994
:104E80000022242128460CF04DF9002E01D00020EC
:104E90002061BDE8F081000070B50C46084605F0C1
:104EA00057FA002000F090F92046144A002102F041
:104EB0001BFB012000F088F900212046FCF720FBB5
:104EC000204600F0E5FB10B120460CF044FDA06840
:104ED000002811D00068002518B10EF0F5FBA0687D
:104EE0000560A068C06818B10EF0EEFBA068C56050
:104EF000A0680EF0E9FBA56070BD0000FFFF0F0089
:104F00002DE9F047A2B080460CF0C1F804464046B7
:104F10000CF0FBF8012700260546122C72D0DFF8B2
:104F20009492152C6CD0182C7AD140460CF0B5F820
:104F3000824601462846FAF7C7FC0021284601F0C0
:104F4000E0F850B105F59070FEF742F8040004D087
:104F5000FDF726FD20460EF0A5FB0021284601F0B6
:104F6000BCF800285CD06846FEF76EF88DF8036048
:104F70008DF81A608DF82A608DF836606A46002137
:104F8000284601F0E9FB0021284601F0C7F98046D8
:104F90000021284601F0BCF9044605F1140120A8BF
:104FA000FCF7BEFBBDF88010A1EB0800BDF8841033
:104FB000ADF8800001EB0800ADF88400BDF8820078
:104FC0005146001BADF88200BDF886002044ADF8C4
:104FD00086000EA800F0F0F820A81B96CDE910700E
:104FE000CDF83C90CDF848D00EAA1A2128460CF0F6
:104FF00099F820AA69465046FEF712F8D4E001E07D
:1050000055E00DE040460CF07EF80446007802289A
:1050100006D00021284601F074F820B1022020704B
:1050200022B0BDE8F0870021284601F03DF9824614
:105030000021284601F072F981460021284601F03E
:1050400067F9804605F114016846FCF769FBBDF875
:1050500000105246A1EB0900BDF80410ADF80000A5
:1050600001EB0900BDF80210ADF80400A1EB080047
:10507000BDF80610ADF8020001EB0800ADF806001F
:105080006946606804F0EDFF68B10021284601F030
:1050900018F8FD2807D328460021602201F0BDF84A
:1050A000C0B2FD2801D22770BAE72670B8E74046A3
:1050B0000BF0F3FF80466846FDF7C6FF0021284647
:1050C00001F00BF828B19DF8230040F001008DF8A5
:1050D00023006A460021284601F03EFB00212846B5
:1050E00001F01CF907460021284601F011F9044699
:1050F00005F114018A4620A8FCF712FBBDF88000D8
:105100004146C01BADF88000BDF884003844ADF8BE
:105110008400BDF88200001BADF88200BDF8860057
:105120002044ADF886000EA800F046F820A8CDE98E
:105130001060CDF83C90CDF848D00EAA1A21284630
:105140001B960BF0EFFF0021284600F0DAFF20B19C
:10515000BDF8000008B1012700E00027049C07B15A
:10516000049620AA69464046FDF75AFFE7B1182089
:105170000EF04CFA0746BDF9002000235146FDF71A
:1051800095FE05F590713846FDF736FA64B18DF855
:1051900003608DF822608DF82A608DF8366020AAB1
:1051A00069464046049427E70EAA1B2128460BF0C7
:1051B000B9FF35E7209D010870B50D46044648212A
:1051C00012F08FFF256070BD014908707047000024
:1051D0005C3700202DE9FF41884608460BF057FF59
:1051E000044640460BF057FF0546012C23D0082CFF
:1051F00023D0032C3ED02A2C3ED00D2C4CD00E2C8C
:105200007DD0092C7CD00A2C7BD00F2C7AD0292C75
:1052100079D0222C78D0242C77D0132C76D0152C52
:1052200003D0182C01D0122C34D104B04046BDE874
:10523000F041FFF765BE2021FAE02021FFF79EFD37
:1052400040460BF03BFF0DF072FB002822D10821F5
:10525000284601F04DF900281CD095F820004FF0A9
:105260000101C007284602D0FFF788FD30E0FFF7B4
:1052700024FB2DE02021F8E000F05CF90646002434
:1052800006E0A868006850F8240001F054FC641C93
:10529000B442F6D3BDE8FF81082101F029F9F8B145
:1052A00040460BF030FF0478132C06D0112C04D0AC
:1052B000142C07D0122C05D008E001212846FFF756
:1052C000FCFA03E001212846FFF758FD0A2CE1D043
:1052D00004B02846BDE8F04100221C210BF022BF9B
:1052E0004FF40161284601F003F90028D2D0284686
:1052F00001F0CDFB0028CDD10027284607E06DE066
:1053000095E09AE0B0E0B5E0D1E0F2E0F6E000F040
:1053100085FA0646284600F0E1FA044640460BF0BE
:10532000F2FE007812281BD011280CD013282BD0A5
:105330001428AFD1284600F049FA800703D0002E88
:1053400038DC002C36DC284600F0A7F90446284655
:1053500000F03EFBE11704EB9171A0EBA1000BE024
:10536000284600F09AF90446284600F031FBE11780
:1053700004EB917100EBA10001B204B03A4628465B
:10538000BDE8F04102F088BA284600F01FFA800715
:10539000E6D0002E01DC002CE2DD284601F089F881
:1053A0000446284600F00DFBE11704EB917100EB79
:1053B000A1000BE0284601F07CF80446284600F0E6
:1053C00000FBE11704EB9171A0EBA10001B204B066
:1053D0003A462846BDE8F04102F048BA4FF48061F1
:1053E00001F086F818B10121284602F022FA284679
:1053F00000F04EF90CF066FA064602240DF062FA4F
:1054000010B940460BF05AFE0DF09DFA022801D06B
:10541000042800D106241EB144F00801284607E004
:1054200021462846FFF749FA082128461DE0402179
:1054300004B0BDE8F041FFF740BA4021FFF79EFC01
:10544000284600F0F2FD02287FF424AF02AA694644
:10545000284600F0C4FA6946284601F0FEFA02A97F
:10546000284601F0FAFA15E70E2104B0BDE8F04134
:10547000FFF784BC002100F0FFFD04460021284610
:1054800000F04DFE204302D0284601F054FB284690
:1054900000F050F80646002406E0A868006850F8BE
:1054A000240001F048FB641CB442F6D3F2E600216C
:1054B000012200F0B2FE06B228460021042200F0CC
:1054C000ACFE04B20021284600F0D6FD07460021BC
:1054D000284600F024FE384305D142F2D1708642BE
:1054E00001D08442BFD104B02846BDE8F04101F0AC
:1054F00022BB688C40F002006884F4E70021FFF7CB
:10550000D1FA014604B04046BDE8F0410BF02ABE96
:105510008068002809D0002902DA4268511803D4B3
:1055200043680A468B4201D800207047006850F853
:10553000220070478068002800D04068704770B52E
:105540000C46054600F114012046FCF7F2F8A86865
:10555000002812D02188808A081A2080A968A08893
:10556000898A0844A080A9686088898A401A608076
:10557000A968E088898A0844E08070BD70B50C464F
:105580000546002100F0B1FD06462146284600F000
:105590005BF8704202B2114620460AF048FD002135
:1055A000284600F016FE2188084420800021284665
:1055B00000F01BFEA188081AA0800021284600F0F8
:1055C00020FE6188084460800021284600F0F5FD37
:1055D000E188081AE08070BD2DE9F04106460021FF
:1055E00000F00FFE05460021304600F0E6FD0446BF
:1055F0000021304600F079FD0746304600F04DF8B6
:10560000401B001B794200EB410000B2BDE8F08175
:105610002DE9F0410646002100F0DBFD05460021A2
:10562000304600F0E2FD04460021304600F05DFD0A
:105630000746304600F03DFF401B001B794200EB5F
:10564000410000B2BDE8F0810A4600F114011046A5
:10565000FCF76FB810B5416809B100F05DF8044679
:105660000A4805F099F90EE00022416A05E0C36896
:1056700053F82230A34208D0521C9142F7D8014679
:10568000024805F09BF90028EED110BD0C980020CF
:105690008068002800D0806870471430FCF77FB81D
:1056A00070B5064600F034F8051E08D0002408E066
:1056B00021462846FFF72CFFB04201D1204670BD9D
:1056C000641C2846FFF736FFA042F1D84FF0FF30A8
:1056D00070BDF0B4458C00240426C5F3051712E014
:1056E000C56806EBC40C55F80C505FEAC51C09D51B
:1056F00025F07F459D4205D1C06850F83400F0BCCC
:105700000EF094BF641CA742EAD8F0BC002070479A
:10571000002800D04068704700B50146FFF7F8FF49
:105720000028FAD1084600BD2DE9F047DFF8949033
:1057300080464C46FFF7FEFE06460025DFF888A0AF
:105740000FE0D8F808005146006850F82570384638
:1057500000F0D5FE20B9B7F91A00A04200DB0446DC
:105760006D1CB542EDD30021404600F050FD82464D
:105770000021404600F027FD06460021404600F08B
:10578000BAFC05464C4505D0B8F81A00801B401BF2
:10579000201A04B2404600F051FC07464046FFF78D
:1057A0007CFFA0EB0A00801B694200EB4100391A24
:1057B000404600F00DF9081A00B2844200DD204690
:1057C000BDE8F08701E0FFFF01000400806818B128
:1057D000407E00F00F0070470F20704770B50C46F8
:1057E00005460C49FBF7BCFE10B1806A404202E05E
:1057F000284600F0E6F8208007492846FBF7B0FE6F
:1058000010B1806A404202E0284600F0E1F8608072
:1058100070BD0000759401088D9401082DE9F84FC2
:105820000646002100F03AFC012807D0B0680028A5
:1058300002D0008A404200B2BDE8F88F0021304615
:1058400000F0D9FC00900021304600F0C8FC8146F1
:105850000021304600F04FFC824641F6FF7B5C465B
:105860003046FFF767FE804600250EE0B068194914
:10587000006850F82570384600F041FE20B9B7F9AD
:105880001400A04200DC04466D1C4545EED35C4587
:1058900006D0B28A09EB0A001044001B04B200E0F3
:1058A0000D4C304600F0D8FB0546304600F001FEB6
:1058B0000099411AA1EB0901CAF1000001EB400077
:1058C000291A304600F07DF8084400B28442B3DD66
:1058D0002046B1E70100040001E0FFFF2DE9F04799
:1058E0000646002100F0DAFB01280AD0DFF8A0907C
:1058F00030464C46FFF71EFE80460025DFF894A098
:1059000015E0B068002801D0B0F91000BDE8F087BC
:10591000B0685146006850F82570384600F0EFFD39
:1059200020B9B7F91800A04200DB04466D1C4545BC
:10593000EED30021304600F05EFC074600213046E1
:1059400000F04DFC82460021304600F0D4FB0546B5
:105950004C4504D0308BC01B401B201A04B230468B
:1059600000F07AFB8046304600F0A3FDC11BA1EB9E
:105970000A00694200EB4101A8EB0101304600F04A
:1059800020F8081A00B28442C0DD2046BEE70000BD
:1059900001E0FFFF010004008068002802D0007EC3
:1059A000C0F3810070478068002802D0007EC0F3F9
:1059B000011070478068002802D0408A404200B23F
:1059C00070478068002802D0008A404200B27047C9
:1059D0008068002802D0408A404200B270472DE91A
:1059E000F04F8DB016460C464FF0FF3705460022AB
:1059F0003B461146204600970AF033FB00223B4607
:105A00001146304600970AF02CFB1021284600F082
:105A10006FFD002816D0284600F007FB070011D0C4
:105A200000200CF055FF8046022F08D010E00CF04B
:105A30007EFFA84209D040460CF04AFF8046B8F1EC
:105A4000000FF4D10DB0BDE8F08FB8F1000FF9D020
:105A50002846FFF7AFFF09902846FFF765FE0C9038
:105A60002846FFF7DBFE07902846FFF737FF0B902D
:105A70002846FFF7ABFE8146002019F00C0F03907B
:105A800014D0012F10D0032F02D0022F07D00DE029
:105A90000998002808DC0C98002805DC06E0404640
:105AA0000CF036FF0C2801D1012003900020029059
:105AB0005FEA897014D0012F10D0032F02D0022F7B
:105AC00007D00DE00798002808DC0B98002805DCBB
:105AD00006E040460CF01CFF032801D10120029093
:105AE000DDE902010843ADD04FF48037394628463E
:105AF00000F0D4FA012800D000200A903946284648
:105B000000F085FB01903946284600F05CFB0890C8
:105B10003946284600F063FB80463946284600F0A7
:105B20006AFB814628460122394600F076FB0FFACF
:105B300080FB2846FFF7B1FD0090284600F0B9FC35
:105B40000690039800B158468246029800B1584624
:105B5000059028463946212200F05FFBC0B202289A
:105B600008D228463946312200F057FBC0B202283D
:105B7000FFF468AF09990098A02701440C980844E5
:105B800000B204900398002870D004980028FBD03D
:105B9000E88A7080688BF0800A9840B1A98A01EB8E
:105BA00008003080ABF101010844B08007E0298B88
:105BB000A1EB0900B080A0EB0B00401C3080DDE9B8
:105BC0000001411A0898091A0598081A00990990C5
:105BD0004843049990FBF1F000B2039000200BF0D1
:105BE000ADF900EB8001502000EB4100B0F5A07F43
:105BF0000ADB00200BF0A2F900EB8001502000EB43
:105C0000410090FBF7F000E001200399884201DA9F
:105C1000084616E000200BF091F900EB80015020BF
:105C200000EB4100B0F5A07F0ADB00200BF086F905
:105C300000EB8001502000EB410090FBF7F000E00A
:105C40000120099900B2091A0AB2009B0499C91AE5
:105C500009B200290BDCE98A019808447080698B3D
:105C60000898091A0598081A401EF08090E00C9BCD
:105C700012FB03F393FBF1F1511A019AEB8A1144E1
:105C8000194409B2401E71800844F080B5F916200D
:105C900001981044814238DA708000200BF04EF9F0
:105CA00000EB8001502000EB4100B0F5A07F0ADB43
:105CB00000200BF043F900EB8001502000EB410085
:105CC00090FBF7F000E00120B6F902100844B6F9A5
:105CD0000610884219DD00200BF030F900EB80013E
:105CE000502000EB4100B0F5A07F0ADB00200BF054
:105CF00025F900EB8001502000EB410090FBF7F00C
:105D000000E0012071880844F080B5F91A20059858
:105D1000B6F90610121A0898101A814238DDF08080
:105D200000200BF00BF900EB8001502000EB41004C
:105D3000B0F5A07F0ADB00200BF000F900EB80013A
:105D4000502000EB410090FBF7F000E00120B6F995
:105D50000610081AB6F90210884219DA00200BF072
:105D6000EDF800EB8001502000EB4100B0F5A07F82
:105D70000ADB00200BF0E2F800EB8001502000EB82
:105D8000410090FBF7F000E00120F188081A7080D4
:105D9000DDE9060101440B98084400B20590029821
:105DA00000283FF44FAE05980028FAD0698B089878
:105DB000081AE080A0EB0B00401C6080A88A2080BD
:105DC000288BA0800698A0EB0801A1EB0901A1EBAC
:105DD0000A00019006994843059990FBF1F000B242
:105DE000009000200BF0AAF800EB8000502606EB94
:105DF00040004FF4A07B584509DB00200BF09EF8D3
:105E000000EB800006EB400090FBF7F000E0012083
:105E10000099884201DA084613E000200BF08EF862
:105E200000EB800006EB4000584509DB00200BF03A
:105E300085F800EB800006EB400090FBF7F000E0F7
:105E40000120019900B2091A0AB2DDE90513C91A45
:105E500009B2002916DCA98A0A9840B14144AAF186
:105E6000010008442080298BA1EB090008E001EB28
:105E700008002080298BA1EB0901A1EB0A00401E3C
:105E8000A080DFE50B9B12FB03F393FBF1F1511AAA
:105E90000A9A09B2EAB3AA8A401E531808EB0A020A
:105EA000991809B221800844A080B5F91400104463
:105EB000884233DD208000200BF040F800EB8000AA
:105EC00006EB4000584509DB00200BF037F800EBEB
:105ED000800006EB400090FBF7F000E00120B4F9F1
:105EE00000100844B4F90410884217DD00200BF0BC
:105EF00025F800EB800006EB400058450ADB002047
:105F00000BF01CF800EB800006EB400090FBF7F074
:105F100001E039E0012021880844A080B4F9041090
:105F2000B5F9182077E0A08000200BF007F800EB0F
:105F3000800006EB40005D46A84272DB00200AF0BC
:105F4000FDFF00EB800006EB400090FBF7F0B4F99A
:105F50000410081AB4F90010884292DA00200AF0FE
:105F6000EDFF00EB800006EB4000A8425BDB002069
:105F70000AF0E4FF00EB800006EB400090FBF7F036
:105F8000A188081A20805DE5AB8A4144194409B212
:105F9000401E21800844A080B5F9142002EB0800BF
:105FA000814232DA208000200AF0C8FF00EB800036
:105FB00006EB4000584509DB00200AF0BFFF00EB6C
:105FC000800006EB400090FBF7F000E00120B4F900
:105FD00000100844B4F90410884216DD00200AF0CD
:105FE000ADFF00EB800006EB4000584509DB0020C8
:105FF0000AF0A4FF00EB800006EB400090FBF7F0F6
:1060000000E0012021880844A080B5F91820B4F9E7
:106010000410A2EB0A02A2EB0900814283DC11E525
:10602000FFE7012093E70120AAE7806818B1007E0E
:1060300000F00300704703207047000008B50549D1
:106040006A46496800912C210BF06CF8BDF90200FA
:1060500008BD00003C9D010808B505496A4609686D
:1060600000912C210BF05EF8BDF9000008BD000086
:106070003C9D0108008C704710B5092200F0CDF856
:10608000C0B210BD10B5092200F0C7F8C0B210BDF3
:1060900010B5162200F0C1F8C0B210BD10B516221E
:1060A00000F0BBF8C0B210BD70B50C46054620220A
:1060B00000F0B3F8024621462846BDE87040F6F7E6
:1060C00000BA10B5212200F0A8F8C0B210BD10B57A
:1060D000682200F0A2F8C0B210BD10B5342200F062
:1060E0009CF8002800D0012010BD10B5322200F02D
:1060F00094F800B210BD10B5322200F08EF800B254
:1061000010BD10B5172200F088F8002800D001203B
:1061100010BD10B5042200F080F800B210BD10B51B
:106120000A2200F07AF880B210BD10B50A2200F001
:1061300074F880B210BD10B5602200F06EF8C0B2E5
:1061400010BD70B50E460546FFF7F5FF02281AD9B7
:10615000FF24FD2802D2C0EB0020040A0EB1002665
:1061600003E02846FFF7D4FA054655B131462846E4
:10617000FFF7E1FF022806D9FD28F2D24443240AA2
:10618000EFE7022C01D8002070BDFD2C01D3FF20C9
:1061900070BD204670BD10B5372200F03EF8C0B289
:1061A00010BD10B5382200F038F800B210BD10B59F
:1061B000352200F032F800B210BD10B5112200F007
:1061C0002CF800B210BD10B5112200F026F800B274
:1061D00010BD10B5122200F020F800B210BD10B5AD
:1061E000122200F01AF800B210BD10B5132200F010
:1061F00014F800B210BD10B5132200F00EF800B272
:1062000010BD10B5102200F008F800B210BD10B596
:10621000102200F002F800B210BD2DE9F8430E463E
:10622000074615460121104601F050FF8046002424
:1062300014E06B462A4631463846FAF779FD0446A3
:10624000012824D0B8F1000F0CD0022C02D00EB1DE
:10625000002603E03846FFF75BFA0746002FE8D137
:10626000012C14D01EB9012D05D0042D03D02846D1
:106270000EF038FA0AE038680FE0012D0AD0C18A22
:1062800051B160B1012D0CD0B0F91600009000980A
:10629000BDE8F883818AF3E700680028EDD100208B
:1062A000F4E7B0F91400F1E710B50B22FFF7B5FFE2
:1062B00000B210BD10B54122FFF7AFFF00B210BD14
:1062C00010B54222FFF7A9FF00B210BD10B545225C
:1062D000FFF7A3FFC0B210BD10B54322FFF79DFF2B
:1062E00000B210BD10B54022FFF797FF00B210BDFD
:1062F00070B50C4605465522FFF78FFF0246214632
:106300002846BDE87040F6F7DCB85722FFF785BF96
:1063100010B56A22FFF781FF00B210BD10B56922E7
:10632000FFF77BFF00B210BD10B50122FFF775FF2C
:1063300000B210BD10B50722FFF76FFF00B210BD0D
:1063400010B50822FFF769FF00B210BD2DE9FF412B
:1063500007460888ADF800004888ADF802000888B4
:10636000ADF80400C888ADF806008888ADF80800CC
:1063700048880C46ADF80A00A088ADF80C00E0880B
:10638000ADF80E001D4616466946384601F023FD5D
:106390002B463246384601A901F01DFD2B463246F8
:1063A000384602A901F017FD2B463246384603A9AC
:1063B00001F011FDBDF90000BDF90430984201DA89
:1063C000054600E01D46BDF90820BDF90C108A42C3
:1063D00001DA164600E00E46B54203DA984206DBC3
:1063E000184604E08A4201DA104600E008462080A0
:1063F000BDF90030BDF904108B4201DD1D4600E0FF
:106400000D46BDF90820BDF90C00824201DD16469B
:1064100000E00646B54205DD8B4201DD184604E08A
:10642000084602E0824200DD1046A080BDF902303D
:10643000BDF90600834201DA1D4600E00546BDF9BC
:106440000A10BDF90E20914201DA0E4600E0164610
:10645000B54203DA834206DA184604E0914201DAD3
:10646000084600E010466080BDF90210BDF9063014
:10647000994201DD0D4600E01D46BDF90A00BDF957
:106480000E20904201DD064600E01646B54205DDCD
:10649000994201DD084604E0184602E0904200DC23
:1064A0001046E08005221146204609F0C0FDBDE8F7
:1064B000FF811430FBF791B970B50546FFF728F955
:1064C000040012D0E88AE18A451A2046FFF780FAD4
:1064D000054400212046FFF794FE2D1A0021204696
:1064E000FFF703FE281A00B270BDB5F9160070BDA3
:1064F000C069814301D00020704701207047C06906
:10650000084000D001207047008C084000D00120D6
:1065100070477FB50D4606460221FFF7E9FF0028C8
:1065200020D080213046FFF7EFFFE8B902A93046BE
:10653000FFF705F80022294602A803F052FE0400E6
:1065400012D04FF480313046FFF7D2FF70B10120F6
:106550008DF8040000956A46112130460AF0E2FDEC
:106560009DF8040004B070BD0020FBE72046F9E769
:10657000F8B514460D4606465022FFF74EFE00B20F
:106580006080002810D0304629465322FFF745FE90
:10659000C0B22073022807D929463046FFF7D1FD43
:1065A000022802D800202073F8BDFD2804D2217BE8
:1065B00011FB00F0000A2073207B0228F4D952223C
:1065C00029463046FFF729FE024629463046F5F7B0
:1065D00078FF0090BDF80000208030462946542204
:1065E000FFF71BFEA060304629465122FFF715FE3B
:1065F00000B10120617B002D60F382016173D3D073
:1066000029463046FFF763FD617B60F3010161734A
:10661000F8BDF8B514460E4605464622FFF7FDFDC7
:10662000C0B2E072022807D931462846FFF789FD3B
:106630000021022801D8E172F8BDFD2804D2E27AD7
:1066400012FB00F0000AE072E07A0228F4D92180FF
:106650004FF480706080288BA98A4822401A401C21
:1066600000B200EBD0704010A080688BE98A401A1D
:10667000401C00B200EBD0704010E080284631464C
:10668000FFF7CBFD10F0FF00A0720DD0472231467E
:106690002846FFF7C2FD024631462846F5F711FFAE
:1066A0000090BDF800002081002EC5D0314628465C
:1066B000FFF70DFD2073F8BDF8B514460D460646EC
:1066C0005622FFF7AAFDC0B2A076022807D92946B4
:1066D0003046FFF736FD022802D80020A076F8BD2C
:1066E000FD2804D2A17E11FB00F0000AA076A07E56
:1066F0000228F4D929463046FFF7FAFD0090BDF88C
:106700000000A081304629465822FFF786FDA0826E
:10671000304629465922FFF780FD608230462946DF
:106720005A22FFF77AFDA17F60F30201A1773DB104
:1067300029463046FFF7CBFCA17F60F3C501A17766
:1067400029463046FFF7E1FD2060304629465B22AE
:10675000FFF763FD2077F8BDF8B514460D460646F1
:10676000FFF7EFFC074685B1022F09D80020E07043
:10677000A07684F8220084F82A0084F83600F8BD58
:1067800029463046FFF7A3FCA070304629460B226D
:10679000FFF743FD2080E078002857D03046294697
:1067A0002122FFF73AFDC0B2E07002284ED92946F7
:1067B0003046FFF779FC0090BDF80000A08030461D
:1067C00029462622FFF729FD48B1417A490706D01C
:1067D000A31D01460A22184611F05BFC36E0304644
:1067E00029462322FFF719FD0146E07B61F30200F1
:1067F000E073400721D029463046FFF755FC009052
:10680000BDF80000E080222229463046FFF705FD52
:10681000024629463046F5F754FE0090BDF80000C8
:106820006081304629462422FFF7F7FC207230466B
:1068300029462522FFF7F1FC2073304629462722FE
:10684000FFF7EBFCE17B60F3C501E17330462946BD
:106850003222FFF7E2FC00B2208428B394F8220031
:1068600010B3304629463122FFF7D7FCC0B284F876
:106870002200022818D9304629463322FFF7CDFCE2
:1068800094F82310302260F3450184F82310294640
:106890003046FFF7C2FC024629463046F5F711FEA6
:1068A0000090BDF80000E08329463046FFF77FFCEA
:1068B000E084E8B194F82A00D0B129463046FFF7C9
:1068C0006AFC84F82A00022812D929463046FFF7CC
:1068D00068FC2085362229463046FFF79EFC02469A
:1068E00029463046F5F7EDFD0090BDF80000A08484
:1068F000A07E80B3304629462822FFF78EFC206117
:1069000048B3304629462922FFF787FCC0B2A0765B
:10691000022820D92069FDF713FF02286CD02A2213
:1069200029463046FFF779FC024629463046F5F7FE
:10693000C8FD0090BDF800002083304629462B2278
:10694000FFF76BFCE076304629462C22FFF765FC0A
:1069500000B10120207794F8360070B32946304604
:10696000FFF7C0FCE08540B394F83600022824D934
:1069700029463046FFF7AAFC84F8360002281CD9C5
:1069800029463046FFF796FC208629463046FFF719
:1069900097FC608629463046FFF79EFCA08644227D
:1069A00029463046FFF739FC024629463046F5F7BE
:1069B00088FD0090BDF80000A085FD2FBFF4DFAE7C
:1069C00014F8030F10FB07F0000A04F8140BE0782A
:1069D00010FB07F0000AE070E07A10FB07F0000AF5
:1069E000E072E07C10FB07F0000AE074E07F10FB2F
:1069F00007F0000AE077F8BD29463046FFF785FC2E
:106A0000606129463046FFF773FC0090BDF8000036
:106A10002083A0E77CB50546F5F723FD044605F184
:106A200014016846FAF785FEBDF800006946001BB0
:106A3000ADF80000BDF80200001BADF80200BDF883
:106A400004002044ADF80400BDF806002044ADF871
:106A50000600284600F001F87CBD7CB50C460546D2
:106A6000FEF7F8FD0AF0D8FA00280FD02146684654
:106A7000FAF75FFE69462846FDF79AFF002805D021
:106A80002846FEF7E7FD6946F5F778FC7CBD00680F
:106A9000002808D0017E8907F9D0007E00F00300AD
:106AA000012800D0002070470068002809D0017E2E
:106AB00011F00C0FF8D0007EC0F38100012800D047
:106AC0000020704710B504460849FFF718FD08B1CB
:106AD000002010BD2046FEF71BFE0028F9D0002143
:106AE000FFF723FB0028F4D0012010BD01000600B1
:106AF0007CB50546F5F7B5FC044605F1140168467A
:106B0000FAF717FEBDF800006946001BADF800005B
:106B1000BDF80200001BADF80200BDF804002044DF
:106B2000ADF80400BDF806002044ADF80600284684
:106B3000FDF73EFF7CBD10B5418C41F00101418461
:106B4000FEF7EAFD418C41F004014184FEF782FD2D
:106B50004068002803D0BDE8104001F09FBB10BD85
:106B60002DE9F047994616460F468246FEF7E2FCAD
:106B70008046002520E0DAF80800B9F1000F00682F
:106B800050F8254005D04FF480212046FFF7B0FC97
:106B900088B9A08A00233844A082E08A3246304473
:106BA000E082208B394638442083608B30446083F8
:106BB0002046FFF7D5FF6D1C4545DCD3BDE8F087C7
:106BC0002DE9FF47456816460F4604469DB3002150
:106BD0002846FFF7FEFA804600212846FFF711FB02
:106BE00081464FF480212046FFF782FC48B1A98AF4
:106BF00007EB0800084407B2E98A06EB09000844DD
:106C000010E02846FEF7DDFEAA8A02EB0801081A0A
:106C1000384407B22846FEF7DBFEEA8A02EB090198
:106C2000081A304406B200212846FFF75EFA3918E8
:106C300030440FB206B2A08A381A07B2E08A301A7E
:106C400006B20FB9002E43D02046FFF7E3FE02A99B
:106C50002046FEF7F9FC4FF0000875B1694628465A
:106C6000FEF78CFC0022694602A803F0FAF95FEAFD
:106C7000000802D1284600F025FEA08A324638449A
:106C8000A082E08A39463044E082208B00233844D9
:106C90002083608B304460832046FFF761FF25B17D
:106CA0002246222128460AF03DFA2046FFF7B2FE8E
:106CB000002D0DD00022694604F1140003F0D1F933
:106CC000B8F1000F01D1002802D0284600F0FAFDEB
:106CD000BDE8FF872DE9F0410E460746FEF763FE4B
:106CE000A0B93846FEF766FE04463846FEF71CFD9E
:106CF00000280BDA002C09DD4042844200DB044608
:106D000022B233460021384600F088FC3846FEF7B0
:106D100043FE002825D13846FEF780FD044638465C
:106D2000FEF7DCFD054600213846FFF7B7F90128DC
:106D30000BD0002D15DA002C13DD6842844200DBF5
:106D4000044621B23346002206E0002C09DA002D69
:106D500007DD3346002221463846BDE8F04100F009
:106D60005DBCBDE8F0812DE9F0470E4686B00546D2
:106D7000876802A93046FEF767FC3046F5F771FBDD
:106D80000146024602A809F052F902AA394604A8AF
:106D900003F03FF94FF4002420B921463046FFF7B5
:106DA000A7FB00B101205FEA00090DF1100A10D025
:106DB0002A4614213046C5F808A00AF0B3F92A463D
:106DC000152130460AF0AEF92A46162130460AF05F
:106DD000A9F921463046FFF78BFB20B138680090B7
:106DE0007868019006E006F114023946684603F01F
:106DF00010F988B1C5F808D03046FEF79BFB8046F5
:106E0000002407E0B068006850F82410284601F01C
:106E10006DFF641C4445F5D3B9F1000F10D02A462C
:106E200017213046C5F808A00AF07CF92A46182137
:106E300030460AF077F92A46192130460AF072F9ED
:106E4000AF6006B0BDE8F0872DE9F14F82B002983F
:106E5000FFF738FE00287CD10298FEF759FC00901D
:106E600000210298FFF766FA834600210298FFF797
:106E700067FA0546009858B1FEF7CAFB81460098AC
:106E8000FEF7AAFB0746CBF34130012803D013E0FD
:106E90002A4659469AE02BF4C040B0F5FA6F0BDC55
:106EA000B0F57A7F01DDC0F57A7000FB09F064214E
:106EB00090FBF1F00FFA80FBC5F3413001280ED1B1
:106EC00025F4C040B0F5FA6F09DCB0F57A7F01DD3A
:106ED000C0F57A707843642190FBF1F005B200218F
:106EE0006B220298FFF799F904B200216C220298F4
:106EF000FFF793F90FFA80FA0298FFF7DAFA804663
:106F00000298FEF7CAFB0646C4F3413001280FD1B0
:106F100024F4C040B0F5FA6F0ADCB0F57A7F01DDE9
:106F2000C0F57A7000FB08F0642190FBF1F004B228
:106F3000CAF34130012811D12AF4C040B0F5FA6FEC
:106F40000CDCB0F57A7F01DDC0F57A707043642106
:106F500000E05BE090FBF1F00FFA80FA0BEB04002D
:106F600004B205EB0A0005B200210298FFF78AF887
:106F700050B1012828D0801E082825D2DFE800F073
:106F80000C14212C3419393C00210098FFF780F8AB
:106F9000012819D10320EEE709EBD970401008EB66
:106FA000D871A0EB610001E0A9EB0800204404B215
:106FB0000AE007EBD770401006EBD671A0EB61003A
:106FC00000E0B81B284405B22A462146029803B0C7
:106FD000BDE8F04FFFF7F4BD09EBD970401008EBA6
:106FE000D871A0EB610001E0A9EB0800204404B2D5
:106FF000E7E7A9EB080006E009EBD970401008EBC1
:10700000D871A0EB6100204404B2D2E7BDE8FE8F46
:107010002DE9F04F0446408C87B0010501D54005AD
:107020007ED42046FEF774FB5FEA000878D0204645
:10703000FEF7F4FB0590608C002600054FF4FA6B18
:1070400042F2D17A03D52046FFF733FA5DE0002102
:107050002046FFF769F90546504501D1012600E0B9
:107060000026C5F34130012805D125F4C04058451C
:1070700001DC012000E0002081464046FEF7C8FA0E
:10708000074626B12046F5F7F3FE05462BE0B9F199
:10709000000F28D0B8F82200000518D4002140467F
:1070A000FFF742F9504512D100212046FFF71DF8A5
:1070B000054600212046FFF78CF800EB050900216A
:1070C0002046FFF792F8411901EB09000AE025F488
:1070D000C040B0F57A7F01DDC0F57A707843642155
:1070E00090FBF1F005B2204600210222FFF795F84F
:1070F0000FFA80F9204600210322FFF78EF802B232
:107100003B4649462846FAF7C7FB07462046FEF7A6
:1071100051FC0490608C4FF00009400505D500E05B
:107120006BE02046FEF7B9FA53E000212046FEF757
:10713000F0FFA0F51C510546D13906D0002081464C
:10714000C5F34130012802D007E00120F7E725F41C
:10715000C040584501DC012000E000208346404645
:10716000FEF73AFA8246B9F1000F04D02046F5F74F
:107170000BFE05461BE0BBF1000F18D0B8F822004B
:10718000400507D400214046FEF7C3FFA0F51C517F
:10719000D13936D025F4C040B0F57A7F01DDC0F595
:1071A0007A7000FB0AF0642190FBF1F005B22046F2
:1071B00000210522FFF731F80FFA80FB204600215D
:1071C0000622FFF72AF802B2534659462846FAF734
:1071D0002EFB054656EA090605D0DDE90421002309
:1071E000204600F018FB2046FFF763F9B8421BD198
:1071F0002046FEF752FAA84216D1002007B0BDE89B
:10720000F08F00212046FEF770FF05460021204642
:10721000FEF7F7FF00EB050B00212046FEF7CDFF40
:10722000411901EB0B00C1E72046FFF7F3FB69466C
:107230002046FEF709FA02A94046FEF79FF9002210
:1072400002A9684602F00DFF060002D1404600F098
:1072500039FBE08A6D1E2844608300212046FEF73A
:1072600017FF01281CD0A08A7F1E384420836A465D
:107270002921204609F056FF22462221404609F0E6
:1072800051FF2046FFF7C6FB608C002240F0020051
:10729000608402A904F1140002F0E3FE36B904E0B0
:1072A000208BC01B401CA082E1E710B1404600F0DB
:1072B00009FB204600F002F801209FE738B505469B
:1072C000F5F7CFF804460020ADF800006A46132118
:1072D000284609F027FFBDF90000A04202D0284649
:1072E000FFF798FBBDF80000A96831B930B1284616
:1072F000FDF740FBBDF80000A968C882BDF9000099
:10730000A04202D02846FFF785FB38BD70B5054680
:107310000021FFF709F8044600212846FEF7F9FE90
:1073200042F2D1718C4203D0884201D0002070BD5E
:107330002846FFF700FC012070BD00002DE9F84F42
:107340000646514890460C460078002870D03046DA
:10735000FFF760FB04F47F040421404600F0B6FE12
:1073600007460221404600F0B1FE81460121404619
:1073700000F0ACFE00901021404600F0A7FE05464C
:107380004FF6FF7BEFB1B4F5702F12D08CB13046C1
:1073900000210422FEF741FF00B242F2D17A5045AB
:1073A00007D0304600210122FEF737FF00B25045DA
:1073B0004DD100222A21304609F0B4FE3046FFF7B5
:1073C000BAFB4FF4702A544500D084BBD84500D096
:1073D0002FB13046FEF79CF908B1FFF7ACFB5445DE
:1073E00000D024BB1DB3304600216E22FEF715FFEE
:1073F00000B240B9304600216D22FEF70EFF00B208
:10740000B0F5807F01D0022514E0304600216122D2
:10741000FEF703FFC0B2FF2807D1304600216822E3
:10742000FEF7FBFE10F0FF0F03D0012502E00EE097
:1074300028E00025B06820B1817E65F38711817650
:1074400005E025B13046FDF795FAB068F4E75D46F2
:10745000A84502D0B9F1000F02D03046FFF72EFF49
:107460003046FFF7D7FAA84504D0009949EA07004B
:10747000084207D0B4F5803F04D03046BDE8F84F4D
:1074800001F01ABEBDE8F88F5C3700202DE9F0410D
:1074900004460E46408C154600210423C0F3051215
:1074A0000AE0E06803EBC107C059C70103D520F02B
:1074B0007F40A84202D0491C8A42F2D88A4202D1B7
:1074C0000020BDE8F081E06850F8310031460DF051
:1074D000A3F928B1324629462046FFF72FFF01E0E5
:1074E0000028EED00120ECE72DE9F05F0E00044605
:1074F0001FFA82F802F47F074FF6FF7B03D0F07982
:1075000008B94FF0000B00252B4658E0E068042135
:1075100001EBC50A814650F80A004FF6FF7281B2AE
:1075200000F47F0C904501D0414509D1B7F5702F8B
:1075300001D0BC4504D12EB159F83510B14201D06B
:107540006D1C3CE0800104D500233946204602F042
:10755000CBFAE06850F80A10CA0101D489010CD5B1
:1075600050F835000DF0B8F9E06850F835000CF02F
:10757000ABF8E168002041F83500284608230AE00E
:10758000E16803EBC00C01EBC0026144401CD1E98F
:1075900000C1C2E900C1618CC1F30511491E8142DD
:1075A000EED8608C0109491E61F309106084C0F3B4
:1075B0000510C100E0680CF0ABF80123E060608CBE
:1075C000C0F30510A842A1D8002B09D0BBF10000E0
:1075D00006D0024639462046BDE8F05FFFF7AEBE52
:1075E000BDE8F09F70B506460B480078002812D021
:1075F00000200CE0002406E0E86850F82410304633
:1076000001F079FD641C686AA042F5D8284609F0AB
:10761000CDFC0500EED170BD5C370020F0B51546FD
:10762000064691B00C4651EA050078D0012B1DD0DA
:107630003C493046F9F764FF3B493046F9F760FFB3
:1076400000220921304609F06DFD012867D12A4644
:1076500021463046F4F711FF012860D111B03046C1
:10766000BDE8F04000220A2109F05CBD3046FDF77C
:10767000F1FF07466846F9F78BFF2C480096039008
:107680002CB3384609F06CFC401022460021F9F773
:10769000FCFF642801D2642002E0962800D99620DD
:1076A0000B903046FEF78DF94142201A0891CDE942
:1076B00009101D4801901E4807906A46092130466E
:1076C00009F030FD01282AD16846F9F7EBFF002DBB
:1076D00025D0384609F08AFC40102A460021F9F7E7
:1076E000D4FF642801D2642002E0962800D99620B5
:1076F0000B903046FEF76CF94142281A0891CDE90B
:107700000910084801900A4807906A460921304646
:1077100009F008FD012802D16846F9F7C3FF11B04E
:10772000F0BD00008D94010875940108DD910108F9
:10773000F91501082DE9F0471546824699460C4691
:1077400051EA050065D0504600F074FB5046FEF744
:1077500038F940420FFA80F808EB040004B2002127
:107760005046FEF79BFC012813D0002C13DC25DAD1
:107770005046FEF753F806465046FEF7AFF8304441
:1077800000B2002800DA00204042844216DA04B237
:1077900014E0002C02DA4FF000040FE00EDD50463A
:1077A000FEF73CF806465046FEF798F8304400B223
:1077B000002800DA0020844200DD04465046FEF72F
:1077C00007F9404206B2701905B2002D02DD4FF0F4
:1077D000000510E00FDA5046FEF7ECF80746504679
:1077E000FDF7A2FF384400B2002800DA0020404232
:1077F000854200DA05B2A4EB080001B2A81B02B270
:1078000051EA020005D04B465046BDE8F047FFF76D
:1078100005BFBDE8F08770B516461D4604461A46FA
:1078200000F024F82A4631462046BDE8704000F0BA
:1078300033B8F8B50F46054600F0FCFA002000907A
:107840002846FDF765FF044605F114060AE03B46AD
:107850006A462946304601F0C7FC25462846FDF712
:1078600057FF0446002CF2D1F8BD000070B50E465B
:10787000144605460749F9F743FE2846FEF7A1F8E6
:10788000801B01B223462846BDE870400022FFF766
:1078900051BF00007594010870B50E4614460546A8
:1078A0000749F9F72DFE2846FEF792F8801B02B231
:1078B00023462846BDE870400021FFF73BBF00008B
:1078C0008D9401081FB5044602AA6946FEF787F8A1
:1078D000684608F080FB20B902A808F07CFB00286D
:1078E00010D0684608F077FB18B169462046FFF7CC
:1078F000B4F802A808F06FFB002803D002A92046C4
:10790000FFF7ABF81FBD002200F04CB970B50C4674
:107910000546FDF72FF8A868848270BD38B50C467F
:10792000054600236A460421FDF7D3FE012807D04F
:10793000002804D100222146284600F07AF938BDFB
:107940000098A042F6D138BD2DE9F0410C4615460D
:107950001F4606461946F9F750F92A4621460DF00A
:1079600069F8224639463046BDE8F041FFF7E6BCEB
:1079700070B51546044600F0FDF929462046BDE8DD
:10798000704000F00DBA70B50C460546FCF7F2FFEA
:10799000A868417E01F00F01A14200D0447670BD7D
:1079A00070B50C460546FCF7E5FFA868017E64F358
:1079B0008301017670BD70B50C460546FCF7DAFF11
:1079C000A868017E64F30511017670BD70B50C46A0
:1079D0000546FCF7CFFFAB681A7E02F00300A04219
:1079E00007D064F301021A762846BDE87040FFF71D
:1079F00011B870BD70B51546044600F0A5F92946CA
:107A00002046BDE87040FFF789BF2DE9F34F89B0EC
:107A10008346008C0A9988427DD00390ABF82010F1
:107A200058460A9A0399F4F70DFE0290002872D086
:107A30004FF4207420460BF0E9FD8046214610F0FB
:107A400050FB002420466BE0DBF80C00042202EB24
:107A5000C90500EBC90A405920F07F4000F0B9F990
:107A60000190DBF80C00405920F07F4000F0AEF9A7
:107A700007900A990198884350D1DAF804008001F0
:107A80004CD405AA6721DAF8000000F0CFFA0128EB
:107A900044D10027059D39E000261BE006EB860156
:107AA00008EB810106914868049000F092F900907B
:107AB000049800F08BF9296831F817200699098994
:107AC0008A4206D10799884203D1DDE90001884244
:107AD00002D2761CA642E1D3A64216D104EB840062
:107AE000A98928F8201008EB8000298A4180A9681C
:107AF000C1602968641C31F817100181696801614F
:107B0000DAF8041021F07F4141607F1C286830F8CA
:107B1000170018B100E042E0202CBDD309F10100AC
:107B20008146BBF82200C0F30511494501D9202C3C
:107B30008AD300250EE005EB850108EB810670680D
:107B400000F044F90146009658460A9B039AF4F760
:107B5000D9FC6D1CA542EED340460BF0A3FD029864
:107B600001280CD0032810D0022818D15846FEF75F
:107B700051FF0BB05846BDE8F04FFFF79FBB0BB06D
:107B80005846BDE8F04FFEF745BF0BB05846BDE87C
:107B9000F04F4FF6FF724FF47021FFF7CFBB0BB0E1
:107BA000BDE8F08F13460A460921FFF7CDBE134604
:107BB0000A466621FFF7C8BE07B481B01346BDF878
:107BC0000810ADF80010009A522104B0FFF7BCBEB7
:107BD00013460A465321FFF7B7BE13460A46502103
:107BE000FFF7B2BE07B481B01346BDF80810ADF878
:107BF0000010009A202104B0FFF7A6BE13460A46E3
:107C00002121FFF7A1BE07B481B01346BDF80810CB
:107C1000ADF80010009A302104B0FFF795BE13466E
:107C20000A463121FFF790BE13460A463221FFF77C
:107C30008BBE13460A460421FFF786BE13460A464A
:107C40000A21FFF781BE13460A466021FFF77CBE7A
:107C500007B481B01346BDF80810ADF80010009AC3
:107C6000362104B0FFF770BE13460A463721FFF7EE
:107C70006BBE13460A463821FFF766BE13460A4616
:107C80003521FFF761BE13460A461121FFF75CBE9E
:107C900013460A461521FFF757BE13460A4612211E
:107CA000FFF752BE13460A461321FFF74DBE134697
:107CB0000A461421FFF748BE13460A461021FFF773
:107CC00043BE13460A460B21FFF73EBE13460A4643
:107CD0004321FFF739BE13460A464021FFF734BE61
:107CE00013460A465B21FFF72FBE07B481B0134647
:107CF000BDF80810ADF80010009A552104B0FFF748
:107D000023BE13460A465721FFF71EBE13460A46F6
:107D10005821FFF719BE13460A465921FFF714BE32
:107D200013460A465621FFF70FBE13460A460121A5
:107D3000FFF70ABE13460A460721FFF705BE1346A2
:107D40000A460821FFF700BE38B50C460546002359
:107D50006A460121FDF7BDFC012807D0002804D1A7
:107D6000002221462846FFF7E0FF38BD0098A042D8
:107D7000F6D138BD38B50C46054600236A460721C2
:107D8000FDF7A7FC012807D0002804D100222146D6
:107D90002846FFF7CFFF38BD0098A042F6D138BD86
:107DA00038B50C46054600236A460821FDF791FCCC
:107DB000012807D0002804D1002221462846FFF7D9
:107DC000BEFF38BD0098A042F6D138BD00F47F0058
:107DD000704780B270472DE9F0411E46154688462F
:107DE000070025D0F4F743FB022813D000249EB1EE
:107DF0003DB13846FDF78CFC33462A464146FFF735
:107E0000EAFF002C14D0324641463846BDE8F04126
:107E100001F0BEBE0124EAE724B1324641463846AD
:107E200001F0B6FE002D03D03846FDF771FCD7E710
:107E3000BDE8F08170B50B4D2978002910D10121E2
:107E40002970FDF769FC044605E021F00400608418
:107E50002046F9F783F9618C4807F6D40020287092
:107E600070BD00005437002010B51DF0A3FA0F4A72
:107E70004FF49653A2F51651A1F11C0008F067FFCC
:107E80000B4808F073FF0A48F02101804FF4A071FD
:107E90004180084941610849C160016941F004011C
:107EA0000161BDE8104008F08BBF0000BC700020ED
:107EB0003C96002021D80008204B002010B50A482D
:107EC0000AF0C8FC084802210170084941600AF024
:107ED000D5FC074C606009F061FC0146A060606859
:107EE000BDE810400AF042BE8C960020B50F010894
:107EF000283700202DE9FC410E46002507462A467A
:107F0000143102F0AEF8002826D001213046FEF7E9
:107F1000EFFA00BB3046F4F7AAFAE0B900208DF87A
:107F200000006A4612213046019709F0FBF89DF8DF
:107F3000000002280FD03046FDF7FCFA401E040076
:107F40000ED4B068006850F824103846FFF7D2FF0E
:107F5000050009D102E00020BDE8FC81641EF0D5D7
:107F60009DF8000000B935462846F5E72DE9FC41AB
:107F70000025DFF8B4804FE0284490F83001E8BBDA
:107F8000002441E0011991F83011C1BBA5423AD05B
:107F900000EBC40100EBC5003030303102F0B5F821
:107FA00068B37068B04600EBC40200EBC5016846D8
:107FB0003031303202F0A9F9684608F00CF8064674
:107FC000D8F8040000EBC500303008F004F807468C
:107FD000D8F8040000EBC400303007F0FCFF384450
:107FE000864210D2D8F80400464600EBC500694628
:107FF0003030F9F7A7FB0120716801E00BE002E0E7
:10800000214481F83001641CD8F804004646B0F8D9
:108010005011A142B6D86D1CD8F80400B0F8502118
:10802000AA42A9D8BDE8FC816037002070B515468A
:108030008288C479A2F57F43FF3B07D08CB3012C23
:1080400034D90668002306EB84022CE0002313E0F9
:10805000026802EBC302168826F440468E420AD11B
:108060001088010428D4400401D5304613E050683C
:108070002860012070BD5B1C9C42E9D824E032F8E6
:10808000130020F4404088420CD132F813100A0447
:1080900012D4490402D50CF025FBE9E706EB830076
:1080A00010E011E05B1C9C42E9D80DE022F4404353
:1080B0008B4209D1110401D5022070BD510401D5B4
:1080C0001846E8E70068D3E7002070BD10B50C46FD
:1080D00002F038FD204000D0012010BD2DE9F04114
:1080E000074615460E460B4802F07BFC040010D0F4
:1080F000A7604FF0FF3026602061002060610DF026
:10810000A5F8E56004496060012008712046BDE8DB
:10811000F081FEE7009800203038002010B50446BA
:108120000146054802F0D3FC044B01222046DA70D8
:10813000BDE810400BF0C8BA00980020303800208D
:108140002DE9F047494CA07810B10120BDE8F08737
:108150000120A0702078002528B10DF077F85FEAA3
:10816000000A02D007E0A570EFE72069401C2061FB
:10817000642800D925613E4FA946A0463D4888F8AD
:10818000039088F8049002F007FC386033E0394827
:1081900002F014FC3C680646207DC0072AD1002569
:1081A000204600F07EF868B92569002D01DD681EC3
:1081B00020610DF04BF86060A16811B10DB120464F
:1081C0008847012598F8030020B9206910B9204696
:1081D000FFF7A4FF75B198F8041098F80300014365
:1081E00008D038680028C9D14FF0FF35214802F087
:1081F000D3FB11E03E6039680029C8D1F4E7207D47
:10820000C00705D1204600F04CF8A84200D2054630
:108210002146184802F0D2FB0400F0D150460DF080
:108220000EF8D8F80C1044460844C8F80C00D8F8EA
:1082300008000DF004F8B0F5FA7F13D3E16864226A
:108240005143B1FBF0F0C0B26070642801D9002046
:1082500001E0C0F1640060702646C4F80C900CF098
:10826000F5FFB06084F8029028466FE730380020B0
:10827000043800200098002001214161704710B5AA
:1082800004460CF0E3FF2168401A401E606010BDF8
:1082900010B504460CF0DAFF606010BD00214161AA
:1082A000704710B5044640680CF0C9FF2168814250
:1082B00001D8002010BD081A10BD00002DE9FF4FA5
:1082C00085B00546DDE913981E460F460846169C04
:1082D000F9F795FA03903846F9F76DFA0290012CF8
:1082E00013D0022C13D0032C4CD14E4F2888ADF85C
:1082F00000003088B8F1000FADF8040009D098F8FC
:108300000000FD2841D3484642E0474FEEE7474F83
:10831000ECE7DDE900104A46B847049000202DE064
:10832000002420E0BDF8040036F81410884205D17E
:10833000BDF8000035F8141088420ED005EB44005B
:108340004A460088ADF8000006EB44000088ADF80E
:108350000400DDE90010B847049005EB4400BDF8C7
:1083600010100180641C03988442DBDB079805EB46
:108370004005129806EB400608F10100029980467C
:108380008842CDDB09B0BDE8F08F00FB09F0000AA0
:1083900082460246DDE90010B847049000203CE028
:1083A00000242DE018F8040048B3FD2801D3484606
:1083B00002E000FB09F0000ABDF8041036F81420B2
:1083C000914207D1BDF8001035F81420914201D137
:1083D00082450FD005EB440182460988ADF80010B4
:1083E00006EB440102460988ADF80410DDE90010EF
:1083F000B847049005EB4400BDF810100180641CE0
:1084000003988442CEDB0798159905EB4005129836
:10841000884406EB40060BF101000299834688422E
:10842000BEDBAFE77BD30008F9D20008FFD300081A
:108430002DE9FF4F85B00646DDE913791D460C4650
:108440000846F9F7DCF980462046F9F7B4F9834687
:10845000B9F1000F06D0FD2F7ED9A8F104000490D9
:1084600000201DE1FD2F14D300244FEA48070BE044
:10847000304629463A460FF00CFE0798641C06EB7E
:108480004006129805EB40055C45F1DB09B0BDE8FC
:10849000F08F002021E0002415E006EB440A3A4664
:1084A000BAF80000ADF8000005EB44000088ADF814
:1084B0000400DDE90010F9F783FA0090BDF8001020
:1084C000AAF80010641C4445E7DB079806EB400659
:1084D000129805EB400509F1010081465845DADBA9
:1084E000D4E74F46002419E03A78AAB1FF2A06EBF8
:1084F000440018D082460088ADF8000005EB440027
:108500000088ADF80400DDE90010F9F759FA009091
:10851000BDF80010AAF80010641C7F1C444575DAF1
:10852000B807E1D172E005EB440109880180F3E767
:108530003868E8B3401C6DD03A78BAB1FF2A06EB30
:10854000440075D082460088ADF8000005EB440079
:108550000088ADF8040000E0ACE0DDE90010F9F7B8
:108560002FFA0090BDF80010AAF800107A7807F1F1
:10857000010AAAB1FF2A06EB44005ED000904088B1
:10858000ADF8040005EB44004088ADF80800DDE9D3
:108590000110F9F715FA0190BDF804100098418018
:1085A0001AF8012FBAB1FF2A06EB440049D000E0C7
:1085B0002AE000908088ADF8040005EB4400808834
:1085C000ADF80800DDE90110F9F7FAF90190BDF8FE
:1085D0000410009881809AF80120AAB1FF2A06EBC6
:1085E000440032D08246C088ADF8000005EB44005C
:1085F000C088ADF80400DDE90010F9F7E1F900905A
:10860000BDF80010AAF80610241D3F1D04988442EE
:108610008EDB39E005EB440006EB440102880A805A
:1086200042884A8082888A80C088C880ECE7FFE759
:1086300005EB44010988018098E705EB440149886E
:10864000ADE705EB44018988C4E705EB4401C9881F
:10865000C180D9E73A78AAB1FF2A06EB440024D0BA
:1086600082460088ADF8000005EB44000088ADF8B4
:108670000400DDE90010F9F7A3F90090BDF800103F
:10868000AAF80010641C7F1C4445E3DB0798159989
:1086900006EB40061298894405EB40050398401C00
:1086A00003905845FFF61DAFF0E605EB440109883D
:1086B0000180E7E700202BE000241DE019F804000A
:1086C000C8B1FD2801D33A4601E07843020A06EB1F
:1086D000440000900088ADF8040005EB44000088D9
:1086E000ADF80800DDE90110F9F76AF9019000988A
:1086F000BDF804100180641C4445DFDB0798159920
:1087000006EB40061298894405EB40050AF101008A
:1087100082465845D0DBB9E62DE9FF4F85B01D46AE
:10872000DDE913B80E46F4F783F882463046F9F7D0
:1087300066F881463046F9F73EF80390B8F1000F2D
:108740004FF000071ED048E0002415E005EB440080
:10875000CDF808B00088ADF804007088079A384456
:1087600000B2009030880599204403B2DAF8000086
:10877000D0F81CC0E047641C4C45E7DB12987F1C16
:1087800005EB400503988742DEDB09B0BDE8F08FBA
:1087900000241AE018F80400B0B100FB0BF0000A46
:1087A000029005EB4400079A0088ADF80400708839
:1087B000384400B2009030880599204403B2DAF8BA
:1087C0000000D0F81CC0E047641C4C45E2DB159962
:1087D0001298884405EB40057F1C03988742D7DB3D
:1087E000D3E7FD2902D2022901D80020704710FBEF
:1087F00001F000EBC01101EBC030C0F3C75070476F
:1088000070B5094D04466868002808D044B1204678
:10881000F8F7EAF9A9682044884200D3002070BD27
:108820000248006870BD0000683700201038002042
:108830002DE9F04104460022212108F073FC0028B4
:108840007ED0608C40F48050608401E0FFF7F0FF40
:1088500000212046FCF75CFE0028F7D12046FCF7FB
:1088600017FF064600200AF033F8054600271CE0F3
:10887000A86AA04202D0E86AA04203D12146284655
:108880000AF0CEF8686BA04200D16F63686DB04209
:1088900007D10AF027F8A04203D1214628460AF062
:1088A000BFF828460AF014F80546002DE0D120460E
:1088B000F3F7C9FD606804260028204602D0FCF7C3
:1088C000EFFE29E0FCF7C6FE0546416A0022C068BB
:1088D00004E050F82230A3420AD0521C9142F8D84A
:1088E00006E0E86806EB8201415840F82210521C6D
:1088F000686A401E9042F4D8686A401E810068622F
:10890000E8680AF005FFE8601EE0096806EB8002EF
:108910008A5841F82020401C616889684A68521EC4
:108920008242F2D8606880684068401E4860616892
:10893000800089680A68014610460AF0E9FE00E0F6
:1089400007E06168896808602046BDE8F0410AF0E8
:10895000BBBEBDE8F08100002DE9F04F524F064646
:1089600085B078680168CC6BC96889682160016846
:1089700009698A0701D4C90723D008F037FB401ED4
:1089800005B2786808F0ECFA401E03B200221146E6
:1089900003A8009507F065FB03A96160786800688B
:1089A000027CC068920705D5826942F002028261AA
:1089B000A16073E08169826961F341028261A6600E
:1089C0006CE03046F8F70FFF81463046F8F7EDFED1
:1089D0008046786808F00AFB0146B6F90600814235
:1089E00003DC786808F002FB401E05B242464946A7
:1089F000BA467868F8F768F981460027B6F90200A8
:108A00000DF1040B28E03288ADF80420B288ADF8EF
:108A10000820ADF80600ADF80A10C4F804B0C4F898
:108A200008B0DAF804000168C96889682160BDF9F6
:108A30000A10A94201DDADF80A50BDF90A70BD4225
:108A400005D10068C068816941F00201816120465A
:108A500000F02CF80FFA88F000EB0908A8F10101EA
:108A6000A942D0DDBD421CD03188ADF80410B188D8
:108A7000ADF80810ADF80600ADF80A50C4F804B01F
:108A8000C4F808B0DAF804000168C9688968216090
:108A90000068C068816941F002018161204600F0F0
:108AA00005F805B0BDE8F08F603700202DE9F041F2
:108AB0005F4F064690B0786808F04EFAF1680446B9
:108AC00009B130468847786800680188408811FB02
:108AD00000F0E168884201D1012000E00020216817
:108AE00059B1616831B128B907E078680068816AD6
:108AF00001B1884720690028F7D10024786808F080
:108B00005FFA01467068FFF7F5F905467868416934
:108B100019B17068FFF7EEF9044655EA040051D127
:108B2000786808F063FA401E0FFA80F8786808F059
:108B300017FA401E03B2002211460EA8CDF800809D
:108B400007F08FFA306BB0B16846FAF77DFA7868B3
:108B50000EAAC16A049190F829108DF81A10418D5F
:108B6000ADF8041090F829008DF80300336B6946C6
:108B70003046984726E07868C06A98B106A909F09F
:108B8000F5FB01281ED16846F9F7D4F978680EAADA
:108B900090F829108DF80B10C36A69463046F9F732
:108BA00095F90FE06846FAF74FFA7868418DADF80D
:108BB000041090F829008DF8030069463046726869
:108BC000FAF72EFA786890F82810C9070CD005B982
:108BD00005693046294600F09FF97868406990B1F0
:108BE00004B9044621460BE0406928B104B90446A3
:108BF0002146304600F090F90DB97868056929469C
:108C0000304600F089F9786808F0C8F90146304626
:108C100000F082F9786808F0B9F90146304600F0B2
:108C20007BF9786810B0BDE8F041F5F72BBC000087
:108C3000603700202DE9F0412B4F00203860786824
:108C4000B0F85051002D4DD0002603E0411991F8A5
:108C50003011D1B16D1EF9D50068416B01B1884763
:108C600078680168C9688A6922F001028A6101682E
:108C7000C9688A6922F002028A6190F828100024EB
:108C800041F0040180F8281022E02E46E4E70119A3
:108C900091F83011D9B9B44205D10168C9688A691F
:108CA00042F001028A610168C9688A6922F0020201
:108CB0008A6100EBC4003030FFF74EFE786800EBAD
:108CC000C400303007F087F9396808443860641C04
:108CD0007868B0F85011A142D9DC10F8281F21F0B3
:108CE00004010170BDE8F081603700202DE9F04FEC
:108CF0000D4680468BB001212846FDF7F9FB002880
:108D00007ED12846F3F7B3FB040028D02846002183
:108D10006122FDF782FA00F0FF0BBBF1020F6FD367
:108D200006AB224629464046F8F7CFF9012867D11D
:108D300005F114010127002206A80A9101F091F91A
:108D4000A8B100208DF8200006A8099008AA1221D9
:108D5000284608F0E7F99DF8200038B107E00BB08D
:108D600029464046BDE8F04FFDF7FDBF0027012C26
:108D700001D147F002073A4606A94046F9F7B8FB89
:108D800004003DD0284600216F22FDF746FA00B2CC
:108D900060F30F068146284600217022FDF73DFA58
:108DA00000B260F31F468246C9F34130012818D152
:108DB00029F4C049B9F5FA6F13DC0A98F8F713FDE6
:108DC000014630B220F4C040B0F57A7F02DDC9F52B
:108DD0007A7000E048464143642091FBF0F060F374
:108DE0000F06CAF3413001281AD12AF4C049B9F557
:108DF000FA6F15DC0A98F8F7D8FC0146301400E049
:108E000084E020F4C040B0F57A7F02DDC9F57A70C5
:108E100000E048464143642091FBF0F060F31F46B8
:108E20006846F9F787F88DF80BB0284600216E22C6
:108E3000FDF7F3F900B2ADF80000B0F5616F02DDA7
:108E4000A0F5616003E0002803DA00F56160ADF889
:108E50000000284600216D22FDF7DFF9ADF8020081
:108E6000284600216822FDF7D8F98DF80C00294822
:108E700040680068007CC0F3C0008DF81400B8079B
:108E80003AD5D4E90001C4E902016089618A084445
:108E9000401E00B2E081B4F9061088422CDDE18169
:108EA0002AE0B80705D53B46224641462846F8F752
:108EB000D9F829464046FDF756FFA88A6A46811927
:108EC000D8F804000088081AADF80400E88A00EB1E
:108ED0002641D8F804004088081AADF8060021465B
:108EE0004046F9F700FBB8070CD5E089401C6081CB
:108EF000618A0844401EE081B4F90A00BDF91E10E1
:108F00008842CEDD21464046F9F723FB0BB0BDE891
:108F1000F08F0000603700202DE9F0470F008146F8
:108F200005D11B48406808F04BF807002AD03946A5
:108F30004846FFF7DBFE20E00026FCF7FBFA804600
:108F4000002408E0A868006850F82410E6B14846FC
:108F5000FFF7CCFE641C4445F4D34A46172128464B
:108F600008F0E0F84A461821284608F0DBF84A469F
:108F70001921284608F0D6F82F463846FCF7C8FBDA
:108F80000500D9D1BDE8F087B942E3D10126E1E778
:108F9000603700202DE9F04F464C8DB060680168C5
:108FA0000A7CD2077ED0C968496800297FD000F5C5
:108FB000AC7001F083FD002879D160680168C96850
:108FC0008B680C930A68934200D14A68924607F076
:108FD000C7FF0B90202103A80FF083F80025A046BF
:108FE0003CE0411991F83011B9BB00F5AC7001F0CB
:108FF000D3FC0746A0462EE0D8F804003946444684
:1090000000F5AC7001F0DAFC83466068394600EB8D
:10901000C50203A8303200F063FF0646401C19D099
:1090200000240DF10C0909E001F0F9FC09EBC40181
:10903000641C0A6802604968416064B2D8F80400A0
:10904000B442394600F5AC70EEDB01F040FD384625
:109050000AF03AFB5F46002FCED16D1CD8F8040011
:109060004446B0F85011A942BBD8264600F5AC7072
:1090700001F092FC12E00B98CDF800A0CDE90104BC
:109080007068DDE90B2100682346C06B856BA8473B
:109090007068214600F5AC7001F090FC0400EAD144
:1090A000706800E003E000F5AC7001F05FFC0DB00B
:1090B000BDE8F08F603700202DE9F0410746FCF74E
:1090C00039FA0646002412E0B868006850F82450C7
:1090D0002846FDF79FFC00222A21284608F022F8A6
:1090E0002846FDF797FC2846FFF7E6FF641CB442CC
:1090F000EAD3BDE8F0812DE9F0410646488C0D46E3
:109100000022C0F305100EE026B1E96851F83210D4
:10911000B14207D14FF6FF724FF470212846FEF797
:109120000DF902E0521C9042EED82846FCF702FAF4
:109130000746002407E0A868006850F8241030466D
:10914000FFF7D9FF641CBC42F5D3BDE8F0812DE9DF
:10915000FF5F8346DDE90E87DDE91354129EF3F7C6
:1091600067FB00683146FF22D0F8389020460EF0A9
:10917000B1FF002082462DE01099414308EB2122E7
:109180001199414307EB212112124FEA212107D403
:10919000019B9A4204DA002902DB029B994202DB1E
:1091A00004F800A009E0DDF80CC001FB0C210BEB7A
:1091B000410105EB4002098811801599062907D164
:1091C00035F810201FFA89F18A4201D104F800A075
:1091D000401C00B2B042CFDBBDE8FF9F0022006818
:1091E0000A2107F09FBF00002DE9FF4F85B0904690
:1091F0000C460846FCF78CFA06461021FDF778F974
:1092000000286FD03046FCF7E1FA8346002530464F
:10921000FCF7C9FB1434CDE9024000B9059C0021DC
:109220003046FCF768FF824600213046FCF7EFFF2E
:10923000504407B200213046FCF7C5FF504401B24C
:109240000191F08A61883844411AB8F80200728BA3
:10925000091A0FFA81F90199511AE288891A401AFC
:1092600000B200903046FCF718FA0199C01B401A72
:1092700000B20490B9F100010DDB0098002815DA66
:109280000846B9F1000F06DD05463046FCF792FBB3
:10929000401B0AD40AE00098002807DD404205B2CE
:1092A0003046FCF741FAE84200D500250398012832
:1092B00004D0022806D003280CD114E0F08A61887B
:1092C000384403E0718B0198081AE1882944401A58
:1092D000284405B200243046FCF75EFB0090A8B19C
:1092E000029F14E0BEE00498F18A00EBD07007EB17
:1092F00060000A18E0886188401A401C00B200EB48
:10930000D07005EB60000844101AE1E7059F0021CA
:109310003046FCF764FF50440FFA80F900213046D4
:10932000FCF769FF5044B18A0FFA80FA01EB09009B
:109330003988338B421AB8F80010501AA3EB0A028E
:10934000BB8800B2D21A891A09B200280ADB0029A8
:1093500012DA002806DD04463046FCF75FFA001BEF
:1093600009D409E0002907DD484204B23046FCF781
:10937000B5FAE04200D500243046FDF79AF8A0EB9C
:109380000901A1EB0A0001B20098012804D00228CB
:1093900007D003280DD122E0B18A01EB09003988FA
:1093A00003E0318BA1EB0A00B9882144401A204424
:1093B00004B22E493046F8F7A3F807462C49304648
:1093C000F8F79EF8074306D000220A21304607F03E
:1093D000A9FE012846D15FEACB7012D014E001EB60
:1093E000D171B28A09EB61000244B8883988401A09
:1093F000401C00B200EBD07004EB60000844101A6F
:10940000D5E7002C00DA00245FEA8B7002D4002C30
:1094100000DD00245FEA4B7002D4002D00DA002545
:109420005FEA0B7002D4002D00DD00250898B8F922
:109430000010002800D020460844A8F80000B8F921
:10944000021002D14FF0000000E028460844A8F8BE
:109450000200089B09B02A4621463046BDE8F04F7D
:10946000FEF7DCB809B0BDE8F08F00008D9401086C
:109470007594010810B50346FCF7A3FA084401B23D
:10948000BDE8104000221846F2F7F7BF10B50346BA
:10949000FCF79EFA084402B2BDE8104000211846CD
:1094A000F2F7EBBFF8B505460C460846F9F7CCFDD8
:1094B0004FF4803631462846FCF703FEE070022860
:1094C00008D9284631462022FCF7A7FE0090BDF8B7
:1094D0000000A080284631463122FCF79EFEC0B233
:1094E000002784F82200022814D928463146322267
:1094F000FCF793FE00B22084002809DD284631469F
:109500003022FCF78AFE0090BDF80000E08301E005
:1095100084F82270284631464522FCF77EFEC0B210
:1095200084F8360002281AD9284631464022FCF732
:1095300074FE00B2E08500280FDD28464322314644
:10954000FCF76BFEA086284644223146FCF765FEF8
:109550000090BDF80000A08501E084F83670314627
:109560002846FCF7EEFDFD280AD2E17811FB00F158
:10957000090AE1704143080A84F8220084F83600A1
:10958000E07830B994F8220018B994F83600002831
:1095900005D031462846FCF787FE20800120F8BD23
:1095A0002DE9F84F044615460E464FEA61084FEA8A
:1095B000610AC80701D1A8F10108600000900AF013
:1095C00025F807462B46002025E003EB440B3BF82B
:1095D000021C7143601E16D4002200EB0A0C27F80F
:1095E0001010A44501DA33F81C208A1AA0EB0801F8
:1095F000012901D5198803E003EB410131F8021C70
:10960000401E1144E8D539461846009AFBF7FEF88B
:109610005B4609F101008146A042D6DB4FF47F5240
:10962000B2FBF6F100201FFA81FC14FB04F30CE0FE
:1096300035F8101041B1914202D125F810C003E075
:1096400091FBF6F125F81010401C8342F0D8002160
:1096500039E005EB410399461A887243002024E063
:10966000002A02DA4FF0000C01E04FEAA21C27F8B2
:1096700010C0A0EB0A0CBCF1000F02DCB3F800C074
:1096800003E00CFB041C35F81CC0A2EB0C0C00EB37
:109690000802521CA24200DB621E02FB041203EB12
:1096A000440335F81220401C6244A042D8DB4A46ED
:1096B000002005E037F81030138002EB4402401C14
:1096C000A042F7DB491CA142C3DB3846BDE8F84F96
:1096D00009F0E8BF2DE9F0470E468AB01D468046E6
:1096E000014617469246541907A8F8F74FF807EBBA
:1096F000D77005EB600147F30002891A891EADF8A7
:109700002010012101EB6000ADF81E004046F8F783
:1097100088F8BDF82010081AADF81C004046F8F78C
:1097200056F8BDF81E1000230844ADF822002A4662
:1097300007A901A8F9F7BAFB5746BAF1010F01D002
:109740004FEA6A07204609F061FF8046354600204F
:1097500034E021464046FBF769F801A80090DDF8A7
:1097600004C023B20FFA89F200214046E04738B125
:1097700098F80000800190FBF7F02880012017E0A6
:1097800061002846FBF74DF814E008EB000218F8DA
:10979000001012F8012C914204D105EB400131F880
:1097A000021C02E0890191FBF7F125F81010401C22
:1097B000A042EADB05EB440509F101008146A04225
:1097C000C7DB404609F06EFF01A8F9F7E9F8012F61
:1097D00014D020B2324639460546FFF7E1FE0AF0C2
:1097E0000100384401B2012927DD4FF47F5090FB7E
:1097F000F1F2002097B204FB04F318E00020314698
:10980000644304E036F8102092090A54401C844254
:10981000F8DC0AB0BDE8F08736F8102032B1FF2A34
:109820000FD0920192FBF1F226F81020401C8342E7
:10983000F2D832462846FFF7B3FE00203146644393
:1098400006E026F81070F1E716F810200A54401CC4
:109850008442F9DCDDE7F0B597B0074615460E46C1
:1098600001A8F9F7F1FBFF2211461046F8F75DF861
:109870000090BDF800000090BDF80000ADF80800B1
:109880000024324601A93846F9F7CAFB0FA8F8F7B9
:10989000FFFD2B4632460FA938460094F8F764FBCB
:1098A00017B0F0BDFEB5066804460A46708C002568
:1098B0000421C0F305130BE0F06801EBC507C059A4
:1098C000870104D5A76820F07F40B84203D06D1C03
:1098D000AB42F1D8FEBDA18844295CD00EDC33290F
:1098E0004CD006DC202956D0222954D0302913D15F
:1098F00051E0342942D036290ED14CE0622940D0C3
:1099000006DC472947D0552945D0572904D135E0F1
:10991000672933D0682931D062B3FF2A2CD0D4E92B
:1099200003031B1A534300EB23200090F068012728
:1099300001AA50F835000AF079FE60B1DDE90001B6
:10994000884208D1BDF80020BDF804309A4202D107
:10995000884200D10027F068A188009A50F83500AD
:109960000BF068F8002FB5D0A288A1682068FDF739
:10997000E5FCFEBDE068D8E72069D6E7FF2AFBDA00
:10998000F8E7E0680028F7D02369002BCDD0802AC3
:10999000CBDB0093CAE7002A01DCA0892AE0FF2A7A
:1099A00001DB208A26E0208AD3B280B2020242EA9A
:1099B0001020A78982B2B8B2070247EA10201B1D07
:1099C000DF080E4B80B240EA004042EA02421840F3
:1099D0001A40121A7A4300EB5210184040EA104025
:1099E00080B2020242EA1020ADF8080080B2029074
:1099F000BDF80800ADF8000098E700001FF8E00788
:109A00002DE9F041046800262648A788256800F063
:109A1000C3FF10E0A1420BD008682268904207D132
:109A20008868A268904203D18888A288904237D083
:109A30001C4800F0C3FF0100ECD1002E30D1688C2F
:109A40000421C0F3051229E0E86801EBC603C05801
:109A5000830122D5A36820F07F4098421DD1214682
:109A6000104801F034F8204609F02EFEE868394627
:109A700000EBC60420680AF0CFFEE86850F8360014
:109A80000AF029FE00280BD06068216820F07F4290
:109A90002846BDE8F041FDF727BD761CB242D3D879
:109AA000BDE8F0815498002070B50468A068A288D1
:109AB00000F47F0631462068FCF7AFFBE060A58824
:109AC0000020A08023462A463146206800F00CF88A
:109AD000A580A1682068F7F7DCF9A1880068E26832
:109AE000BDE870400AF0A6BF2DE9FF5F074691462A
:109AF0000E460024254800F068FF05464FF4702B01
:109B00004FF0040A3CE0039885423BD029461F48A9
:109B100000F058FF80462868B84230D1A868B042AB
:109B200001D05E452BD1A988494503D0A9F57F41D5
:109B3000FF3924D1002411E0F8680AEBC401415830
:109B40008A010AD55E4503D021F07F41B14204D19C
:109B500050F83400A9880AF05FFE641C788CC0F3CA
:109B60000510A042E8D800212846F7F7C9FC29468D
:109B7000064800F0ACFF284609F0A6FD0124454642
:109B8000002DC0D104B02046BDE8F09F54980020BD
:109B90002DE9F74F934682B0044600216E22FCF770
:109BA0003CFB06B2204600216D22FCF736FB05B2D5
:109BB00016B9B5F5807F67D0204600216F22FCF7EB
:109BC0002CFBADF80000204600217022FCF725FB9D
:109BD000ADF80200BDF9000004F11401C0F34132F8
:109BE00064274FF4FA688A464FF47A79012A14D12F
:109BF00020F4C040404510DC0846F7F7EEFD014672
:109C0000BDF9000020F4C040484501DDC0F57A7080
:109C1000414391FBF7F0ADF80000BDF90200C0F33D
:109C20004131012914D120F4C040404510DC504698
:109C3000F7F7B5FD0146BDF9020020F4C0404845E4
:109C400001DDC0F57A70414391FBF7F0ADF80200F9
:109C5000A08ABDF80010BBF1000F0844ADF8000069
:109C6000E08ABDF802100844ADF8020006D0704248
:109C700006B24FF4803090FBF5F005B26B462A46F1
:109C80003146039809F076FF05B0BDE8F08FF0B5D6
:109C9000D0E90646059D4FF480772EB9BC4203D12A
:109CA00008021860100239E0B0F928C0A1EB0C01DD
:109CB000B0F92AC0A2EB0C029EB1BC421AD1446991
:109CC00006694C4306FB1244066A06EBA4041C60BA
:109CD00003694B434169406A01FB023100EBA1007B
:109CE0001CE0066A01FB04611960416A806902FB9D
:109CF000001013E0466907694E4307FB126666438E
:109D0000046A04EBA6241C6003694B43416901FB10
:109D100002318269406A514300EBA1202860F0BD06
:109D200000000000B34D0108994E0108000000003A
:109D3000D5510108730073004A020000000001E0E1
:109D400001E0000000FF0055AAFF00112233445536
:109D500066778899AABBCCDDEEFF000102030405FB
:109D6000060708090A0B0C0D0E0F1011121314151B
:109D7000161718191A1B1C1D1E1F2021222324250B
:109D8000262728292A2B2C2D2E2F303132333435FB
:109D9000363738393A3B3C3D3E3F404142434445EB
:109DA000464748494A4B4C4D4E4F505152535455DB
:109DB000565758595A5B5C5D5E5F606162636465CB
:109DC000666768696A6B6C6D6E6F707172737475BB
:109DD000767778797A7B7C7D7E7F808182838485AB
:109DE000868788898A8B8C8D8E8F9091929394959B
:109DF000969798999A9B9C9D9E9FA0A1A2A3A4A58B
:109E0000A6A7A8A9AAABACADAEAFB0B1B2B3B4B57A
:109E1000B6B7B8B9BABBBCBDBEBFC0C1C2C3C4C56A
:109E2000C6C7C8C9CACBCCCDCECFD0D1D2D3D4D55A
:109E3000D6D7D8D9DADBDCDDDEDFE0E1E2E3E4E54A
:109E4000E6E7E8E9EAEBECEDEEEFF0F1F2F3F4F53A
:109E5000F6F7F8F9FAFBFCFDFEFF80808081818235
:109E6000828384858687898A8C8D8F919395979933
:109E70009B9EA0A2A5A7AAADAFB2B500FF1FFF1F72
:109E800001E001E090880608000000209C380000F6
:109E900034900208549106089C380020A4F5000074
:109EA00024C2000870B5044600256FF02F0608E0B4
:109EB0002068411C2160007805EB850106EB41011B
:109EC00045182068007800F004F80028F0D12846F2
:109ED00070BD3038092801D8012070470020704734
:109EE0002DE9F0470F46814690461146384600F06E
:109EF0000CF940B100224146384600F0B2F828B1D2
:109F00000020BDE8F0874FF0FF30FAE70026384622
:109F100006F07BF8401E0FFA80FA384606F04FF83C
:109F2000401E02B2B8F80210B7F90200091A09B2CD
:109F300000290FDD3B88012663F30F0460F31F4403
:109F4000BB88084463F30F0560F31F45C9F8004060
:109F5000C9F80450B8F906007988411A511A09B2B3
:109F6000002913DDB7F9062090420FDA3A8862F330
:109F70000F04BA8860F31F4462F30F05084460F3CE
:109F80001F4509EBC600761C04604560B8F9020065
:109F9000B7F90210884200DC0846B8F90610B7F994
:109FA0000620914200DB1146B8F80030B7F90020D6
:109FB000091A9B1A1BB209B2002B10DD00290EDD15
:109FC00062F30F041A4462F30F05421862F31F454F
:109FD00009EBC60260F31F4414605560761CB8F9A3
:109FE00004203B88D71AAAEB07031BB2002B0EDD17
:109FF00062F30F0460F31F441A4462F30F05084430
:10A0000060F31F4509EBC600761C046045603046CE
:10A0100077E770B5B1F90040B2F900309C4200DD3D
:10A0200023460380B1F90240B2F90250AC4200DC91
:10A030002C464480B1F90450B2F90460B54200DB0B
:10A0400035468580B1F90610B2F90620914200DB51
:10A050001146C1800120AB4201DC8C4200DD0020B2
:10A0600070BDF8B50D460446B0F90000B1F9001016
:10A070001646884247DBB4F90210B5F90220914236
:10A0800041DBB4F90410B5F9042091423BDCB4F98A
:10A090000610B5F90620914235DC96B3ADF8000004
:10A0A0006088ADF8020032466946284600F099F80B
:10A0B000002827D0A088ADF800006088ADF8020025
:10A0C00032466946284600F08CF800281AD02088CD
:10A0D000ADF80000E088ADF8020032466946284637
:10A0E00000F07FF800280DD0A088ADF80000E088CF
:10A0F000ADF8020032466946284600F072F80028A2
:10A1000000D00120F8BD0020F8BDB0F90020B1F961
:10A1100004309A4213DCB0F90420B1F900309A42BD
:10A120000DDBB0F90220B1F906309A4207DCB0F934
:10A130000600B1F90210884201DB012070470020BF
:10A140007047F8B50D460446B0F90400B1F90010A7
:10A150001646884243DBB4F90600B5F9021088427E
:10A160003DDBB4F90000B5F90410884237DCB4F9DE
:10A170000210B5F90620914231DC76B3ADF800004B
:10A180006088ADF8020032466946284600F029F89A
:10A1900018BBA088ADF800006088ADF80200324618
:10A1A0006946284600F01DF8B8B92088ADF80000CF
:10A1B000E088ADF8020032466946284600F011F802
:10A1C00058B9A088ADF80000E088ADF8020032462A
:10A1D0006946284600F005F808B10020F8BD0120C6
:10A1E000F8BD2DE9FC4105460F46B1F90000B5F96F
:10A1F0000010144688423BDBB5F90410884237DC76
:10A20000B7F90200B5F90210884231DBB5F9061042
:10A2100088422DDC002C76DD284605F0F6FE00EBAA
:10A22000D0704610284605F0CAFE00EBD0704010F2
:10A23000864200DA3046844200DD04462888ADF8C4
:10A240000000288800222044ADF804006888ADF89A
:10A250000200688839462044ADF806006846FFF7DA
:10A26000C0FF40B1BDF804002044ADF804003FE059
:10A270000020BDE8FC81E8880022001BADF8020048
:10A28000E888ADF8060039466846FFF7AAFF28B10E
:10A29000BDF804002044ADF8040011E0A8880022B5
:10A2A000001BADF80000A888ADF8040039466846E8
:10A2B000FFF797FF50B1BDF80000001BADF800009C
:10A2C000BDF80200001BADF8020016E06888ADF88A
:10A2D0000200688800222044ADF80600394668462E
:10A2E000FFF77FFF70B1BDF80000001BADF8000064
:10A2F000BDF806002044ADF806003946684609F06E
:10A30000D7FCB6E7FFE70120B3E710B5B1F900309D
:10A31000B2F90040A34200DB23460380B1F90230CA
:10A32000B2F90240A34200DB23464380B1F9043076
:10A33000B2F90440A34200DC23468380B1F9061041
:10A34000B2F90620914200DC1146C18010BD000028
:10A35000084949680AE04A68824202D00A68824293
:10A3600003D10A7E42F001020A7649690029F2D13E
:10A370007047000034370020704700000421014876
:10A3800000F027BB249800202021014800F021BBC9
:10A390003C9800202DE9FF410446DDE90A571E00E4
:10A3A0004FF0000002D1B5F5807F2BD003900190D3
:10A3B0000290ADF80C100090ADF80410ADF80A2032
:10A3C000ADF80E203B462A463146684609F0D2FBDE
:10A3D0003B462A46314601A809F0CCFB3B462A46BB
:10A3E000314602A809F0C6FB3B462A46314603A87F
:10A3F00009F0C0FBBDF90030BDF90420934209DA31
:10A400001D4608E02080491E6080A180521EE28027
:10A41000BDE8FF811546BDF90800BDF90C10884262
:10A4200001DA064600E00E46B54205DA934201DA4B
:10A43000184604E0104602E0884200DB0846801E11
:10A440002080BDF90030BDF90400834201DD1D46C6
:10A4500000E00546BDF90820BDF90C108A4201DD77
:10A46000164600E00E46B54203DD834206DD18467F
:10A4700004E08A4201DD104600E00846801CA0800E
:10A48000BDF90230BDF90620934201DA1D4600E015
:10A490001546BDF90A10BDF90E00814201DA0E46DB
:10A4A00000E00646B54205DA934201DA184604E0B8
:10A4B000104602E0814200DA0846801E6080BDF945
:10A4C0000230BDF90620934201DD1D4600E015462D
:10A4D000BDF90A10BDF90E00814201DD0E4600E013
:10A4E0000646B54205DD934201DD184604E01046FC
:10A4F00002E0814200DD0846801CE08088E7000021
:10A500002DE9F04115460E460746114C0AF09EFE15
:10A5100080462B4632463946204607F053FF20B18D
:10A520000020A062E06950B110E020462C210DF01F
:10A53000D8FD4FF00040A0620020BDE8F081404609
:10A540000AF07DFEE06108B90120E0612046F4E7F1
:10A550006098002010B51421074800F03AFA07F07F
:10A56000F7FE40B105490160054941600549816038
:10A570000549C16010BDFEE748980020391D02085A
:10A58000AD20020871220208051D020870B50546BB
:10A590000C46084610210DF0A4FD2868007801281B
:10A5A00004D0022807D0042807D008E0A88A208019
:10A5B000E88A608003E0E86800E00A2060602868BC
:10A5C0004268002A03D02146BDE87040104770BDA4
:10A5D0002DE9FE430446808A10B9E08A002874D031
:10A5E000D4F82C805FEA080010D1204602F042FD2A
:10A5F0005FEA000869D0204604F06CFC00220921C3
:10A60000404606F08FFD607880075ED44FF4807975
:10A6100000274D4646460021304609F0EBF9384404
:10A6200007B20021304609F0EBF9C11700EB1160C9
:10A63000001210FB05F005B23046FBF769F8060082
:10A64000E9D10FB94D450CD0784201B24FF48030BA
:10A6500090FBF5F002B26B4604F11400009609F08D
:10A6600089FAADF80860ADF8046094F8400000F095
:10A670000F000328404616D0FBF79CF905464046DC
:10A68000FBF752F803460C200090B4F916102A4646
:10A69000404602F09CFBADF804004046FBF796F8FC
:10A6A000C10713D018E0FBF719F905464046FBF740
:10A6B000B5F8024603200090B4F914102B4640462A
:10A6C00002F085FBADF80800E7E736E0BDF90810B9
:10A6D000002901DDADF80860810705D4BDF9081037
:10A6E000002901DAADF80860410705D4BDF904106E
:10A6F000002901DDADF80460000705D4BDF90400B0
:10A70000002801DAADF8046001AA02A920460BF086
:10A710002EFBBDF90420BDF908104046F1F7ADFE4F
:10A720006078800709D4208BBDF808100844208386
:10A73000608BBDF8041008446083BDE8FE832DE9FA
:10A74000FC5F0446C06A5FEA000B71D094F84000D9
:10A7500000076DD008F0B6F8019000684021457EF2
:10A760005846FBF7C5FE4FF0000818B9A4F81E8044
:10A77000A4F81C805846FBF70FF982465846FBF7B1
:10A7800012F9064694F840004FF0640900F00F00FB
:10A790000C2802D003284CD09AE0A4F81C8056B1B3
:10A7A000B4F91E50002708F08DF800684946407E35
:10A7B000C0F1640022E0E08BC5F1640110FB01F1FF
:10A7C00091FBF9F0E0835846FAF7AEFF054658468C
:10A7D000FBF7F0F802460C200090B4F91E102B464F
:10A7E000584602F0F4FAE083024600231EE07A198C
:10A7F00017B210FB05F292FBF1F215B2002DF6D163
:10A80000ADF80070A4F81E806A46002120460BF0C7
:10A81000AEFA41F6FF72BDF900305142584602F0DF
:10A82000BFFDBDF800100123084402B200214CE036
:10A830009AE0A4F81E80BAF1000F0AD0B4F91C50B7
:10A84000002708F03FF800684946407EC0F16400E8
:10A8500022E0A08BC5F1640110FB01F191FBF9F03E
:10A86000A0835846FAF7DAFF05465846FBF736F854
:10A87000034603200090B4F91C102A46584602F003
:10A88000A6FAA083014600231EE07A1917B210FB36
:10A8900005F292FBF1F215B2002DF6D1ADF8007081
:10A8A000A4F81C800022694620460BF060FA41F6AD
:10A8B000FF72BDF900305142584602F0EFFCBDF87E
:10A8C00000100123084401B200225846FCF7A6FEFE
:10A8D000A08B002848D1E08B002845D1C6B9584646
:10A8E000FBF768F805465846FAF71EFF002D06DC10
:10A8F00000280DDD002D02DA01232A4604E000289D
:10A9000006DA0123404202B200215846FCF786FED7
:10A91000BAF1000F19D15846FAF780FF054658469C
:10A92000FAF7DCFF002D07DC00280EDD002D03DA2E
:10A9300001230022294605E0002806DA012300222F
:10A94000404201B25846FCF769FE0A215846019A76
:10A9500006F0E8FB6078800706D414F8400F20F07A
:10A960000F00207044F8148CBDE8FC9F70B50546BC
:10A9700000F012F804460CE02146284600F01EF8CC
:10A9800006462146284600F0A2F8204608F09CFE24
:10A990003446002CF0D170BD002800D040687047CC
:10A9A00000B503460022FFF7F7FF03E01846521CEC
:10A9B00000F004F80100F9D1104600BD0068091D3F
:10A9C00040587047006840587047002800D08068A1
:10A9D000704700224260C91C21F0030182600160BF
:10A9E000704770B504460068083008F0E1FD0500C6
:10A9F00013D00146002220460AF0BCFF294620461B
:10AA000062680AF0AEFF616819B12A4620460AF072
:10AA1000B1FF6560A06800B9A560284670BD2DE94A
:10AA2000F0410D4606000AD04DB1FFF7B5FFA84230
:10AA300008D13046FFF7D5FF041E01D01EE00020EC
:10AA4000BDE8F0813068083008F0B2FD041EF7D090
:10AA5000306822464759304639460AF082FF3A4666
:10AA6000214630460AF086FF2246294630460AF043
:10AA700081FF2A46214630460AF073FF2046DFE771
:10AA800070B504460068083008F092FD050013D048
:10AA90000146002220460AF064FF29462046A268AB
:10AAA0000AF068FFA16819B12A4620460AF059FF4A
:10AAB000A560606800B96560284670BD28B141682E
:10AAC00009B9806808B1002070470120704770B54F
:10AAD00004000DD0FFF760FF00228842204608D115
:10AAE000FFF76CFF606010B1002201461EE0A2601B
:10AAF00070BDFFF76AFF8842206808440AD10168E8
:10AB0000A16029B12046BDE8704000220AF029BFAB
:10AB1000626070BD05682046FFF750FF064602469A
:10AB2000294620460AF01DFF2A4631462046BDE848
:10AB300070400AF01FBFC0F30410072800D9072097
:10AB400070470000A0F57F41FF3905D0002804D0F0
:10AB5000712803D208490AE01F207047074971385D
:10AB600080B2096829B1064A5268904201D2085C55
:10AB70007047002070470000186F0208143800204A
:10AB8000283800202DE9F041094C90460E466268B5
:10AB90001D46074619469047306020B12868626814
:10ABA000384400219047C8F80000BDE8F08100005B
:10ABB000443800202DE9F04F87B08A46DDE910586F
:10ABC0001F4693460446002105B129805CB12078D8
:10ABD000002809D0BAF1000F05D0002618F0060FA2
:10ABE00015D0002004E0002007B0BDE8F08F401C25
:10ABF000215C0A2904D00D2902D00029F7D100E0F8
:10AC0000401C002DF0D04FF0FF312980ECE75FEAC7
:10AC1000887001D541F6FF77894608468DF81010F7
:10AC2000059125E00598CDF8189058B3002104ABA4
:10AC3000CDE902310DF1180CCDE9008C20443B46E2
:10AC40005A4651460AF04AFC06997A1A314417B21C
:10AC50000EB288B105990844059021780A290BD0D5
:10AC60000D2909D0205C0A280ED00D280CD005989B
:10AC7000205C08B1002FD5DC059848B105B12E80C5
:10AC80000598B1E70121D2E70598401C0590F3E74C
:10AC9000064A05A92046526890470146002DEFD08C
:10ACA0000022504606F053FB06B2E8E74438002085
:10ACB00000230278232902D0012A0DD00FE02AB107
:10ACC0000021012A04D0022A04D008E0012101E079
:10ACD000017004E0017001E0202902D00123184630
:10ACE00070470221F6E72DE9F0410B460F468046FA
:10ACF0000246002108460AF0F9FD05460026401CE0
:10AD000008F056FC040008D066553B464246691CD4
:10AD10000AF0ECFD2046BDE8F081FEE72DE9F047A2
:10AD2000984614460D468246DDF8209013E06608EA
:10AD300006FB0857394650464A469047002808DD2A
:10AD400044F30000C0EB540407EB0805A4F1010430
:10AD500001E005DA3446002CE9D12046BDE8F08751
:10AD60003846FBE72DE9FC5F0CAD9E4692468B46CC
:10AD700095E81201DDE91132DDE90F7C96074FF00D
:10AD8000300519D453B1D60708D002F00C0656EAA4
:10AD9000080603D05B1E01E00D55641C644504D217
:10ADA000202CF9D301E00D55641C5FEAC27903D071
:10ADB0009C4201D2202CF6D3D60624D556050AD4BF
:10ADC0004CB1644501D09C4205D1641E03D0102FC4
:10ADD00003D1641E04E0102F02D0022F0AD00EE02F
:10ADE000960603D4202C1ED2782606E0202C1AD2F8
:10ADF000582602E0202C16D262260E55641C202C08
:10AE000011D20D55641C202C0DD2B8F1000F01D0C9
:10AE10002D2506E0550701D52B2502E0150702D5A3
:10AE200020250D55641CCDE900EB064655468B46A2
:10AE300098469146900713D1274606E02A46DDE959
:10AE400000316D1C2020B0477F1C4745F6D307E03A
:10AE50002A466D1C641EDDE900311BF80400B04772
:10AE6000002CF5D15FEA897006D409E02A46DDE9B5
:10AE700000316D1C2020B047A5EB0A014145F5D3F8
:10AE80002846BDE8FC9F2DE9F04F8FB099468B46D0
:10AE9000DDE91818DDE91C63DDE91A4786469246AC
:10AEA000002009B923F010035A0507AD00D5C9B138
:10AEB000B1FBF4F204FB1212D2B20A2A01D23032F0
:10AEC00009E05FEA836C02D54FF0410C01E04FF0DE
:10AED000610C62440A3AB1FBF4F12A54401C09B1F6
:10AEE0002028E5D3CDF80880CDE90563CDE90050F1
:10AEF000CDE903474B46524659467046FFF732FFAD
:10AF00000FB0BDE8F08F2DE9FF4F8FB01CACDDE92D
:10AF1000239594E8030820AC94E8C004002450EA88
:10AF2000010201D125F010056A050DF11C0802D5BA
:10AF300050EA010217D032463B460DF073F8D2B208
:10AF40000A2A01D2303206E0AB0601D5412300E0E7
:10AF500061231A440A3A08F80420641C50EA0102EA
:10AF600001D0202CE7D3CDE90084CDF808B0CDE99D
:10AF70000595CDE9036A0FAF97E80F00FFF7F2FEE2
:10AF800013B0BDE8F08F9A4200D2885470477047E2
:10AF90002DE9FF4F89B082460A980024169D0028AB
:10AFA00001D1DFF8F0A367E1252802D02246641C16
:10AFB000E2E1491C002608460C9101782B291BD0A0
:10AFC00004DC20291BD0232904D11BE02D290ED01D
:10AFD000302909D00027C8B2FEF77BFFA8B10CA822
:10AFE000FEF760FF07461CE046F0010601E046F070
:10AFF0000206401C0C90E0E746F00406F9E746F034
:10B000000806F6E746F01006F3E70C9801782A29BF
:10B0100007D180CD002F02DA46F002067F42401CA5
:10B020000C900C984FF0000801782E2917D1401C85
:10B030000C9046F480660078FEF74BFF20B10CA818
:10B04000FEF730FF80460AE00C9908782A2806D1DE
:10B0500001CD002800DC0020491C80460C910C9892
:10B0600001786C290AD004DC68290FD06A2918D12C
:10B0700027E0742928D07A2913D125E0401C0C90B0
:10B08000017846F480766C291BD00AE0401C0C90B5
:10B09000017846F08006682903D146F04006401C3E
:10B0A0000C9002460078692822D015DC62281FD057
:10B0B0000DDC252877D050281AD058287FF476AF99
:10B0C00016E046F40076EAE746F48076E7E7632880
:10B0D0006AD06428F2D10BE073286FD004DC6F28AB
:10B0E00006D07028EAD103E0752801D07828E5D190
:10B0F00078280DD058280BD070280BD0502809D0B4
:10B100006F2816D0622816D00A2126F0100616E005
:10B11000102107E05078102146F48876562804D193
:10B12000521C0C921078582807D01078502804D060
:10B1300005E0082108E0022106E046F0200610782C
:10B14000692803D0642801D026F00C06700501D5CB
:10B1500026F001061078692813D0642811D05628EB
:10B1600054D0B00560D5ED1D0020CDE90410CDF818
:10B1700018800290CDE9077625F00705F5E8020171
:10B1800021E0B00528D5ED1D25F007050023F5E8E1
:10B1900002020DF11009002A89E80A01CDE90776BB
:10B1A00003DA012102E0E4E070E0002100230291D3
:10B1B00019461B1A914102DA114604E08EE0002183
:10B1C000404261EB0201CDE90001DDE90A132246AC
:10B1D0005046FFF798FE4BE0F00503D501CD0BE09C
:10B1E000404210E0700602D515F8040B04E030066A
:10B1F000F4D535F8040B00B2CDE90218CDE9047698
:10B20000C10F0028ECDDCDE900012BE001CD416844
:10B210000968009103680B98021B0A9801195046AF
:10B22000FFF7B6FE044424E0F00508D5CDE9021886
:10B23000CDE9047602CD0020CDE9001012E07006C1
:10B2400002D515F8040B06E0300603D535F8040BDB
:10B2500080B200E001CDCDE902180021CDE9000166
:10B26000CDE90476DDE90A1322465046FFF70BFECE
:10B2700004460C98401C0C900C99087800287FF428
:10B2800093AE0B9884427BD222467AE04FF00108BD
:10B29000B00707D50BE02246DDE90A13641C202025
:10B2A000D446E047404608F10108B842F3D3DDE94F
:10B2B0000A13224615F8040B641CD446E047B00775
:10B2C00006D4D6E72246DDE90A13641C2020D047C5
:10B2D000414608F10108B942F4D3CAE755F804BB66
:10B2E000B8F100005A4601D0014601E04FF0FF31AD
:10B2F000584600E0401C03780BB1491EFAD2A0EB7F
:10B300000209700505D548464146C14500D30846A7
:10B310008146B00707D514E02246DDE90A13641C14
:10B320002020D446E047494609F10109B942F3D348
:10B3300007E0DDE90A1322460BF1010B641CD44639
:10B34000E0479BF8000020B17105F2D5B8F1010883
:10B35000EFD2B00706D48CE72246DDE90A13641C5D
:10B360002020D047494609F10109B942F4D380E7CA
:10B3700006E02246641C2520DDE90A13D04778E761
:10B38000421E034600200A99D0470DB02046BDE872
:10B39000F08F00008FAF010810B503004FF00000E0
:10B3A0000DD04A1E114200D0FEE71944491E9143B8
:10B3B0000A46B1F5004F02D20C2A01D9084610BD49
:10B3C0000C2010BD08444A1E401E9043114200D07C
:10B3D000FEE770472DE9F0410446012000250F46A5
:10B3E00060862E460BE01B490CF0C1FE10B16D1CAF
:10B3F000ADB202E0608E401C6086761CB6B257F893
:10B40000260010B101780029EDD1208EA8421ED06F
:10B41000A06A002610B108F057F9A662E06A10B1E0
:10B4200008F052F9E662E80008F0C2F8A06238B10C
:10B43000680008F0BDF8E06218B1A16A11B102E03D
:10B44000FEE7FEE7002569000CF04BFE2586BDE80F
:10B45000F08100004806020870B5044640680D46B9
:10B4600008B1FFF7F9FF2268002A04D029462046D8
:10B47000BDE87040104770BD89B204F0AFBC89B21E
:10B4800004F032BD70B50D46044600F04DF800B131
:10B49000FEE76868616820F00300001D08446060F2
:10B4A000204600F049F8204670BD4068103120F079
:10B4B0000300884201D301207047002070472DE926
:10B4C000FC47054648680C4620F0030001AA69467F
:10B4D0000AF031FADDE9006005EBC61101EB8009E5
:10B4E0008046D9F8380060B164B1C4E9020504F1BE
:10B4F0000807C46038460421FFF764FF874202D082
:10B50000FEE7FEE7FEE7C9F838400123286903FAA1
:10B5100006F10843286105EB860003FA08F1426949
:10B520000A434261BDE8FC87406830F0030001D067
:10B53000002070470120704710B5044600F08CF8D9
:10B54000046010BD2DE9FC474FF0000780460E0057
:10B5500001973D46009745D00C460DF1040AE94697
:10B56000802907D308460BF023FB411F01208840A8
:10B57000401E04444A46514620460AF0DCF9019C2C
:10B58000092C2FDA08EB8400009940694FF0FF3254
:10B5900002FA01F1454608400CD1641C2869A2401A
:10B5A000104016D00BF0FCFA0446019005EB800029
:10B5B000406980B10BF0F4FA05EBC411009001EB87
:10B5C0008000856B75B1686820F00300B04203D23B
:10B5D000FEE73D46F6E7FEE7DDE900322946404654
:10B5E0000AF036FB2846BDE8FC8710B50446FFF795
:10B5F000A3FF416841F002014160606840F0010032
:10B60000606010BD10B5044600F026F8416821F0D6
:10B6100002014160606820F00100606010BD70B5FB
:10B6200006460D46084600F017F8040008D02079B9
:10B6300010F0010F0ED02846FFF776FF08B1FEE7A5
:10B64000FEE72146304600F03EF821462846FFF747
:10B6500019FF0546284670BD10B5426800F1080183
:10B6600022F00302121F8C18FFF75EFF00B1FEE705
:10B67000204610BD70B506460C004FF000001FD0EC
:10B68000FAB12079154610F0010F1BD01146204663
:10B69000FFF70BFF78B12946204600F025F8054654
:10B6A0002046FFF749FF6868294640F002006860BD
:10B6B0003046FFF704FF2046FFF7A4FF04F108001F
:10B6C00070BDFEE7FEE77CB5054648680C4620F0F5
:10B6D00003006A4601A90AF02EF9DDE9003221468D
:10B6E00028460AF0B5FA7CBD2DE9F0410D46044626
:10B6F0000830091F4618606806F1080720F00300AB
:10B70000401BA0F1040838460421FFF75BFE874286
:10B7100000D0FEE7606808EB050120F00300091D7A
:10B72000884200D0FEE7307900F0030040EA0800CC
:10B73000706020F003000C2800D2FEE7207900F0B2
:10B740000300284360603046FFF74FFF3046BDE8F6
:10B75000F08170B505F0D9FC0546F9F7D9FF04462C
:10B76000284605F00EF801462046BDE8704000224C
:10B7700009F092BC2DE9F04F0C4687B00546002138
:10B78000F9F7C6FE60B32146284600F021F92146AC
:10B79000284600F06FF80021284608F0A1F805902F
:10B7A0000021284608F0DEF804900021284608F021
:10B7B00050F8012800D0002080460021284608F0DB
:10B7C0002BF906460021284608F066F842F2D179A6
:10B7D00007464E450BD1688C000508D4012607E0CA
:10B7E00007B02046BDE8F04F1C210CF07ABC0026C3
:10B7F0002846F9F70DFFDFF878A083462846002198
:10B80000BAF80420FAF709FDD4F810C0A36821683B
:10B81000CDF800C0CDF80C80CDE90131C2B231467F
:10B820005846059B02F096FC20834F4504D1688C56
:10B83000400501D4012600E000262846F9F7CCFE99
:10B84000074628460021BAF80820FAF7E6FCC2B2FB
:10B85000606900256368E1688DE82B003146384651
:10B86000049B02F077FC608307B0BDE8F08F000016
:10B87000883700202DE9F34F81B00C46019802F083
:10B8800051FA80460198F9F7C3FE8346404600F01E
:10B890008AFB2061400007F0B9FE2060206940006B
:10B8A00007F0B4FE002541F69A79A06035E038F93A
:10B8B0001510454E49452FD10027DFF810A11CE097
:10B8C00039460198F9F724FE51460090FAF717FE21
:10B8D00090B9009802F038FA01280DD1009802F0D2
:10B8E00029FAA84208D10098FAF7E3FDB04203DB39
:10B8F0000098FAF7DEFD06467F1C0198F9F71AFE5C
:10B90000B842DDD8002E03DBA06820F8156003E004
:10B91000A168002021F815006D1C2069A842C6D836
:10B9200000252F46284641F69B764A4615E038F911
:10B930001010B14204DB0D44A5F5F8559B3D0BE01A
:10B94000914204D1A16831F81010394403E0A36892
:10B9500023F8101039440FB2401C21698142E6D807
:10B960000021019807F0BCFF2169C1F1010200FB31
:10B9700002B0C01B01B2002900DA002100224FF002
:10B98000FF37104610E038F91030B3420BDBA3F557
:10B99000F8539B3B1AB211FB02F3B3FBF5F3A76814
:10B9A00027F810300746401C23698342EBD8002F4C
:10B9B00007DBA81A4843B0FBF5F0081AA16821F884
:10B9C0001700BDE8FE8F000001E0FFFF0100060048
:10B9D0002DE9F84F0C46834602F022FB804600F02A
:10B9E000E2FA6061400007F011FE606060694000AB
:10B9F00007F00CFE002541F69A79E06035E038F951
:10BA00001510474E49452FD10027DFF818A11CE03B
:10BA100039465846F9F77CFD51460090FAF76FFD1C
:10BA200090B9009802F00EFB01280DD1009802F0A9
:10BA3000FFFAA84208D10098F9F72FFEB04203DBC5
:10BA40000098F9F72AFE06467F1C5846F9F772FD62
:10BA5000B842DDD8002E03DBE06820F8156003E073
:10BA6000E168002021F815006D1C6069A842C6D865
:10BA700000252F46284641F69B764A4615E038F9C0
:10BA80001010B14204DB0D44A5F5F8559B3D0BE0C9
:10BA9000914204D1E16831F81010394403E0E368C1
:10BAA00023F8101039440FB2401C61698142E6D876
:10BAB0000021584607F056FF81465846F9F78CFD9D
:10BAC0006169C1F1010209FB0200C01B01B200293A
:10BAD00000DA002100224FF0FF37104610E038F95D
:10BAE0001030B3420BDBA3F5F8539B3B1AB211FBAA
:10BAF00002F3B3FBF5F3E76827F810300746401C64
:10BB000063698342EBD8002F07DBA81A4843B0FBD8
:10BB1000F5F0081AE16821F81700BDE8F88F000079
:10BB200001E0FFFF010006002DE9FF4F87B0C87854
:10BB3000189CC0070D46002801D0E84800E0E848FE
:10BB4000059001D0E74800E0E748824601D1E5488A
:10BB500000E0E54804906188A2884FF0000BA1EB5B
:10BB60000201584609B25A46D4F810C010E002EB60
:10BB700082034FF01007E66807EB8307F75DFF07C6
:10BB80000AD0082707EB8303F35AC91A09B2521CDB
:10BB90009445ECD8002246E00C2707EB8303F35AC8
:10BBA000184400B2F3E709EB89031022E66802EBC0
:10BBB00083020092B25CD20733D1A8B191FBF0F7B7
:10BBC0000C2202EB830E36F80E207A43042707EB93
:10BBD000830736F907C0062707EB8307F75F12B222
:10BBE000974202DD904601E0FEE7B846C44501DD1C
:10BBF000674602E0974200DD1746974205D0009A5B
:10BC00004FF0010CE34646F802C0E668082202EB5A
:10BC10008302B752E36833F80E20801AC91B00B2C2
:10BC200009B209F10102236991464B45BBD8BBF12A
:10BC3000000F90D10021079807F005FE012800D0E1
:10BC4000002083460020ADF80800ADF80C0003A9E1
:10BC500002A8CDE900012089B4F9022003B22878B6
:10BC6000169909F093FEE97811EA0B0F07D00798AF
:10BC7000F9F7CEFCBDF808100844ADF808000999A2
:10BC80000798F9F745FC0BE098493046FAF737FC7E
:10BC900078B1E87809AAC0F38001079802F0ADF9FD
:10BCA000060003D0DDE909018842EDD10BB0BDE803
:10BCB000F08F0021304607F0DFFDE8B3002738465B
:10BCC00021690FE0E26800EB800352F82320B242C2
:10BCD00007D100EB8002E168082000EB82000F5ED4
:10BCE00002E0401C8142EDD8E878C007708C04D097
:10BCF00020F4806040F4006003E020F4006040F431
:10BD00008060708406F11400804651468847B8422E
:10BD100028D03046FAF77EFEB08AADF80000F08AEF
:10BD2000ADF80200308BADF80400708BADF8060062
:10BD300039464046059A00E010E090476A462921BE
:10BD4000304605F0EFF93046F9F7E2FC32462221A1
:10BD500005F0E8F93046FAF75DFE03E0708C20F458
:10BD60004060708468784FF0000901280FD00228E5
:10BD700015D1049906F114008847B4F90010491C44
:10BD800021F00101081A00EBD070401005E0049981
:10BD900006F1140088472188081A0FFA80F9E8781C
:10BDA00010EA0B0F08D006F1140051468847BDF881
:10BDB0000810081AADF80800304600216B22FAF787
:10BDC0002CFA0FFA80F8304600216C22FAF725FA97
:10BDD00007B23046FAF76DFB00903046F9F75DFC8C
:10BDE0000146C8F34130012810D128F4C040B0F515
:10BDF000FA6F0BDCB0F57A7F01DDC0F57A70009A3E
:10BE00005043642290FBF2F00FFA80F8C7F3413000
:10BE100001280ED127F4C040B0F5FA6F09DCB0F567
:10BE20007A7F01DDC0F57A704843642190FBF1F020
:10BE300007B2B18A1498411A01EB080002B2F18AE4
:10BE40001598401A384401B2E878C007002802D09B
:10BE5000BDF9080000E04846104407B201D048464A
:10BE600001E0BDF9080008440FFA80F857EA08001D
:10BE700019D03046FAF7CEFDB08A3844B082308B04
:10BE800038443083F18A01EB0800F082718B01EBBA
:10BE9000080070833046FAF7BDFD0023424639465C
:10BEA0003046FAF75DFEE87810EA0B0F0CD106F188
:10BEB00014005146884717990844BDF80C100844EF
:10BEC000BDF80810084406E0BDF80C1017980844A7
:10BED000BDF80810081AADF80800DAE67B00020881
:10BEE00071000208FFFF0108B3FF0108010006000E
:10BEF000F8B5044605F009F90546204605F0C7F8EF
:10BF000006462846F9F704FC04462B2E37D00A2EA5
:10BF100034D106F0D7FC10B1007901282ED0694643
:10BF20002846F9F75BFC94F82C0010F00C0F28461B
:10BF30002ED0F9F76DFB05460021204607F08FFC57
:10BF40000128BDF9000005EBD5711ED000EB6100A2
:10BF500090FBF5F001B2002900DA0021608D002588
:10BF6000884200D001250122204609F095F8002DD5
:10BF700004D000221C21204605F0D4F8F8BD618DC4
:10BF8000BDE8F840002209F087B8C0EB6100DFE7A8
:10BF9000F9F722FBBDF9021000EBD07201EB620150
:10BFA00091FBF0F0D6E70146002041F6FF7200E079
:10BFB000401C31F910309342FAD1704708B5084659
:10BFC000114604F0B2FD0090BDF8000008BD00006D
:10BFD0002DE9F04F93B0834605F059F806465846D0
:10BFE00005F093F80446122E7ED0152E01D0182E9F
:10BFF0007BD1FAF75EFA06902046F9F74EFB0590E2
:10C00000204600213222FAF708F905462046002191
:10C010001222FAF702F928440FFA80F8204600218C
:10C020001322FAF7FAF828440FFA80FA2046002182
:10C030001022FAF7F2F8284407B220460021112214
:10C04000FAF7EBF82844618E0FFA80F901EB08004B
:10C05000ADF83C00A08E3844ADF83E0094F83900AD
:10C0600000F0030001287DD00FA9E08ECDE900018A
:10C07000DDE90521B4F9303003A8FEF78BF9BDF8EE
:10C080000C10A08A0844ADF80C00BDF80E10E08A30
:10C090000844ADF80E00BDF81010A08A0844ADF8B1
:10C0A0001000BDF81210E08A0844ADF8120004F147
:10C0B00014010D4610A80D9103F06CFF03A928464A
:10C0C00003F068FF5946D24807F08EFB012860D183
:10C0D00010A90D9803F05EFF152E5AD1E08D0028AF
:10C0E00057D0A08D002801E056E052E051D0E08EFC
:10C0F00000284ED0584604F0D0FF064601A80D99FE
:10C1000003F048FF204606F0DBFA054694F83900B4
:10C1100000F0030001287CD0BDF81000BDF80C1021
:10C12000401ABDF804100844ADF80800BDF812002C
:10C13000BDF80E10401ABDF806100844BDF80410F2
:10C14000ADF80A0001EB0800ADF80400BDF80600E8
:10C15000BDF808103844ADF80600A1EB0A00ADF8B0
:10C16000080000E07DE0BDF80A10A1EB0900ADF881
:10C170000A0094F8381001F0030001286FD08907F5
:10C180006DD002286CD00023194630460D9AF5F781
:10C190009DFE13B0BDE8F08F584604F0B4FF05468D
:10C1A00000780228F5D094F838004FF00106C1431A
:10C1B00089074ED000F0030102294AD0C0F3840061
:10C1C000042801D0012844D1204600214622FAF754
:10C1D00024F8C0B2FF283CD1208ED0BB584604F0D2
:10C1E00092FF0746E08EB0F5807F34D02046F9F705
:10C1F00054FA80462046FAF75CF9014604F132020F
:10C20000E08ECDE900020023424602A8FEF7C2F804
:10C2100000E02BE0BDF80800A18A00220844ADF838
:10C220000800BDF80A00E18A0844ADF80A00BDF82C
:10C230000C00A18A0844ADF80C00BDF80E00E18A9C
:10C240000844ADF80E0002A93846FDF70AFF0028A1
:10C250009FD12E709DE7002204F11401F4E730E035
:10C26000C5E003A92046F9F7EFF920E7B4F92C005F
:10C2700029B2401ABDF80410401C00EBD070A1EBAD
:10C280006001ADF80410BDF80810BDF80620A1EB60
:10C290006000ADF80800B4F92E002914401A401CC3
:10C2A00000EBD070A2EB6000ADF80600B4F92E00F0
:10C2B000401ABDF80A10401C00EBD070A1EB6000E2
:10C2C0003CE707A8F5F736FE07AA00212046FAF753
:10C2D000A0F9E08EADF81E00208EADF81C00608E37
:10C2E000ADF82000A08EADF8220094F83800BDF81B
:10C2F0000C10C0098DF8300001EB0800ADF83400D7
:10C30000BDF80E00BDF810103844ADF83600A1EBB2
:10C310000A00ADF83800BDF812100DAAA1EB090013
:10C32000ADF83A00B16810468846FDF772FE002865
:10C3300090D00DA8B060B4F92800B4F92C1090FB8F
:10C34000F1F201FB1207B4F92A00B4F92E1090FBA8
:10C35000F1F201FB1200BDF90610084400B2ADF87D
:10C360001600884203DDE18D401AADF81600E18D1C
:10C3700080B20844401E2FE0BDF90410C81900B275
:10C38000ADF81400884203DDA18D401AADF8140009
:10C39000A18D80B20844401E0DE005AA07A93046D1
:10C3A000636AF5F793FDBDF814002844ADF8140056
:10C3B000BDF818002844ADF81800BDF91400BDF907
:10C3C00008108842E9DBBDF8161028140144ADF8C6
:10C3D0001610BDF81A100844ADF81A00BDF9160081
:10C3E000BDF90A108842C7DBC6F80880D1E605A867
:10C3F000F6F74EF805AA00212046FAF75DF900206D
:10C400000090636A05A930460D9AF5F7ADFDC0E6C8
:10C41000FC6F02082DE9F0438FB0044604F075FE6E
:10C420000546F9F775F9064601A8F6F731F801AAAD
:10C4300000213046FAF740F9284606F079FD28B188
:10C440009DF8210040F001008DF82100204604F005
:10C4500024FE816804460F4606F114020DA8FDF77C
:10C46000D8FD002850D00DA8A0600BA9304601F0DF
:10C47000F3FDA88AADF82400E88AADF82600288BE1
:10C48000ADF82800BDF82E00ADF82A0009AA104624
:10C49000A168FDF7BEFD4FF000080DF1240978B149
:10C4A000A6682846C4F8089006F047FD034605F143
:10C4B000140201A92046CDF80080F5F755FDA660CD
:10C4C000A88AADF82400BDF83200ADF82600288B0C
:10C4D000ADF82800688BADF82A0009AA1046A168BB
:10C4E000FDF797FD78B1A6682846C4F8089006F0D5
:10C4F00024FD034605F1140201A92046CDF8008071
:10C50000F5F732FDA660A7600FB0BDE8F08300002C
:10C510002DE9F04FCDB0054604F0F7FD0446008E3E
:10C5200000287CD0284604F0B8FD4590608C40F08F
:10C5300008016184204643A9F9F786F80026B4F87B
:10C5400020802684608C374640F00801354661849F
:10C550002DA8F6F779FD3BA8F5F79AFF4FF4A0292F
:10C560002DAA49462046FAF7F7F83BAA4946204645
:10C57000FAF7A2F8608C20F008016184A4F820800A
:10C580000021204607F006FA4C900021204607F0D3
:10C5900095F94B900021204607F0BAF94A90002106
:10C5A000204607F0CDF9499011A84599F8F704FE07
:10C5B000B248CDE9120503A8159025A8CDF87890CA
:10C5C000169050E17F1CBFB2606AADA150F8270001
:10C5D0000BF0CDFD0028F5D0E06A30F81600C0F36E
:10C5E0000011002976D10025C0F3002101B10125F9
:10C5F000C0F3801010B145F0800518E0A08EB04265
:10C6000015D15FEA886001D545F020055FEA8870A2
:10C6100001D545F002055FEA487003D500E02AE144
:10C6200045F004055FEA087001D545F00805A06AE9
:10C6300000EBC60123A803F0A4FCBDF88C10BDF8E4
:10C640000C010144ADF88C10BDF88E20BDF80E1120
:10C650000A44ADF88E20BDF890201044ADF890004B
:10C66000BDF892000844ADF8920045B32584608C73
:10C6700040F00801618403A8F6F7E6FC25A8F5F769
:10C6800007FF4FF4A02903AA49462046FAF764F8A9
:10C6900025AA49462046FAF70FF8A4F82080608CB6
:10C6A00020F008016184E06A30F81600C0F3C02071
:10C6B00000289DF8B1000ED040F001000DE003A865
:10C6C0002DA938220BF0E5FC25A83BA920220BF070
:10C6D000E0FCE8E7C3E020F001008DF8B10023A8FA
:10C6E000149011AA1A211F96204604F01BFD9DF8F4
:10C6F0002F004108C9063CD520F03E001E308DF8C1
:10C700002F00B4F914304A99BDF98C2019448A429B
:10C7100003D120F008008DF82F00B4F918204998B3
:10C72000BDF99010101A814205D19DF82F0020F01C
:10C7300010008DF82F00B4F916204C98BDF98E101A
:10C740001044814205D19DF82F0020F004008DF89F
:10C750002F00B4F91A204B98BDF99210101A81429B
:10C7600007D19DF82F008108490061F345008DF83D
:10C770002F00BDF89210BDF98E00091A491C0FFA5E
:10C7800081F9A90608D5E16A31F81610490503D5E3
:10C79000A0EB0900ADF88E0023AA03A94598F6F78F
:10C7A0003FFC25984890606ABDF9A8B0BDF9A6A0E5
:10C7B00050F82700469043A803F02DFC9DF8B120C7
:10C7C000CDF800A0CDE901025B4647A8489A4699FA
:10C7D00008F026FF23A803F01EFCBDF91C31BDF8AC
:10C7E0008C10C01A00EBD07001EB6001ADF88C101A
:10C7F000BDF89200BDF88EC0BDF91E21A0EB0C0063
:10C80000401C00B2801A00EBD0700CEB600000B24C
:10C810001944ADF8901081180AB2ADF88E00ADF849
:10C820009220A9060ED5E16A31F81610490509D5FE
:10C8300009EBD971A0EB6100ADF88E00A2EB6100AD
:10C84000ADF892000020009023AA25A9469B4598A8
:10C85000F5F78AFB11AA1B21204604F063FC761C25
:10C860007F1CB6B2BFB2208EB0423FF6ADAE608C38
:10C8700020F0080060844DB0BDE8F08FC46F02085E
:10C880000A0000002DE9F04790B0054604F03DFC99
:10C890000446284604F001FC06460BA92046F8F79A
:10C8A0006DFE94F848000025C10600D501258006DC
:10C8B00001D545F002050021204607F0B3F8A0F5A8
:10C8C0001C51D13904D1608C000501D445F0040518
:10C8D00003A8F5F7DDFDB4F84400ADF82200B4F884
:10C8E0004600ADF824008DF8295003AA0021204607
:10C8F000F9F7E2FE9DF828004FF0010808B98DF81D
:10C900002880E06B0490206C059004994FF6FF702E
:10C9100081421ED0059981421BD04FF480292746C1
:10C92000552249462046F9F778FC024649463846E2
:10C93000EFF7C7FD0090BDF80000ADF81A002046E3
:10C9400020224946F9F769FC0090BDF80000ADF8D7
:10C950001C0094F8480041F6FF7A00F00700022816
:10C9600001D003281AD19DF82800022801D00328FD
:10C9700014D1BDF91E10CDE9001A0295BDF9203081
:10C98000039A0DA8616A08F04BFE0BA803F049FB5F
:10C99000BDF93410884201DA8DF8288094F84800F7
:10C9A00004F1300700F00700032805D00BA803F0BE
:10C9B0000CFBB0F5806F00DA00270BA90EA8B26857
:10C9C000FDF727FB00287DD094F8480040070BD1E5
:10C9D0002046F8F7EFFF404202B200210BA803F017
:10C9E00033FB608BADF8320094F848000DF1380944
:10C9F00000F00700022813D0032811D000970BAADB
:10CA000003A93046636AF5F7AFFAB068C6F8089034
:10CA1000804694F8480000F0070003280FD058E043
:10CA2000D6F80880C6F8089000970BAA03A93046EC
:10CA3000636AF5F799FA4046C6F80880E6E7BDF95B
:10CA40001E10CDE9001A0295BDF92030039A0DA8F9
:10CA5000616A08F0E5FD0BA803F0E3FABDF93410B4
:10CA6000884219DA20221146039804F070FCB4F8C9
:10CA70004410BDF8342000EB400011440844ADF8E8
:10CA80002200B4F84600ADF8240000970BAA03A9D1
:10CA90003046636AF5F768FA0BA803F096FA014688
:10CAA000BDF93600814214DAB4F84410ADF8221012
:10CAB0000399B4F84620098910440844ADF82400CD
:10CAC000009700E007E00BAA03A93046636AF5F778
:10CAD0004BFAC6F8088010B0BDE8F0872DE9F043A6
:10CAE00093B0074604F0D3FA0546384604F00DFB30
:10CAF00004464FF48026152D7ED0182D7DD1384662
:10CB000004F0CBFA054603A8F5F7C2FC03AA3146A8
:10CB10002046F9F7D1FD0EA9204601F09DFA0EAA94
:10CB200010A8A968FDF775FA002866D0204601F024
:10CB300061FA814606F0FCF928B19DF8290040F021
:10CB400001008DF829002046F9F7B3FC0646484657
:10CB500006F0F3F90146BDF91E00CDE900060222F8
:10CB60000292BDF920300DA8039A08F059FD204625
:10CB7000F8F793FDB4F9161000EBD076B9F916006A
:10CB800001EB6601471A4846F8F787FDB90391FBA8
:10CB9000F0F70021204606F018FF0399B0F90800CD
:10CBA000B1F90810081A00EBD070BDF8361040102B
:10CBB000091A09B2ADF83610E28A794302EB66022F
:10CBC00002EBA1310E1A0021204606F04EFE8046EF
:10CBD000204600211222F9F720FB074620460021BB
:10CBE0001322F9F71AFBA28A07EB08011144ADF8EA
:10CBF0002C10ADF82E6001E023E01FE0218B081A15
:10CC0000A0EB0800ADF83000BDF836003044ADF8B8
:10CC100032009DF8290040F002008DF8290010A88C
:10CC2000AC68A860484606F088F9034600200090EA
:10CC30000BAA03A92846F5F797F9AC6013B0BDE835
:10CC4000F083384604F029FA05460EA9204601F083
:10CC500003FA6846F6F7F8F96A4631462046F9F7CE
:10CC60007BFD0EAA69462846F6F7DAF9E6E72DE9D4
:10CC7000F043A1B0054604F048FA0446284604F003
:10CC80000CFA81460021204606F048FE07460021A6
:10CC9000204606F05BFE06460021204606F080FE98
:10CCA00005460021204606F00FFEA38AE28AADF871
:10CCB0007A20218BADF87C10B4F81AC0891BADF82E
:10CCC0007C103B44ACEB0000ADF878305119ADF866
:10CCD0007E00ADF87A106846F6F7B6F96A464FF46A
:10CCE00000312046F9F738FD1EAA69464846F6F796
:10CCF00097F92046F8F7D1FC0646208BA18A401A06
:10CD0000401C801B05B2606A411C06D06843C117F5
:10CD100000EB1160001207B208E02046F9F7AAF90B
:10CD2000C0F3000008B12F4600E000272046002194
:10CD30001622F9F772FAC0B2012801D1E81B07B236
:10CD4000A08A4FF440353844ADF870003044ADF857
:10CD50007400E08AADF87200608BADF87600294669
:10CD6000204606F0DBFD07462946204606F0EEFD8C
:10CD700080462946204606F013FE064629462046F0
:10CD800006F0A2FDBDF87010BDF87420C91BADF807
:10CD9000701002EB0801ADF87410BDF87210891B19
:10CDA000ADF87210BDF876100844ADF876000EA804
:10CDB000F6F74AF90EAA29462046F9F7CDFC1CAA37
:10CDC0000EA94846F6F72CF921B0BDE8F0832DE90D
:10CDD000FF4F81B00C4680462021DDF838A0F9F7DE
:10CDE00087FB002878D0BAF1030F404621D0F8F72E
:10CDF000DAFD814605F076FD0546002708F11400AE
:10CE000000903E46BAF1030F3946404614D006F072
:10CE1000B5FD82460021404606F044FD8346484663
:10CE2000B9F1010F59D002285FD0B9F1030F63D1D6
:10CE300038E0F8F7B1FDDCE706F05EFD834600213F
:10CE4000404606F071FD82464846B9F1010F19D0FF
:10CE500002281FD0B9F1030F4ED1009803F0C9F892
:10CE6000A0EB0B01A1EB0A00B8F8141000EBD07294
:10CE70000BEB6200084407B205F1140003F0B9F8A7
:10CE8000A98A23E0B8F81410B5F9146001EB0B007F
:10CE900007B231E0B8F81810B5F91860A1EB0A0034
:10CEA00007B229E0009803F07EF8A0EB0A01A1EB9D
:10CEB0000B00B8F8161000EBD0720AEB62000844C1
:10CEC00007B205F1140003F06EF8E98A00EBD070A8
:10CED00001EB600006B20FE030E0B8F81610B5F9CB
:10CEE000166001EB0A0007B206E0B8F81A10B5F9AF
:10CEF0001A60A1EB0B0007B2A01E049900B2002932
:10CF000010DAB9F1000F15D0BE4221DC12E0002C7E
:10CF100001DDA41C24B2E01704EB9070801005B072
:10CF2000BDE8F08F0399002912DAB9F1000F01D0A2
:10CF3000BE420DDB002CEADA0446E8E70498E04242
:10CF400002D50498404204B20398001B00D5039C0C
:10CF50002046E4E770B5044605F0B4FC48B100682B
:10CF600082680AB1217A9047207E810743D4C007A6
:10CF70007CD101260021606806F04CFC00251AE0F7
:10CF8000016899B1017ACA0910D0802904D0227AA7
:10CF900021F08001914209D14168E1600168204699
:10CFA0008847207E810726D4C0075FD16D1C2946A3
:10CFB000606806F02FFC08B1002EE1D12146002068
:10CFC00006F012FC051E03D00021606806F022FC6A
:10CFD000002619E0016891B1017A0A060FD411B157
:10CFE000227A91420BD14168E1600168204688476E
:10CFF000207E810701D5012070BDC00736D1761C87
:10D000003146606806F006FC10B1012DE2D02FE039
:10D01000012D2DD16068416851B3217E490727D485
:10D02000217A232919D0242917D0A903F9F760FA06
:10D03000F0B1207A11381C280FD2DFE800F019195E
:10D040001919191919191919190E0E190E0E19197C
:10D0500019190E0E0E0E19190E19606840686060DD
:10D060002046FFF777FF0546012801D0002070BD5C
:10D07000284670BD2DE9F04F89B00546002002908A
:10D08000039005F01FFC00680026B146047E686A24
:10D090000090288BA98A08442883688BE98A084471
:10D0A00068830098E5E04FF000084FF48077CDF8F2
:10D0B0001C8000980EE0002106F09CFC40440FFA12
:10D0C00080F80021504606F09BFC47433F12504633
:10D0D000F8F71EFB5FEA000A5046ECD1A869019000
:10D0E000B8F1000F02D1B7F5807F0AD0C8F1000077
:10D0F00001B24FF4803090FBF7F207AB01A806F0C5
:10D1000039FDBDF90410002900DC4942BDF90600D3
:10D11000002800DC4042814201DD012601E04FF0A1
:10D12000010910210098F9F7E3F900287ED0B046F4
:10D13000CB46CA4647460098F8F748FBC10700D1DE
:10D140008846810700D40027410701D44FF0000B27
:10D15000000701D44FF0000A0098F8F72BFC069066
:10D160000098F8F7E1FA05900098F8F757FB04905B
:10D170000098F8F7B3FB0699002902DC059900290D
:10D1800012DDBBF1000F03D0BDF90610A14207DA92
:10D19000BAF1000F08D0BDF906106242914203DCDB
:10D1A000009902910C2103910499002901DC0028C7
:10D1B00010DDB8F1000F03D0BDF90410A14205DA6B
:10D1C00047B1BDF904106242914203DC009902911B
:10D1D000032103910699002901DC4FF0000B05990A
:10D1E000002901DC4FF0000A0499002901DC4FF00E
:10D1F0000008002800DC0027B8F1000F03D0BDF9BB
:10D200000400A04216DA27B1BDF904006142884249
:10D2100010DDBBF1000F03D0BDF90600A04209DA12
:10D22000BAF1000F11D0BDF9060000E00DE0614237
:10D2300088420ADC0EB1032000E00C2095F8401073
:10D2400060F3030185F8401016E04FF480710098F8
:10D25000F9F74EF936EA00000ED14FF4007100984C
:10D26000F9F746F939EA000006D10098F8F750FAC4
:10D27000009000287FF417AF029858B195F840004D
:10D28000039961F3030085F840000298E8620020EA
:10D2900028836883029809B0BDE8F08F2DE9FF5F0D
:10D2A0000646F8F779FBB0F1000A72D041F6FF7438
:10D2B0000021304606F020FB80460021304606F073
:10D2C00033FB81463046F8F735F98346002758E0AE
:10D2D000B0683249006850F827502846F9F70FF92E
:10D2E000F0BB4FF480512846F9F702F9C0B350461D
:10D2F000BAF1010F05D0022809D0BAF1030F3FD1CE
:10D300001AE0B18AB5F9145001EB080004E0318B42
:10D31000B5F91850A1EB09000399019A294409B203
:10D3200000B291422CDB029A914229DC081A00B229
:10D3300000281CDD01461BE005F1140002F059FE37
:10D34000A98A00EBD07001EB600005B206F1140071
:10D3500002F04FFEA0EB0801A1EB0900B18A00E04A
:10D360000EE000EBD07208EB62000844D4E74142C3
:10D37000002C01DD224600E06242914200DA0446C0
:10D380007F1C5F45A4D3A4F5F850FF3804D0604259
:10D3900000B204B0BDE8F09F0020F9E701000400EE
:10D3A0002DE9FF5F0646F8F7FEFAB0F1000A72D0E9
:10D3B00041F6FF740021304606F0E0FA8046002175
:10D3C000304606F06FFA81463046F8F7B3F88346E8
:10D3D000002758E0B0683249006850F827502846C6
:10D3E000F9F78DF8F0BB4FF480512846F9F780F833
:10D3F000C0B35046BAF1010F05D0022809D0BAF1E6
:10D40000030F3FD11AE0F18AB5F9165001EB08007D
:10D4100004E0718BB5F91A50A1EB09000399019A48
:10D42000294409B200B291422CDB029A914229DCD4
:10D43000081A00B200281CDD01461BE005F11400AB
:10D4400002F0B1FDE98A00EBD07001EB600005B29B
:10D4500006F1140002F0A7FDA0EB0801A1EB090002
:10D46000F18A00E00EE000EBD07208EB62000844A5
:10D47000D4E74142002C01DD224600E062429142A5
:10D4800000DA04467F1C5F45A4D3A4F5F850FF38AA
:10D4900004D0604200B204B0BDE8F09F0020F9E77C
:10D4A000010004002DE9FF4F83B00F46DDE910A411
:10D4B00093460021039806F0A9FA05460021039837
:10D4C00006F0E4F9F9788A070BD5CB0742F2D1725E
:10D4D00002D0954202D007E0904207D121F002002D
:10D4E000F870F878C00701D0744800E074480190E3
:10D4F000F878C0070CD072485946814600206080F9
:10D50000A08020612080A060E060CDF800B0A2E0A3
:10D510006A48F1E70099594506D04FF400013046BA
:10D52000F8F7E6FF00287DD166493046F8F7E7FFB7
:10D53000002878D10021304606F09EF95FEA000805
:10D540005CD02069401C2061A28802EB0A01A18006
:10D55000217DC90762D000EB8000800006F056F8FC
:10D5600005001BD0E16851B12069401E00EB80002E
:10D57000820028460AF08DFDE06806F093F82069E5
:10D580004FF0000100EB800005EB800040F8146CC8
:10D59000F878C007304602D0022201E0FEE70522FB
:10D5A000F8F73BFE216900B201EB810105EB810137
:10D5B00021F8100CF8784FF00001C007304601D078
:10D5C000032200E00622F8F728FE216900B201EBF1
:10D5D000810105EB810121F80E0C2069002100EB8F
:10D5E000800005EB800040F8088C206900EB80008B
:10D5F00005EB800040F8041CE5600FE0019930461F
:10D600008847F978890705D5B4F904100A180699EE
:10D610008A4226DCA28850441044A0803046494605
:10D62000884701E01DE00BE00146B4F900008142AB
:10D6300002DD3046494688472080A068401CA06033
:10D64000F878400702D54FF0FF3000E00120009944
:10D650004118009105D40398F7F75AFF061E7FF48E
:10D6600059AFB4F90400002802DDA0EB0A00A08045
:10D67000206908B1069801E0B4F904006080CEB1D9
:10D680000098584516D103996A468968096851F887
:10D690002050F878C0F38001039800F0AEFC4DB143
:10D6A0002846494688472080019928468847608057
:10D6B0000120A060009807B0BDE8F08FB3640108B6
:10D6C0009B560108010006002DE9F04FB34D93B0C1
:10D6D000044600216A88F8F7A0FD9DF81710421C47
:10D6E00062F30001820862F34101C00860F3820125
:10D6F0008DF8171020460021AA88F8F78EFD8DF8C6
:10D70000140020460021EA88F8F787FD8DF81500FF
:10D71000204600212A89F8F780FD8DF816000021A7
:10D72000204606F090F8012800D0002083469DF89E
:10D7300017004FF00001C00720460CD006F00CF98E
:10D7400006469DF817004FF00001C007204605D09F
:10D7500006F0C0F804E006F0BDF8F1E706F0FCF8CA
:10D7600081469DF81700C007204602D0F7F750FF0A
:10D7700001E0F7F731FF0C90204600213222F8F744
:10D780004CFD0546204600211022F8F746FDE18AAF
:10D79000284447182046F8F71BF9381AADF834002A
:10D7A000204600211222F8F738FDA18A28444518A6
:10D7B0002046F8F706F9281AADF83C009DF8170046
:10D7C0009DF81680C00701D00DAD00E00FAD00211F
:10D7D000204606F01BF911900021204606F056F86D
:10D7E00010909DF81700C10709D01099A1F51C529F
:10D7F000D13A02D1618C490509D5C10709D11199E6
:10D80000A1F51C52D13A04D1618C090501D44FF025
:10D810000008BBF1000F0CD0C0070AD1B8F1000F0F
:10D8200003D0B8F1010F02D003E0012000E0002096
:10D8300080460027ADF83870BA46B8F1000F3AD0EC
:10D840009DF81700400703D5A0684268521E13E0F8
:10D85000002211E000200B9006A8CDE9009005A958
:10D8600020460C9BFFF71EFEBDF81810BA19114494
:10D870000FB20AF1010A0246A0684068904201DD39
:10D88000002AE7DABAF1000F01D0B81B07B29DF801
:10D890001700C007204602D0F7F79EFE01E0F7F719
:10D8A000B7FE0EA9CDE9005101460FFA8AF33A46B8
:10D8B000404608F06BF89DF81710480703D5A0689C
:10D8C0004068401E00E000208046BBF1000F04D0FD
:10D8D000C80702D12888384428800DF1180AA068AA
:10D8E0004168414546DDB8F1000F43DB01200B9054
:10D8F000CDE9009A424605A920460C9BFFF7D2FDD0
:10D900000746BBF1000F08D09DF81700C00704D1EF
:10D910002888BDF81810401A2880BDF934300C9AB8
:10D9200002A8019380E80406BDF93C0000903B4644
:10D93000424605A92046FEF7F7F8B846099805F0D3
:10D94000B1FE00200990BBF1000F03D09DF8170035
:10D95000C00709D02888BDF818100844BDF8381051
:10D96000314408442880BAE7BDF83810288831448B
:10D97000401AF7E7119942F2D170814202D0109912
:10D98000814202D12046F9F743FB00222B21204699
:10D9900003F0C8FB13B0BDE8F08F00007C37002017
:10D9A0002DE9F74F0546007F93464FF0000AC00768
:10D9B00060D14FF00108EC680026C1467CB9287F91
:10D9C000C0F3C000401E304254D1B9F1000F51D015
:10D9D0000199284688474FF000080446C1460EB911
:10D9E000261E47D0B8F1000F06D0214628465A46D9
:10D9F00090470446B0423DD04FF00108002CDDD0E6
:10DA00002068F8F737FB0006D8D427681FE001210B
:10DA10003846F8F76DFDB0B12FB101213846F8F75F
:10DA200067FD0028CAD1E868A04223D0B0B12846DB
:10DA300000F024FA0246E8680F21006803F072FB48
:10DA4000012817D106E03846F7F762FE0746002F97
:10DA5000DDD1E8E7E8680068F8F7DCFF2846EC600D
:10DA600000F00CFA0246E8680E21006803F05AFB49
:10DA7000012802D05046BDE8FE8FE8680068F8F73C
:10DA8000C9FF296909B1284688470120F3E770B525
:10DA9000426B818C12F0060F06D0C2F34102022ABB
:10DAA00004D0012A05D022E0008D00E0C08C08449B
:10DAB0001CE0B0F92C40468DA2B2B24202D202F56F
:10DAC000B47214B2B0F92830C58C9AB2AA4202D20C
:10DAD00002F5B47003B2301900EBD07040108542EB
:10DAE00001DA681802E0834203DD501881B208B2FF
:10DAF00070BD0844FAE72DE9F34F87B0074680462A
:10DB00006946F7F7A1FD3846F8F7D3FC039038468D
:10DB1000F7F7C3FD06900021384605F0F9FE81466F
:10DB20000021384605F00CFF05460021384605F077
:10DB300031FF06460021384605F0C0FE0290002164
:10DB4000384605F015FF04460021384605F0CEFEA4
:10DB500004F0010104EBD47201EB620100F0010258
:10DB600000EBD07002EB6000491C401C09B200B20F
:10DB70000B2900DB0B218B460B2800DB0B20824698
:10DB80000B2D00DB0B250B2E00DB0B2602980B2840
:10DB900001DA074600E00B27002469E0D8F82800E6
:10DBA00000EBC40104A802F0ECF9BDF910004946ED
:10DBB000484513DCBDF90020B9F10B0F00DB0B2148
:10DBC000511A0844ADF81000BDF91200B0421EDC35
:10DBD000BDF902200B2E07DA314606E0BDF8002021
:10DBE000A2EB0A010844EDE70B21511A08440399FE
:10DBF000ADF81200BDF91400491B891E88421EDBD6
